:020000040000fa
:020000040001f9
:084000000ea9040000000000fd
:020000040000fa
:020000040001f9
:10521c00efc32200007f2400000188000000000082
:10522c000a00070011000700000020000000e00049
:10523c0002003200000002000000000066060200be
:10524c00020000000040da000000fe004440a9000b
:10525c0000ba23000000e000030032002000200010
:10526c00a00188004440a8000000060060832600ce
:10527c00210020001500370062004000e08048004b
:10528c00910188009001ba0062004000e080480063
:10529c00910188009002ba0062004000e080480052
:1052ac000002eb006028e10004003a000059eb001a
:1052bc008301e900fdff3e00040037006128e10096
:1052cc00010032000082eb0005000700910188000c
:1052dc001001ba000200e000e7ff3a0000000500f0
:1052ec00910188008002780062004000e080480054
:1052fc003559ba008301e900080032002559ba007b
:10530c008301e900050032000400e000f4ff3200e4
:10531c0015d9ba008301e900f1ff3a00000006003c
:10532c005a7e040002000000147f040002000000fa
:10533c00ae8e040002000000be8e040002000000cd
:10534c007eab040000000000a8ab040000000000cd
:10535c00f2ab040000000000f6ca040000000000dc
:10536c000000040000000000889fbe00e304400021
:10537c000900a100808f54004a003600e38f5400ce
:10538c0001003e0049002000f20281000200e00012
:10539c0002003200820078000c0037000106220067
:1053ac0003003700908f5400230036008080e80003
:1053bc00110078000000e000faff3a000f003700ff
:1053cc00908f54001c0036008080e800110078009b
:1053dc000000e000faff3a001201780001062200fa
:1053ec0003003700908f5400130036008080e800d3
:1053fc0011007800820f5000faff3a00e802810099
:10540c00890f54000100310009047800080078006d
:10541c00270107000000e00004003a00890f540047
:10542c00200032000804d100f5ff3700081878007e
:10543c001f000700d4ff370011017800920178009b
:10544c0064805100890f500003003100120090005d
:10545c0080087800070037000900410080087800b8
:10546c00920190001300980011007800128814002b
:10547c0009097800910078000100e0000500320075
:10548c00110090000000e000020032000180e800f2
:10549c00010037000000eb00f00289000280e800f8
:1054ac00010037000000eb004f04be0000000600b6
:1054bc000000e000310032008080e90091027800a9
:1054cc00e38f52002d0036000508a3002b003a0094
:1054dc00020381000200e00002003200828f5000c3
:1054ec00040031000208780001038900160037001f
:1054fc0003017800920190000300e00002003200ea
:10550c00818f5100faff390012027800040041002b
:10551c00808f500019003900810f500003003a00b1
:10552c000509420082007800070037000300e00004
:10553c000300320005804000808f51000f003900bd
:10554c009300980011019800110190000200e000f6
:10555c000a00320011804000820f500007003a0010
:10556c00e00522000008eb0011009000110178000a
:10557c009008410010009000900098000000060078
:10558c0000037800800178000002eb000100370076
:10559c008059780084025100820f520009003200b9
:1055ac0064c078000402e8000004e000f8ff3a0050
:1055bc00830078008058eb0005804100808f5000fc
:1055cc00fcff3a0006007800000006008001eb00aa
:1055dc0002003700817178008301e800828f51004e
:1055ec00fcff3a0000000600800078000100370044
:1055fc000000e8001004e000fdff3a00010050003c
:10560c00000006008001780000017800314078002d
:10561c00005978000004e000fcff3a000300780019
:10562c0000000600040037000204e00001003a000c
:10563c00000005000000e80010417800814f510087
:10564c00f9ff3a0000000600800078001106b10056
:10565c00030035009101b10001003c000050a10095
:10566c0000000600800078001104b1000300350032
:10567c009101b10001003c000050a00000000600a8
:10568c00889fbe000004be00d00381000000e00033
:10569c0001003200000001000800e00001003a00a7
:1056ac00c80381000800be00570107000004440035
:1056bc001804e00004003a00c0072200c00389006f
:1056cc000004eb00070037000800be006001070073
:1056dc00000044001004e000010032000058eb0010
:1056ec00c0038900080078004f04be0000000600cb
:1056fc00900178000200e00002003a000308e90083
:10570c00050037008080eb001304e000020032003b
:10571c000308e8009300fb0001007800000006007d
:10572c000200fa00f0bf9f003fb99700ea815700d2
:10573c008f80e900e0b72a00570107000080fa00cb
:10574c0000000600881f780002047800270107007b
:10575c00080040004f047800000006000000fa002a
:10576c00881f7800000478003fb99700ea81570041
:10577c008000780080ba2a000f02070080007800b1
:10578c000000e000020035000040eb0000f478005f
:10579c00010078004f0478000080fa000000060039
:1057ac008001eb0008003700e342780063c2780008
:1057bc008301e80084cf5200030032000080eb002c
:1057cc000400390010000500828f5100f6ff3a00ea
:1057dc000000eb0000000600889fbe0080047800eb
:1057ec000100780002047800890178001100200083
:1057fc00aa020700880f5000010032008004eb0061
:10580c00090078004f04be00000006000000fa00fa
:10581c004fb99700e881570041c3210020bf2a00ef
:10582c00e50107000080fa000000060041c32100da
:10583c00ef02370041c32100130307000000e00012
:10584c000600350041c32100a0002000e80207003b
:10585c008000eb000000e00001003d008080eb00c8
:10586c000100780000000600040037000204e0008c
:10587c000a0032000000e8008100e80010417800c6
:10588c00914f5100f9ff32000081eb00104078007d
:10589c00914f500004003900020037000001eb006a
:1058ac000100370012002000020078000000060002
:1058bc000000e00003003400db160700e10f40009d
:1058cc0001003a000000eb00000006001200fa0094
:1058dc00889fbe008a9fbe008c1f7800020478004f
:1058ec00a0b79f00b1b79f00830078007880570065
:1058fc002b0307000000eb00e0b79f00d8b79f0018
:10590c0000067800dfb49700194578000a80fb0088
:10591c000000ea00cf05de000a00fb0025030700ab
:10592c000000e0001a0032006fb097000000e800a1
:10593c00e0b79f003fb09700120020008000eb0002
:10594c00afb19700030001000004780019030700b1
:10595c00000178000000e000f3ff3a006fb0970000
:10596c00e10f4400070032000000e900e0b79f009f
:10597c003fb0970088007800afb19700030001009a
:10598c00230037000000e900e0b79f00200037003b
:10599c0050c2b300804f5500020032000b04780057
:1059ac00190037000b04e900170037006fb097009f
:1059bc000000e800e0b79f003fb097001200200005
:1059cc008000eb00afb1970003000100800078006d
:1059dc001900fb00808f50000a003200e18f40005c
:1059ec007c0032006fb097000000e900e0b79f0028
:1059fc003fb097000001eb00afb19700030001002e
:105a0c00740037008904e8000804e900e7ff3b0054
:105a1c005fb0970080804500d1b79f0050c2b300a3
:105a2c00804f5500030032000a04e000b5ff3a0035
:105a3c0068003700a2c2b3000040eb00914f110088
:105a4c0003003a000100e800d0b79f000240780044
:105a5c00a0f79f000000eb0080bf9f000b003700f9
:105a6c008fb89700f0ff2700808f500004003200a1
:105a7c006a08b900000041000300400080bf9f008d
:105a8c005fb097000000e800d0b79f00dfb497002c
:105a9c00194478000801fb0003fd2f0003004100ae
:105aac00e90f5000eeff360082007800c0012200a2
:105abc00dcfe07000000e00002003a000044780021
:105acc00020037000900e800d0b79f00b8f79f002c
:105adc0080c6b300804f540005003a00dfb0970039
:105aec00914f14000c003a0066405000070037003c
:105afc00c0c6b300804f540007003a00dfb09700d7
:105b0c00914f140004003a0065404000b0f79f002c
:105b1c000100e800d0b79f005fb097009000fb0039
:105b2c0030022200bffe07000000e00019003a001e
:105b3c006fb097000000e800e0b79f003fb09700ff
:105b4c00120020008000eb00afb1970003000100b1
:105b5c000004780097020700000178000000e000c4
:105b6c00f3ff3a006fb09700e10f440007003200da
:105b7c000000e900e0b79f003fb097008800780074
:105b8c00afb1970003000100020037000000e900ec
:105b9c00e0b79f007c805700580307000000e0002e
:105bac0003003c000c00e000090032000900370043
:105bbc004ff097000004e000010032000c06e800f2
:105bcc005fb097000000e800d0b79f004dff370092
:105bdc00000678000c0078004f0678004f05be00d8
:105bec004f04be000080fa00000006008001eb00ac
:105bfc000200370061f079008301e800828f5100c8
:105c0c00fcff3a0000000600000278000b00370091
:105c1c0001017800924178000304e00002003a0090
:105c2c00040050000000060083cf52000200320036
:105c3c000201e800f7ff37000000e800904278000e
:105c4c000504e000f2ff3a000400500000000600da
:105c5c00000278000700370083cf52000a003200a0
:105c6c000201e800924178000304e000faff3a00d8
:105c7c000000e800904278000504e00004003200c7
:105c8c0001017800f7ff3700040050000000060007
:105c9c0004005000000006001200fa00889fbe00ad
:105cac008a9fbe008c1f780002047800a0b79f006a
:105cbc00b1b79f0083007800788057003802070046
:105ccc000000eb00e0b79f00d8b79f0000067800fb
:105cdc00dfb49700194578000a80fb000000ea0049
:105cec00cf05de000a00fb00320207000000e000d6
:105cfc001a0032006fb097000000e800e0b79f0078
:105d0c003fb09700120020008000eb00afb197006d
:105d1c00030001000004780026020700000178004f
:105d2c000000e000f3ff3a006fb09700e10f440071
:105d3c00070032000000e900e0b79f003fb0970079
:105d4c0088007800afb197000300010023003700f2
:105d5c000000e900e0b79f002000370050c2b300fc
:105d6c00804f5500020032000b04780019003700f8
:105d7c000b04e900170037006fb097000000e80033
:105d8c00e0b79f003fb09700120020008000eb00ae
:105d9c00afb1970003000100800078001900fb00f0
:105dac00808f50000a003200e18f40007c003200ee
:105dbc006fb097000000e900e0b79f003fb097007c
:105dcc000001eb00afb19700030001007400370035
:105ddc008904e8000804e900e7ff3b005fb0970086
:105dec0080804500d1b79f0050c2b300804f550052
:105dfc00030032000a04e000b5ff3a0068003700e7
:105e0c00a2c2b3000040eb00914f110003003a0016
:105e1c000100e800d0b79f0002407800a0f79f0077
:105e2c000000eb0080bf9f000b0037008fb897007d
:105e3c00f0ff2700808f5000040032006a08b90080
:105e4c00000041000300400080bf9f005fb097003e
:105e5c000000e800d0b79f00dfb497001944780029
:105e6c000801fb0003fd2f0003004100e90f500067
:105e7c00eeff36008200780080022200e9fd070068
:105e8c000000e00002003a000044780002003700f5
:105e9c000900e800d0b79f00b8f79f0080c6b30098
:105eac00804f540005003a00dfb09700914f14006a
:105ebc000c003a006640500007003700c0c6b30023
:105ecc00804f540007003a00dfb09700914f140048
:105edc0004003a0065404000b0f79f000100e80064
:105eec00d0b79f005fb097009000fb00f00222003b
:105efc00ccfd07000000e00019003a006fb09700dd
:105f0c000000e800e0b79f003fb0970012002000af
:105f1c008000eb00afb19700030001000004780093
:105f2c00a4010700000178000000e000f3ff3a0034
:105f3c006fb09700e10f4400070032000000e90049
:105f4c00e0b79f003fb0970088007800afb1970092
:105f5c0003000100020037000000e900e0b79f00d9
:105f6c007c805700650207000000e00003003c0045
:105f7c000c00e00009003200090037004ff09700d8
:105f8c000004e000010032000c06e8005fb097004e
:105f9c000000e800d0b79f004dff370000067800e6
:105fac000c0078004f0678004f05be004f04be0071
:105fbc000080fa00000006006200fa00889fbe0014
:105fcc008a9fbe000004be000205780083007800a2
:105fdc0060f92f000f0040007101070088979f00a7
:105fec0099979f000000eb00a09f9f009a457800b6
:105ffc000b80fb000000ea00cf04de0050c2b300af
:10600c0080cf5500020032000904780001003700ef
:10601c000904e9000800e0000b0034001f90970011
:10602c00080178008a0078008f9197000300010026
:10603c0090979f000000e000930032002f9897008b
:10604c0000004400a09f9f000905450050c2b3000a
:10605c0080cf5500040032000b04e000e3ff3a004f
:10606c002f989700890037000000eb00809f9f005d
:10607c00f0979f00e0979f00d0979f00c0979f00dc
:10608c00b0979f00c09f9f0009003700e0f12100ee
:10609c00008050000000400021f12100e100780058
:1060ac004f98970001007000c09f9f000a05e80000
:1060bc001a4478008800fb00e0f1210059fd07002c
:1060cc00800078000000e000f0ff3a00a0c2b300ae
:1060dc00804f54000e003a00bf8897000180e90001
:1060ec00b08f9f0010007800b09f9f000000e00070
:1060fc0005003d000000ea00b09f9f004f989700fc
:10610c000020a000c09f9f000a05e8001000370087
:10611c00b19f9f0009003700bf989700f0ff270040
:10612c00808f5000040032006a08b9000000410062
:10613c0003004000b09f9f000a05e8001a01fb0015
:10614c0003fd2f0003004100e90f5000f2ff360061
:10615c00e0c2b3009a4f1000040032000080eb0044
:10616c00909f9f008a0478001c0037008a04e80086
:10617c00a0c2b300994f100007003a00bf889700e7
:10618c000180e900b08f9f0010007800909f9f0065
:10619c008a84e800110037000000eb00909f9f00fc
:1061ac00090037009f989700f0ff2700808f500060
:1061bc00040032006a08b9000000410003004000ee
:1061cc00909f9f008904e8001901fb0003fd2f003c
:1061dc0003004100e90f5000f2ff3600194478002b
:1061ec008800fb00400522000efd07000000e000c7
:1061fc0002003a0000447800010037008904e800ee
:10620c00a87f9f0080c6b300804f540004003a0062
:10621c00994f14000a003a006640500006003700ff
:10622c00c0c6b300804f540005003a00994f1400cb
:10623c0003003a0065404000a07f9f008904e800fd
:10624c000905e800c8fb2f000f04440060f92f007b
:10625c000f0040008085e800880178001941780023
:10626c00800078000b007800510207000000e0006d
:10627c0005003a00880078000b007800d500070074
:10628c000000e00059ff3d000080eb004f05be0010
:10629c004f04be000080fa0000000600889fbe007c
:1062ac008a9fbe008c9fbe008e1f780081067800ee
:1062bc0083047800000678000288b9000007780093
:1062cc000000e00002003a000001780042003700b4
:1062dc000d00e0004000320000057800c90090007d
:1062ec0069009000808f500004003900090078008c
:1062fc00ac0307000000e00029003500004020003e
:10630c001900600003003a000a0478008005780048
:10631c000b0037000a017800a10020000c00780067
:10632c00e3030700800578000000e00002003a005b
:10633c000a047800020037000c0050000004e8004a
:10634c00c90190006900900003005000880f5000b4
:10635c0002003100000478008005eb000801780091
:10636c008c0078000300780020fe07000806460029
:10637c00080555004900900000004400c004980036
:10638c000b00e0000400320009007800d203070083
:10639c000000e00002003a000a00e000cfff3a00e3
:1063ac000080200019006000020032000900780013
:1063bc00c903070000c02000190060000200320071
:1063cc0049009000e00498000a00570011000900f1
:1063dc000d80d80000017800020078004f0778008b
:1063ec004f06be004f05be004f04be000000060065
:1063fc00889fbe008a1f7800800478000104780012
:10640c0000457800c100900068009000808f50001b
:10641c000400390008007800620307000000e00067
:10642c001500350048009000095878004004980089
:10643c001800780000b8a30004003a0000a8a300dc
:10644c0006003200ea4f550004003a0008007800bc
:10645c00a10307000000e00007003a0000c0200084
:10646c0018006000020032004800900060049800a0
:10647c000a80fb00010037000080eb004f0578001c
:10648c004f04be0000000600889fbe008a9fbe001d
:10649c0000057800810478002d003700c9009000b9
:1064ac0069009000808f50000400390009007800ca
:1064bc003c0307000000e0003500350000402000e0
:1064cc001900600009003200a10020000a007800c9
:1064dc00be030700800578000000e00004003200d5
:1064ec000a0050000004e800040037008005780022
:1064fc000a0078003cfc070000047800c9019000f9
:10650c006900900003005000880f50000200310019
:10651c00000478008005eb00080178008a00780000
:10652c0003007800b1fd0700080545004900900004
:10653c0000004400c00498000b00e000040032008e
:10654c0009007800640307000000e00010003a0026
:10655c001a04e000d1ff3a0000802000190060000e
:10656c0004003200090078005b0307000000e00023
:10657c0007003a0000c0200019006000050032003e
:10658c0049009000e00498000000eb000100370087
:10659c000080eb004f05be004f04be00000006005b
:1065ac000200fa00f1bf9f00010878000080fa0099
:1065bc00000006006900e100040035006d00e100f8
:1065cc00030034000002b10001003200000005009d
:1065dc00100005000400fa00889fbe008a9fbe00d0
:1065ec008c1f780000047800010678007008900079
:1065fc00f800900001005000880890000100500045
:10660c009808900001005000a8089000010050006c
:10661c00b808900001005000c80890008105500097
:10662c000002220090bf9f0000032300a0bf9f0028
:10663c00081090000028a30018003a000b00e0009e
:10664c00160034008b04780009057800e28f5400a2
:10665c00020036002a002000020037000900e0008a
:10666c000b00340058009000c80190000a0178001b
:10667c00ee80570003000100500498000000e00079
:10668c00960032006808900000004500600c9800ed
:10669c008a8454004240a900ebff3c007801900032
:1066ac000200e0000b00340058009000c80190007c
:1066bc008c00780003000100500498000000e000fa
:1066cc008600320068089000f8009000010040003d
:1066dc00600c9800880c90000900e0001500340054
:1066ec0009057800e28f5400020036002a002000d1
:1066fc00020037000900e0000b0034005800900045
:10670c00c80190000a017800ec80570003000100da
:10671c00500498000000e0007000320068089000ff
:10672c0000004500600c98008a8454004240a90087
:10673c00ebff3c00180990000200e0000b00340055
:10674c00e800900058009000c80190000300010080
:10675c00500498000000e0006000320068089000cf
:10676c009808900001004000600c9800a80c900064
:10677c000900e0001500340009057800e28f540090
:10678c00020036002a002000020037000900e00059
:10679c000b00340058009000c80190000a017800ea
:1067ac00ec80570003000100500498000000e0004a
:1067bc004a0032006808900000004500600c980008
:1067cc008a8454004240a900ebff3c003809900039
:1067dc000200e0000d003400e80090001808900062
:1067ec008080400058009000c80190000300010018
:1067fc00500498000000e000380032006808900057
:10680c00b808900001004000600c9800c80c900083
:10681c000900e0001500340009057800e28f5400ef
:10682c00020036002a002000020037000900e000b8
:10683c000b00340058009000c80190000a01780049
:10684c00ec80570003000100500498000000e000a9
:10685c00220032006808900000004500600c98008f
:10686c008a8454004240a900ebff3c0008109000c1
:10687c000028a3001b0032000b00e00019003400bc
:10688c008b04780009057800e28f54000200360072
:10689c002a002000020037000900e0000b00340041
:1068ac0058009000c80190000a017800ee80570053
:1068bc0003000100500498000000e00007003200c3
:1068cc006808900000004500600c98008a84540011
:1068dc004240a90003003400eaff37000080eb00bf
:1068ec00010037000000eb004f0678004f05be009a
:1068fc004f04be000080fa0000000600881f7800dc
:10690c00000478000040eb00005498003800900020
:10691c009040780040c6b30080cf50003d0032005c
:10692c0020003c007140500080cf50007c003200b1
:10693c000d003c006c40500080cf50008f003c009c
:10694c0000c0e90080cf500035003d0050c2b300bc
:10695c0080cf5000740032007c40400080cf50004b
:10696c0086003a002e00370010c6b30080cf5000ce
:10697c002b00320007003c006940500080cf5000d3
:10698c00240032006340400080cf50007b003a006e
:10699c008000370030c6b30080cf500077003a003b
:1069ac001a00370000c7b30080cf50000d003c0028
:1069bc000040e90080cf500016003d0068405000b8
:1069cc0080cf50001600340000c0e80080cf50008b
:1069dc00100032006540400080cf500067003a0044
:1069ec001200370050c7b30080cf500009003200ae
:1069fc006340400080cf50000600320065405000dc
:106a0c0080cf5000460032005c0037008000eb0065
:106a1c006100370008007800770207006200370039
:106a2c0008007800720507005f0037006848900086
:106a3c000004e0005b003a00f8489000c0c6b300c8
:106a4c0080cf5000270032000a003c006440500008
:106a5c0080cf50002b00320000c0e80080cf5000e7
:106a6c00150032006840500080cf500025003a00dd
:106a7c000a00370040c7b30080cf5000210032001d
:106a8c006640400080cf50001e003200694050002c
:106a9c0080cf50001b003a00070037002800900000
:106aac000080e9002004980010007800084c900049
:106abc00084878003b003700280090000080e9006f
:106acc00200498001002780048009000cf80de006f
:106adc000101780082017800009abe000292be008b
:106aec0030003700280090000080e9002004980056
:106afc001001780048009000cf80de000089be00b5
:106b0c0028003700280090000080e900200498003d
:106b1c001000780048049000080878002100370025
:106b2c00110020001c003700480090000000e80015
:106b3c004004980018009000980178001200200082
:106b4c008000eb0003000100800078005002200060
:106b5c00808f50001300320048009000e18f4000fd
:106b6c00080032000000e900400498001800900072
:106b7c00980178000001eb00030001000000eb001d
:106b8c00090037000000e90040049800010078007b
:106b9c00050037008080eb00080078006f030700c9
:106bac0001003700100020004f04780000000600a0
:106bbc00889fbe008a1f78000004780001027800cc
:106bcc00824478000305780070c6b300804f5100f2
:106bdc0021003c0000c0e900804f5100de003d0068
:106bec0072405000804f51004b0132000d003c00b0
:106bfc006c405000804f51005e013c0000c0e90029
:106c0c00804f5100d4003d0050c2b300804f510062
:106c1c00550132007c404000804f510055013a0034
:106c2c00cd00370010c6b300804f5100ca003200af
:106c3c0004003c0069405000804f51004d013a0067
:106c4c007200370030c6b300804f5100180032007c
:106c5c000040e8000900370000c7b300804f510026
:106c6c001e01320008003c0000c0e900804f5100ba
:106c7c00e400320065003c006540500080cf5400b9
:106c8c003c013a000f00370050c7b300804f510051
:106c9c005e00320063404000804f51005b003200c8
:106cac0065405000804f510032013a001a01370004
:106cbc009180e900010a78007800900091717800c9
:106ccc0032013700a8609000c0c6b30080cf5000de
:106cdc000a003a009400780064805000000a7800a2
:106cec001000be004f89de00cf91de000002be0016
:106cfc0002037800820378001300370010c7b3003a
:106d0c0080cf500003003200a0c6b30080cf5000eb
:106d1c0006003a009400780068805000000a780061
:106d2c003002be002003be00070037001480e900cb
:106d3c00000a78001000780000027800cfa2de0074
:106d4c000503780086037800049cbe000694be0000
:106d5c00a860900080c6b30080cf50000e003200b7
:106d6c0020c6b30080cf500005003a000400fb00a1
:106d7c00cf80de0001017800820178000a00370024
:106d8c0040c7b30080cf5000030032006640400083
:106d9c0080cf500006003a0004007800cf80de005f
:106dac000101780082017800009cbe000294be00b4
:106dbc003800be002801be00e00f5000e08f5800e4
:106dcc00e00f5900e08f590003003d00780090005f
:106ddc00d1c2b3000a003700081090000018a300bd
:106dec000300320078009000b1c2b30004003700f9
:106dfc000008a300530032007800900001c2b300d9
:106e0c00017578000000e8004d003700a860900084
:106e1c00c0c6b30080cf500006003a009400780042
:106e2c0064805000000a78001002be006033b80085
:106e3c001300370010c7b30080cf5000030032009e
:106e4c00a0c6b30080cf500006003a009400780032
:106e5c0068805000000a78003002be002003be009b
:106e6c00070037001480e900000a78001000780051
:106e7c00000278000500200006002000070020001a
:106e8c00049cbe000694be00a860900080c6b300af
:106e9c0080cf50000e00320020c6b30080cf5000cf
:106eac0005003a000480fb000100200002002000d5
:106ebc00030020000a00370040c7b30080cf500009
:106ecc00030032006640400080cf500006003a00bc
:106edc0004007800010020000200200003002000c4
:106eec00009cbe000294be00081090000038a30065
:106efc00140032003800be002801be00e00f500024
:106f0c00e08f5800e00f5900e08f59000d0032005f
:106f1c0080c7b30080cf54000300320080c5b3009b
:106f2c0080cf540007003a007800900001c3b300f2
:106f3c00017578008000e80009f578000080e80011
:106f4c0070049800780090000000450060049800e0
:106f5c00894078006d003700a8609000c0c4b30071
:106f6c0080cf500006003a009400780068805000f2
:106f7c00000a78005001be004000be00050037003a
:106f8c009400780064805000000a78001000be0065
:106f9c0022130700009cbe000294be003800900033
:106fac000000e00003003d0078009000d1c2b30067
:106fbc000a003700081090000018a30003003200ec
:106fcc0078009000b1c2b300040037000008a300a1
:106fdc00050032007800900001c2b3000175780002
:106fec000000e80070049800780090000000450054
:106ffc0060049800894078000800780003070700b7
:10700c0064003700a8609000c0c6b30080cf500069
:10701c00250032000a003c006440500080cf500034
:10702c002800320000c0e80080cf5000140032006d
:10703c006840500080cf500022003a000a00370010
:10704c0040c7b30080cf50001e00320066404000a5
:10705c0080cf50001b0032006940500080cf5000a0
:10706c0018003a00060037001480e900000a780086
:10707c0010007800485c9000084878004500370004
:10708c001480e900000a780010027800680890006b
:10709c00cf80de000101780082017800009abe00ea
:1070ac000292be003b0037001480e900000a780011
:1070bc001001780068089000cf80de000089be00c7
:1070cc00340037001480e900000a780010007800c2
:1070dc00680c9000080878002e0037001180e90039
:1070ec008008780010007800cf80de000101780065
:1070fc0082017800009cbe000294be0078009000d3
:10710c00000045006004980081c7b30008007800b7
:10711c00ff0207001f0037001480e900000a780006
:10712c001000780060049800580990000200e000fc
:10713c0002003d002cf90700090037008000eb002d
:10714c005b000700800078000000e00003003200c4
:10715c006800900000805000010037005808900033
:10716c00100c98000b003700780090000275780026
:10717c000600370078009000800045000904e0000c
:10718c0001003a0059c2b300894878000000e800b9
:10719c00700498000000eb004f0578004f04be000f
:1071ac0000000600889fbe0000047800c00190001b
:1071bc00600090008000eb00808f51003900390096
:1071cc00180178002000290000006100e20f500037
:1071dc0007003200002020000200e0000100350012
:1071ec0000202400000c71008080eb002d00370083
:1071fc000100260001006100810f500008003a00d8
:10720c0038009000808f510005003900080078008c
:10721c00310007008080eb000000e00021003a0004
:10722c0000c020001800600017003a00a80490006d
:10723c006002200008004000808f540012003a00c9
:10724c000020200048f807008000780020049800f7
:10725c000000e00005003a00290498004904980059
:10726c000900e80030049800060037001860a00000
:10727c00400498000020b00030049800410c9800a5
:10728c00510c98008a0807002800900050049800c0
:10729c00380090006004980000002600180c700064
:1072ac008000eb00010078004f04be0000000600d7
:1072bc008001eb00040037008301e80090cf100040
:1072cc00040032000000e800828f5100faff3a00ff
:1072dc000000eb0000000600889fbe000004780050
:1072ec000000e0000e003a0080047800c8bf2100c6
:1072fc00180078000000e00004003200f6ff0700e0
:10730c000000e00001003d008084eb000884e800f0
:10731c00c0c02100800f540029003200f4ff370058
:10732c00000022001800600024003200a804900025
:10733c000800370009015000384090000000fb00a5
:10734c00890078004e1007000000e00013003400a4
:10735c008084440048009000808f5400f5ff390071
:10736c0028009000400498001801780000c020000c
:10737c000000610002003200a800900001003700fc
:10738c00b800900000002400000061000a003200e8
:10739c00610498008004eb0009003700280090007d
:1073ac004004980060049800500c98001890a000bd
:1073bc008084eb0002003700510c980080047800a8
:1073cc00090078004f04be00000006008001eb00ad
:1073dc0010417800814f510001003a008001780083
:1073ec000204e000020032000000e800f8ff370061
:1073fc0003007800000006002f02b000889fbe003a
:10740c008a9fbe008c9fbe008e1f7800800478007f
:10741c00600090000000e00001003c00f0ff27003d
:10742c000000e900d0049800c90090000c00330063
:10743c000100e800c0049800190090009901780040
:10744c00120020008000eb00030001000005780012
:10745c00b0022000800f550006003a000b003700e8
:10746c000100e800c00498002cfd2f000f06460018
:10747c001b003700d0022000800f550003003200a3
:10748c002cfd2f000f0646001600370030fd2f0094
:10749c000f044000aad79f00590090000000e9009b
:1074ac00d0049800c90090000a0033000100e800e5
:1074bc00c004980019009000990178001200200077
:1074cc008000eb000300010000057800080678003e
:1074dc00040037000100e800c0049800080678009a
:1074ec000085eb0058e42100390090009000fb006f
:1074fc00080078004bf8070008005000e1e3210079
:10750c00614478008805fb0000032000800f5500c3
:10751c0033003a00590090000000e900d0049800b4
:10752c00c90090000c0033000100e800c004980072
:10753c001900900099017800120020008000eb00e7
:10754c00030001000005780080072000800f550023
:10755c0005003a00070037000100e800c00498005d
:10756c000085eb001b00370080052000800f5500c4
:10757c0018003a000804e00002003200f04f5400fa
:10758c001d003a00590090000000e900d00498005a
:10759c00c9009000090033000100e800c004980005
:1075ac001900900099017800120020008000eb0077
:1075bc000300010000057800030037000100e8001b
:1075cc00c00498000085eb000047eb000b01200085
:1075dc00110037000804e000b80032000600370044
:1075ec000047eb000804e00004003a00ad00200066
:1075fc00084778001c0037001ec0b300ad00200007
:10760c00ea4f540018003200e88f550002003a008f
:10761c008b067800140037006d0120001200370033
:10762c00590090000000e900d0049800c9009000b7
:10763c00090033000100e800c00498001900900014
:10764c0099017800120020008000eb00030001007b
:10765c0000057800030037000100e800c004980022
:10766c000085eb001ec0b30000032000800f550006
:10767c00ebff32000e04e00018003200005e7800d0
:10768c00160037006f805700800f56000100310044
:10769c000a5e7800590090000000e900d0049800c0
:1076ac00c9009000090033000100e800c0049800f4
:1076bc001900900099017800120020008000eb0066
:1076cc000300010000057800030037000100e8000a
:1076dc00c00498000085eb001ec0b300e10f45000c
:1076ec00070032000d0178008a007800d0e42100f8
:1076fc00effe07000000e000e2ff3a0066003700f2
:10770c00490090000000e900c00498000e04e0005d
:10771c0008003a0020fd2f000f004000800f56009b
:10772c005b003a00e10f450059003a008a007800ee
:10773c0065003700004eeb006948900011002000f6
:10774c000004e00060003a0039009000904078009e
:10775c0040c6b30080cf50000300320065404000ab
:10776c0080cf50000a003a000b0178008000eb003b
:10777c0020fd2f000f004000a50707000203be00ec
:10778c000002be0010c0b300805498000d003700fa
:10779c000b0178008000eb0020fd2f000f00400053
:1077ac00f50707000203be000002be0010c0b300c4
:1077bc0080549800b900900000c7b300914f10009e
:1077cc002c003200f9489000c0c6b30080cf5000a6
:1077dc00220032000a003c006440500080cf500070
:1077ec002400320000c0e80080cf500014003200aa
:1077fc006840500080cf50001e003a000a0037004d
:10780c0040c7b30080cf50001a00320066404000e1
:10781c0080cf5000170032006940500080cf5000dc
:10782c0014003a0006003700290090000080e9009f
:10783c00a00498001000780004487800120037006b
:10784c00290090000080e900a00498001000780046
:10785c000498be000690be000b0037002900900073
:10786c000080e900a0049800100078000488be0095
:10787c0005003700290090000080e900a004980062
:10788c001000780004087800110020000e0037006a
:10789c008000eb000c003700490090000000e9006c
:1078ac00c004980019009000990178000001eb00c9
:1078bc008a0078000300010094ff37001ec0b3005b
:1078cc008b00200052ff3700010078004f07780032
:1078dc004f06be004f05be004f04be002f02b10084
:1078ec000000060080017800100037000302e80059
:1078fc00d0c2b300944f100008003a0093cf100090
:10790c0003003e002340900080cf50001200360050
:10791c0063824100630151000300370093cf1000d4
:10792c000d0032000201e90084017800e20f5100e1
:10793c00eeff3e000002eb000400370064c079004b
:10794c000402e800814f500003003200820f520005
:10795c00faff3a000000050010000500f087470010
:10796c00889fbe008a9fbe008c9fbe008e1f780031
:10797c0000047800810678000000eb00c0b79f007f
:10798c00f8489000c0c6b30080cf500002003a0007
:10799c0011002000c1b79f000d00e00023003d0046
:1079ac00b80090000100e80030049800e2c5b30074
:1079bc008041eb0083f79f00904f110003003a00c9
:1079cc000180e8003004980082f79f00b804900012
:1079dc00d0c5b300994f10000200320009007800a6
:1079ec00010037000900e800d10520000df7070061
:1079fc00d0b79f008000eb000000e000bd0032001b
:107a0c0009065000e20f5600080034000c81e90012
:107a1c000900e800d102200025fe070011c0b300c8
:107a2c00c1ef9f000000e00002003a008041eb0033
:107a3c00c3ef9f00680090000000e00004003c00d1
:107a4c00f0ff27000d00e00001003a0010002000bc
:107a5c0050049800684890000004e0000d003a00c3
:107a6c0028009000cfb097000100e0000500320024
:107a7c000080e9002004980010007800b0b79f0047
:107a8c00040037000080e900200498001000780002
:107a9c00f0b79f000045eb005e0037000d00e000e2
:107aac000300340009007800c2fa07001e003700fa
:107abc000d00e0001e003200cfe997000304e00047
:107acc000c003a00380090008ff097000104e000a1
:107adc0004003a000c01780089007800f4fd0700de
:107aec000b0037000c01780089007800f0fd0700ce
:107afc000d003700380090008ff197000304e00070
:107b0c0006003a000c0178008900780075ff070028
:107b1c000000e00006003a006d0037000c01780010
:107b2c00890078006fff07000000e00068003a0051
:107b3c004fb097000000e00009003a006848900040
:107b4c000004e00032003a00ffb09700895878003a
:107b5c00f1b79f0010c0b300005498002c00370000
:107b6c00c9e79f008905fb000b007800010032007b
:107b7c0010002000000578001e0020000000e0002e
:107b8c0016003a000904e00004003a007c8057001b
:107b9c0095f607000005e800100037000e07e90015
:107bac00fc81570063407f008000fb00480190007f
:107bbc00e14f4000070032000200e9004004980049
:107bcc0018009000980178000001eb000300010000
:107bdc00020037000200e900400498008e0f5500a7
:107bec00eeff3500684890000004e00005003a0004
:107bfc003fb097000b187800b0b79f0010c0b300cf
:107c0c0000549800680090000000e900600498009f
:107c1c002ac0b300580090000000e90050049800fe
:107c2c00480190000b0033000200e800400498006b
:107c3c001800900098017800120020008000eb00e2
:107c4c000300010080047800e10f400093ff3a002c
:107c5c00020037000200e800400498004800900041
:107c6c000000e900400498000d00e0000200320022
:107c7c00e24f5500040032000a00fb008080eb004c
:107c8c001c00320010003700684890000004e0002f
:107c9c0009003a00cfb097000100e0000300320069
:107cac00bfb197008009eb00030037008fe8970005
:107cbc007fb09700014878000d00e00002003d0005
:107ccc00dfb1970033049800110020000900370041
:107cdc00480090000000e900400498001800900053
:107cec00980178000001eb00890078000300010086
:107cfc00ddff3700010078004f0778004f06be000b
:107d0c004f05be004f04be000f01b100000006007d
:107d1c00ef02b000889fbe008a9fbe008c9fbe0001
:107d2c008e1f78000006780050e72100c0b79f0036
:107d3c0080c5b30080cf50000800320042e621001d
:107d4c00c2b79f007740400080cf500003003a003c
:107d5c0083002000b3b79f000a00370080c7b30030
:107d6c0080cf500005003200a4002000b4b79f0063
:107d7c0080c5b30080cf500002003a000001200003
:107d8c00b0b79f003c04be002c05be0040c6b3003b
:107d9c0080cf5000030032006540400080cf50007f
:107dac000b003a00e00f5400e08f5c00e00f5d0028
:107dbc00e08f5d0006003d006000b8006011b80067
:107dcc0008045000898458000a0559008b85590015
:107ddc00e00f5400e08f5c00e00f5d00e08f5d0071
:107dec0004003a005c0890008d0120000000e000c7
:107dfc000c003200bfb0970001027800cfa2de0069
:107e0c0005037800860378000800be000a01be0056
:107e1c00221007004fb2970064407800d0df9f001b
:107e2c007d0120003fb0970000027800cfa2de0059
:107e3c0005037800860378000800be000a01be0026
:107e4c000f100700009ebe000296be000d00e90058
:107e5c0061fc2f008f804000008740001e0037001f
:107e6c003fb1970002047800cfc4de00090578000a
:107e7c008a0578000802be000a03be007fa897009e
:107e8c008fb097001fb19700afb197000710070094
:107e9c00d0b79f00e1b79f00f2b79f0083bf9f0050
:107eac008d06e9000802be000a03be00851007001b
:107ebc007faa970000005200cfb09700615778005e
:107ecc005fb09700efb097007fb197008fb9970024
:107edc00009ebe000296be003c00be002c01be00ff
:107eec00f0af9f0081b79f0092b79f00a3b79f0090
:107efc00e00f5000e08f5800e00f5900e08f590060
:107f0c00020034000d00e000d5ff3c00bfb097002c
:107f1c00e88f500010003a000c1090000038a300bd
:107f2c000d003200f78f560006003e0062fc2f0059
:107f3c000f0141008d00410000c3b300914f1000b0
:107f4c00050032008d06e90000c3b30063fc2f006e
:107f5c008f81410080f17e0078811600120e98000e
:107f6c006c00900063fc2f008f8141008d804100dc
:107f7c001ef707001c0990005c089000800f510050
:107f8c0006003d0002005000000e98000c109000fe
:107f9c000040a100001698000f0037000000e00020
:107fac000d003d000c10900074006000f00f5000ac
:107fbc0009003a007c089000fc0090000100500081
:107fcc008c08900001005000020050004240a900b3
:107fdc0001003400000e98004f0778004f06be00d9
:107fec004f05be004f04be00ef02b10000000600ba
:107ffc006f04b000889fbe008a9fbe008c9fbe009d
:10800c008e1f780000047800600090000000e000f3
:10801c0001003c00f0ff27000000e900500498002c
:10802c00c80190000c0033000300e80040049800e5
:10803c001800900098017800120020008000eb00de
:10804c000300010080047800b0022000808f5400ef
:10805c0007003a00090037000300e80040049800cc
:10806c0060fb2f000f0540008084eb0051003700af
:10807c00d0022000808f540015003a0071fb2f00b5
:10808c000f854000e9779f00580090000000e90040
:10809c0050049800c8019000090033000300e80068
:1080ac0040049800180090009801780012002000fd
:1080bc008000eb000300010080047800060037000c
:1080cc000300e800400498008084eb00b500370002
:1080dc0064fb2f000f05420000032000808f54002a
:1080ec0034003a00580090000000e9005004980059
:1080fc00c80190000c0033000300e8004004980015
:10810c001800900098017800120020008000eb000d
:10811c00030001008004780080072000808f540049
:10812c0006003a000a0037000300e80040049800fb
:10813c008084eb00ae00200069013700ae00200007
:10814c001cc0b30080052000808f540065013a00ec
:10815c0000c3b300004d780080c7b30010459800f1
:10816c000a85e800580090000000e90050049800cf
:10817c00c8019000090033000300e8004004980097
:10818c001800900098017800120020008000eb008d
:10819c000300010080047800030037000300e800ae
:1081ac00400498008084eb006e0120000046eb0038
:1081bc004c013700e1062000818f5400030032008f
:1081cc00e0042000808f540076003a008a05780085
:1081dc00815d7800580090000000e9005004980080
:1081ec00c8019000110133000300e800400498001e
:1081fc001800900098017800120020008000eb001d
:10820c00030001008004780010062000808f5400c9
:10821c000300320010042000808f540009013a0042
:10822c0010c6b300804d78008a85e8005800900095
:10823c000000e90050049800c8019000fb003300d6
:10824c000300e800400498001800900098017800a2
:10825c00120020008000eb00030001008004780075
:10826c00e0062000808f540003003200e004200060
:10827c00808f5400f3003a00580090000000e90091
:10828c0050049800c80190000c0033000300e80073
:10829c00400498001800900098017800120020000b
:1082ac008000eb00030001008000780080022000b9
:1082bc00808f500004003a00110037000300e800e2
:1082cc00400498000a003700e18f4000080032009b
:1082dc00480090000000e90040049800180090004d
:1082ec00980178000001eb00030001002b0037001f
:1082fc00480090000000e900400498002700370077
:10830c00580090000000e90050049800c80190004b
:10831c00090033000300e8004004980018009000a6
:10832c0098017800120020008000eb00030001008f
:10833c0080047800030037000300e8004004980034
:10834c008084eb0009007800ed050700000178003f
:10835c000000e000eaff3a00f0052000808f540096
:10836c00e7ff320090022000808f54000b00320097
:10837c00c8019000e18f4400050032000300e900c1
:10838c00400498001800900098017800b500370060
:10839c000300e90040049800cd013700e0c6b300ab
:1083ac00b900370091062000818f5400050032007f
:1083bc00ae0020000046eb0090042000808f54009b
:1083cc00c8003a008a057800815d7800580090005a
:1083dc000000e90050049800c8019000930033009d
:1083ec000300e80040049800180090009801780001
:1083fc00120020008000eb000300010080047800d4
:10840c00e0062000808f540003003200e0042000be
:10841c00808f54008b003a00e0c6b300804d78008a
:10842c008a85e800580090000000e900500498008c
:10843c00c80190007d0033000300e8004004980060
:10844c001800900098017800120020008000eb00ca
:10845c00030001008004780060062000808f540027
:10846c000300320060042000808f540075003a0035
:10847c00580090000000e90050049800c8019000da
:10848c000c0033000300e800400498001800900032
:10849c0098017800120020008000eb00030001001e
:1084ac008000780090062000808f500004003a0075
:1084bc00140037000300e800400498000d0037005a
:1084cc0090042000808f50000e003200e18f40009d
:1084dc0008003200480090000000e90040049800b9
:1084ec0018009000980178000001eb0003000100d7
:1084fc0064003700480090000000e9004004980038
:10850c0060003700580090000000e900500498000b
:10851c00c8019000450033000300e80040049800b7
:10852c001800900098017800120020008000eb00e9
:10853c000300010080047800e0062000808f5400c6
:10854c0003003200e0042000808f54003d003a000c
:10855c00580090000000e90050049800c8019000f9
:10856c00320033000300e80040049800180090002b
:10857c0098017800120020008000eb00030001003d
:10858c008004780090062000808f54000300320095
:10859c0090042000808f54002a003a00580090006c
:1085ac000000e90050049800c80190001f0033003f
:1085bc000300e8004004980018009000980178002f
:1085cc00120020008000eb00030001008004780002
:1085dc0040072000808f540003003200400520002b
:1085ec00808f540017003a00580090000000e900fa
:1085fc0050049800c80190000c0033000300e80000
:10860c004004980018009000980178001200200097
:10861c008000eb000300010080047800900720002c
:10862c00808f540004003a00160037000300e80065
:10863c00400498000e00370090052000808f5400f5
:10864c0010003200e18f4400090032004800900015
:10865c000000e90040049800180090009801780090
:10866c000001eb00890078000300010018013700bd
:10867c00480090000000e900400498008084eb0062
:10868c001301370060c6b300804d7800e305450048
:10869c008006eb000d07780015013700580090009c
:1086ac000000e90050049800c80190000900330054
:1086bc000300e8004004980018009000980178002e
:1086cc00120020008000eb00030001008004780001
:1086dc00030037000300e800400498008084eb009e
:1086ec001cc0b30000032000808f5400ebff32004d
:1086fc000c04e00001003200005d78008a0578006f
:10870c008006eb000d0578001900370030022000c0
:10871c00800f550003003c00895d78000a05e800d5
:10872c00010037008d06e800580090000000e900b9
:10873c0050049800c8019000090033000300e800c1
:10874c004004980018009000980178001200200056
:10875c008000eb0003000100800478000300370068
:10876c000300e800400498008084eb001cc0b300b8
:10877c00e18f44001b0032000e0178008900780064
:10878c00a0ef2100cafa0700800078000000e0008a
:10879c00deff3a00e0022000808f540011003a0006
:1087ac00895d7800580090000000e90050049800a2
:1087bc00c8019000080033000300e8004004980052
:1087cc0018009000980178001200200003000100ae
:1087dc0080047800030037000300e8004004980090
:1087ec008084eb000a00e0001400320033003700f4
:1087fc008d06e900580090000000e9005004980034
:10880c00c8019000090033000300e8004004980000
:10881c001800900098017800120020008000eb00f6
:10882c000300010080047800030037000300e80017
:10883c00400498008084eb001cc0b30000032000af
:10884c00808f5400eaff32000005eb000d00e000c1
:10885c001a003d00805d78008d06e8001700370097
:10886c0030022000800f550002003c00895d78002a
:10887c000a05e800580090000000e9005004980038
:10888c00c8019000090033000300e8004004980080
:10889c001800900098017800120020008000eb0076
:1088ac000300010080047800030037000300e80097
:1088bc00400498008084eb001cc0b300e18f44009e
:1088cc00060032000e01780089007800a0ef21002c
:1088dc0077fa07000000e000e1ff3a000c04e0002a
:1088ec006c003200ea0f570005003a0050062000d9
:1088fc00808f540008003200500420000400370020
:10890c0000072000808f5400030032000005200077
:10891c00808f54005f003a000b057800095d7800e9
:10892c00580090000000e90050049800c801900025
:10893c001e0033000300e80040049800180090006b
:10894c0098017800120020008000eb000300010069
:10895c0080047800b0022000808f540003003200a5
:10896c00d0022000808f540013003a00094d78008b
:10897c000b85e800580090000000e90050049800b6
:10898c00c8019000090033000300e800400498007f
:10899c001800900098017800120020008000eb0075
:1089ac000300010080047800030037000300e80096
:1089bc00400498008084eb000046eb001200370066
:1089cc00580090000000e90050049800c801900085
:1089dc00090033000300e8004004980018009000e0
:1089ec0098017800120020008000eb0003000100c9
:1089fc0080047800030037000300e800400498006e
:108a0c008084eb001cc0b30000032000808f540056
:108a1c00ebff32000c04e00001003200005d780036
:108a2c008a0578000005eb0016003700e70f5500ab
:108a3c0002003c00895d78000a05e80058009000af
:108a4c000000e90050049800c801900009003300b0
:108a5c000300e8004004980018009000980178008a
:108a6c00120020008000eb0003000100800478005d
:108a7c00030037000300e800400498008084eb00fa
:108a8c001cc0b30000fd2f0000804400e90f500013
:108a9c00e6ff3600c8019000e18f44000800320068
:108aac000300e90040049800180090009801780039
:108abc000001eb0089007800030001000200370080
:108acc000300e900400498000c04e00008003a00a0
:108adc0065fb2f000f804200808f550043003a0049
:108aec00e18f440041003a008900780040003700d3
:108afc00804deb0068489000110020000004e0005d
:108b0c003b003a0066fb2f000f004300ea0f5700b2
:108b1c0008003c006169b9008000eb000604070006
:108b2c00f0979f00819f9f00929f9f00a39f9f00a3
:108b3c000c0037006011b8008000eb00fe0307004a
:108b4c00f0979f00819f9f00929f9f00a39f9f0083
:108b5c004269dd00cf91de00e0fa2f000f004000eb
:108b6c00ad04070010c0b300005498007849900081
:108b7c00c0c6b300804f510003003a00280090009b
:108b8c000080e90005003700a8009000c0c4b300c5
:108b9c00804f51000a0032000180e9002004980047
:108bac00100478007f9097008f9897001f9997007a
:108bbc00af999700710d0700008cbe0009003700bb
:108bcc000180e90020049800100078007f92970043
:108bdc008f9a97001f9b9700af9b97000498be003d
:108bec000690be0011002000010037008000eb0051
:108bfc00010078004f0778004f06be004f05be00fd
:108c0c004f04be006f04b100000006008f04b000da
:108c1c00889fbe008a9fbe008c9fbe008e1f78006e
:108c2c00f0b79f0081f79f005001be004000be00ce
:108c3c00f0979f00819f9f00929f9f00a39f9f0092
:108c4c0010c6b3000ff19700804f51001600320090
:108c5c0010c4b300804f510013003200ffb19700d5
:108c6c00530890000000e00003003d00600020006d
:108c7c00d00998000c0037000000e0000a003a0010
:108c8c0070c6b3000ff29700804f52000300320001
:108c9c0070c4b300804f520003003a001000200053
:108cac00ffb29700d00a9800ffb09700c0fa2f00cf
:108cbc000f004000d104070080017800e20f500043
:108ccc0015003a0030002000ffb097009008980083
:108cdc0010c6b3000ff19700804f51000a0032000c
:108cec0064404000804f5100070032000040e80013
:108cfc00804f510004003200e1dd21000040e8000b
:108d0c00804f510001003a0021de2100ffb1970095
:108d1c0063009000160037000000e00018003400db
:108d2c00300020007fb29700100a980010c6b300e4
:108d3c008ff2970080cf52000a003200644040004e
:108d4c0080cf5200070032000040e80080cf520074
:108d5c000400320061de21000040e80080cf5200a8
:108d6c0001003a00a1de21007fb197006200900063
:108d7c00315878003158780011487800c601370016
:108d8c0014c6b3008ff2970084cf52000300320058
:108d9c0010c4b30080cf520013003a007fb097008c
:108dac00600190008200780000c3b3008058780006
:108dbc00ffb29700e102980080c7b3008ff29700d2
:108dcc0084cf52000100320080c5b3008048780087
:108ddc000280e800ffb09700e0009800710090005e
:108dec000080e800f00098000300e00005003a0065
:108dfc00e3979f0064fb2f000f01420003077800ec
:108e0c00a0013700e5de2100e5b79f0010c6b300d6
:108e1c008ff0970080cf50000500320010c4b300d3
:108e2c0080cf5000a7003a00f2df2100e2b79f008c
:108e3c00ffb19700530890001e0220000000e000d4
:108e4c00010035000007e8000e02e800d4b79f00cf
:108e5c006022b8006033b8007f9097008f9897001d
:108e6c001f999700af999700ef0c0700ffb0970080
:108e7c003102be002103be000000e00004003d00f2
:108e8c000400be000601be0003f0a2000200370081
:108e9c000400be000601be00f0979f00819f9f005a
:108eac00929f9f00a39f9f006f91970064015100b8
:108ebc00e2979f00c3fa2f008f8141006a80410026
:108ecc000048eb006b824100c4b79f0031003700b3
:108edc00c201200003002000e5fa2f000f804200a1
:108eec00cd0307007f9497008f9c97001f9d9700e0
:108efc00af9d97000800be000a01be00cf0c070012
:108f0c000006be005fb1970067015100d2b79f0009
:108f1c004240a9000a003400f40c07000002be0015
:108f2c000203be000800be000a01be00f20c0700de
:108f3c00f0979f00819f9f00929f9f00a39f9f008f
:108f4c00cfb1970067804100710020000500370009
:108f5c006f6066004c6add004466de000c06720031
:108f6c00c4eede00e00f5600e08f5e00050034001a
:108f7c008100e900e18f4000f5ff3a000100370065
:108f8c000060eb008100e900fdff3b006700400042
:108f9c00c0b79f00dfb297000500e0000900340065
:108fac006022b8006033b8007f9097008f989700cc
:108fbc001f999700af999700d10c07000000e000b3
:108fcc00c3ff3c0060fb2f008f0040004fb19700a7
:108fdc00010051000000e9008e0f500001003d001f
:108fec00000778000e00e00003003d0073fb2f002b
:108ffc000f8141002c003700800f570005003d0009
:10900c000e80400010409000f3c0b300e74f5000ba
:10901c0001003c008041eb00c4fa2f000f0242001b
:10902c000e0042006a0040008e00780001003700fc
:10903c000000e9008100e90010417800834f5100e5
:10904c00fbff32000107e800efcf510001003a00ae
:10905c000248e8000100e0000300350075fb2f001a
:10906c000f814200060037000e07e8006f90970052
:10907c0064004000e0979f0061fb2f000f814000cf
:10908c008e0041008e017800030037001100fb00b8
:10909c006fb29700e44878008301e9008100e90091
:1090ac000300e000f9ff3d00ffb297005508900067
:1090bc000000e000f3003d000e00e900d00a98002b
:1090cc00f00037007f9497008f9c97001f9d9700ae
:1090dc00af9d97006022b8006033b8000800be0056
:1090ec000a01be00500c07000000e00005003d0026
:1090fc000bf0a200f8979f00899f9f009a9f9f00fa
:10910c00ab9f9f006f909700725927000280b900a7
:10911c00026a28001300200044090700e4005000f4
:10912c00e1979f0015003b00e3801000c0ff2f006b
:10913c00008460000800ea00e0979f007f90970091
:10914c008f9897001f999700af999700e9d4210049
:10915c00070037000808a300030032003902be00e4
:10916c002903be006b0c07000884d100e88444007e
:10917c000800e000f7ff3c001b0037000100e00096
:10918c001d003400c0ff2f0000806000e0979f009e
:10919c00000478006000b8000200200003ff2300e8
:1091ac00e9d42100070037000808a30003003200af
:1091bc003902be002903be00560c07000884d100fa
:1091cc00e88444000800e000f7ff3c000002be0009
:1091dc000203be007f9097008f9897001f9997000d
:1091ec00af999700c00c0700f0979f00819f9f00dc
:1091fc00929f9f00a39f9f00ffb097005109900082
:10920c0060c6b3008ff1970080cf5100040032008c
:10921c006100200060c4b30080cf510002003a000e
:10922c006f929700ea00420001074100f30f5700cc
:10923c00010034003e01200000c3b300e0779f0022
:10924c0075fb2f008f824200b5b79f0033003700ab
:10925c000800be000a01be00f80b07000006be00a5
:10926c00680757004240a9000e0034001f0c07008d
:10927c000002be000203be000800be000a01be00d0
:10928c001d0c07006022b80046782d0077192400c9
:10929c00200c0700f0979f00819f9f00929f9f00da
:1092ac00a39f9f003fb097006804400089002000f6
:1092bc000d003700a4002000050020000c01be00aa
:1092cc00e0fd2f000f004000780307007fa89700f7
:1092dc008fb097001fb19700afb1970004c3b300d4
:1092ec00046441000006be00e00f5600e08f5e00f3
:1092fc00060034008904e900e18f4400edff3a00d8
:10930c000200370000c3b300006478008904e90050
:10931c00fcff3b0068044400b8b79f000e00e0005f
:10932c000b0034007f9497008f9c97001f9d970033
:10933c00af9d97006022b8006033b8000800be00f3
:10934c000a01be00ee0b07000000e000c0ff3c006d
:10935c00c5fa2f008f8242006a804200bfb097008e
:10936c00008050008001e9006f919700e7004100f8
:10937c006b814200010037000201e80000c3b3001a
:10938c00924f1000fcff320074fb2f000f004200c4
:10939c00808040008280500000804100020250001a
:1093ac00e1979f00ffb29700d509900060c6b3000b
:1093bc008ff2970080cf52000300320060c4b300dc
:1093cc0080cf520002003a008100e8000a0037000a
:1093dc0050c6b3008ff0970080cf500005003200cc
:1093ec008000eb0050c4b3008ff2970080cf520086
:1093fc0001003a0011002000018741008e0f52003d
:10940c0001003d00040778000e00e0001d0035004f
:10941c00840f570005003d00e2407f0095c3b30068
:10942c0040c3b30080cf500001003c0005c3b30023
:10943c000e0041008000e9008e0178000100370029
:10944c008100e9008301e90011427800854f520048
:10945c00fbff32000307e80090c3b30080cf52003b
:10946c0001003a008448e8000300e00005003d00dc
:10947c000201e9000e07e8006f9097000000e80079
:10948c00e0979f006f9297008e0178008ff0970005
:10949c007fb09700220307004f0778004f06be00ed
:1094ac004f05be004f04be008f04b1000000060043
:1094bc00881f7800e80722001804e00004003a0036
:1094cc0060af2c004a04070020c0b300004c7800a9
:1094dc004f04780000000600889fbe00000478004e
:1094ec007df707008004780000042000180060005d
:1094fc000200320028009000edef07000000eb00a6
:10950c0020049800384090000004e000050035006d
:10951c000000fb000e0807000000e0000100320014
:10952c008084eb00181090000000e000080032006e
:10953c00100807000000e000010032008084eb00fe
:10954c0018109000daef07000000eb0010149800e0
:10955c000008200018006000100032000000eb0032
:10956c00c1bf2100910f1400070032000000e80079
:10957c008180e800e80f5000faff3a0008007800fc
:10958c00cbef07001300370000004000c1bf2100e3
:10959c00010040000008eb00f8ff3700000c7800d9
:1095ac0000c0eb003044980060022000080040002e
:1095bc00200498004004980050049800400c980037
:1095cc0060049800500c98007004980076004400d9
:1095dc00000c9800090078004f04be000000060043
:1095ec00881f7800a8c02100180078000000e00057
:1095fc0001003200b8ff07000884e900a0bf210079
:10960c00800f5400f8ff3a004f0478000000060069
:10961c000200fa00889fbe008a9fbe008c1f780053
:10962c008005780001057800020678000100e00052
:10963c0001003a006c8557000b04780001003700dc
:10964c000804e800984478000900fb00d9f30700ef
:10965c000000e000faff3a00d0c2b30080cf540003
:10966c000500320000c0e90080cf54000200320037
:10967c0080447800010037000804e8000c017800f1
:10968c008a007800080078003b0007000203be0047
:10969c000002be009a0f540001003a000b0d780036
:1096ac009a8f550005003a00e00f5200e08f5a00e7
:1096bc00e00f5b00e08f5b0014003a00b0c2b30017
:1096cc0080cf540006003a00e00f5200e08f5a00a1
:1096dc00e00f5b00e08f5b0020003d000b003700cb
:1096ec00d0c2b30080cf54001c003a006000b80018
:1096fc0002002000030028000020e10001a8e10086
:10970c0002b0e10003b8e1000e0036002002200098
:10971c00600389006b40400080cf540004003a0085
:10972c006000b80002002000030028000d00370084
:10973c00f0ff2f00f1ff2f00f2ff2f00f3ff2700a7
:10974c00080037006000b8006011b8000402500037
:10975c008582580006035900878359000400be0017
:10976c000601be004f0678004f05be004f04be0038
:10977c000080fa0000000600fc874700889fbe00ae
:10978c008a9fbe008c9fbe008e1f78000007780059
:10979c00810678008204780000047800010037000c
:1097ac000804e800184678000c00fb0081f3070061
:1097bc000000e000faff3a00d0c2b300804f560020
:1097cc000500320000c0e900804f56000200320054
:1097dc0000467800010037000804e8000900e000aa
:1097ec0005003500e18f54000300320040022000d8
:1097fc00808f5400040034000d00e000b0003200f3
:10980c008e0e7800ae0037000900e0000e00340028
:10981c00f08f54001a003a0000c3b300984f1000a8
:10982c0016003a009840900080c7b30080cf5000db
:10983c000300320080c5b30080cf50000f003a0007
:10984c000884e8000e003700a900200000c3b30014
:10985c00984f10000a003a009840900080c7b3005f
:10986c0080cf5000040032008900200080c5b30076
:10987c0080cf500002003a000884e8000901200063
:10988c0008057800010037000a05e80000c3b300a2
:10989c009a4f1000fcff32008a0578006022b80055
:1098ac006033b8002600370090d2210080c05000f1
:1098bc0081ef9f0009027800cfa2de00050378003b
:1098cc00860378000fb097009fb097002fb19700d8
:1098dc00bfb19700fb090700d0b79f00e1b79f000d
:1098ec00f2b79f0083bf9f000fe897000002fb00b8
:1098fc00cfa2de0005037800860378008b05e80014
:10990c000fb097009fb097002fb19700bfb1970091
:10991c00c0af9f00d1af9f00e2af9f00f3af9f009d
:10992c005fb09700efb097007fb197008fb99700a9
:10993c000002420081824a0002034b0083834b00e9
:10994c0084b79f0095b79f00a6b79f00b7b79f003d
:10995c001b00fb0043ef0700800078000901780032
:10996c0090d2210052f60700800078000000e00041
:10997c00cdff3a008b0f54000a003a000d00e000b6
:10998c004f0032008e0e78006022b8006033b800b1
:10999c0084b79f0095b79f00a6b79f00b7b79f00ed
:1099ac004d0037008a80550040d0210060c07c00fb
:1099bc000000fb00008050002c0033004240a90046
:1099cc0020003c008fea97000500fb00cf80de00f2
:1099dc0001017800820178000fb297009fb29700c6
:1099ec002fb39700bfb397000000520081805a003c
:1099fc0002015b0083815b000020e10001a8e10013
:109a0c0002b0e10003b8e1000e0039000902780051
:109a1c00cfa2de0005037800860378001809070042
:109a2c004faa9700dfaa97006fab9700ffab970088
:109a3c000400e1000588e1000690e1000798e100d0
:109a4c000a0032002002200060038900f0ff2f0082
:109a5c00f1ff2f000001be0080b79f0091b79f005f
:109a6c00a2b79f00b3b79f0011003700d0c2b3005c
:109a7c00804f56000e003a006000b8006011b8002c
:109a8c000fb297009fb297002fb39700bfb3970008
:109a9c000402500085825800060359008783590040
:109aac0084b79f0095b79f00a6b79f00b7b79f00dc
:109abc000d00e000080032008b0e78000600370025
:109acc006000b8006011b80080b79f0091b79f008c
:109adc00a2b79f00b3b79f000fb097009fb097003d
:109aec002fb19700bfb197004f0778004f06be000b
:109afc004f05be004f04be00cf01b10000000600b0
:109b0c000003b1000b0035009000b10008003400d8
:109b1c008000b100070035009001b1000400340052
:109b2c007000b100030035009001b10001003c0051
:109b3c0010000500000005002600fa00889fbe00fa
:109b4c008a9fbe008c9fbe0090b79f0001047800d6
:109b5c000206be00800478007e805700b702070022
:109b6c00e80560000030a100e10f50003f003a0012
:109b7c0060fd2f000f0540009fb0970024002000cf
:109b8c008a0178000801780009007800300307008a
:109b9c00800478006000b8006011b8000900e00093
:109bac0029003200424cdd00080045001000be00c8
:109bbc00ce090700e0b79f00f1b79f0082bf9f005e
:109bcc0093bf9f0064045400080545000904780005
:109bdc0069e92100150037001a00be00e00f5000a3
:109bec00e08f58000f003200c00907003902be0098
:109bfc002903be00c70907000002be000203be0015
:109c0c006fb09700ffb097000fb997009fb99700fe
:109c1c008f0a0700e0b79f00f1b79f0082bf9f003b
:109c2c0093bf9f00e8844400640555000804e900d4
:109c3c004240a900e8ff3c006fb09700ffb09700ce
:109c4c000fb997009fb99700f0a79f0081af9f00b5
:109c5c0092af9f00a3af9f0061fd2f000f804000cb
:109c6c0030024600a0824e0042003700e20f500046
:109c7c0046003a0062fd2f000f0541009fb097008f
:109c8c00000278008a017800080178000900780049
:109c9c00d1030700800478006000b8006011b800a0
:109cac000900e00029003200424cdd0008004500ac
:109cbc001000be008d090700a0b79f00b1b79f0030
:109ccc00c2b79f00d3b79f00640454000805450039
:109cdc000904780069e82100150037001a00be005d
:109cec00e00f5000e08f58000f0032007f09070092
:109cfc003902be002903be00860907000002be001f
:109d0c000203be002fb09700bfb097004fb1970071
:109d1c00dfb197004e0a0700a0b79f00b1b79f00b4
:109d2c00c2b79f00d3b79f00e88444006405550078
:109d3c000804e9004240a900e8ff3c002fb097005e
:109d4c00bfb097004fb19700dfb19700f0a79f000d
:109d5c0081af9f0092af9f00a3af9f003fa99700d8
:109d6c00cfa99700e0fc2f000f0040002a0007004d
:109d7c000c02be007fa097008fa897001fa9970028
:109d8c00afa99700a304070013003700e30f50009e
:109d9c0004003a006000b8000200200003ff270016
:109dac0006003700e40f500009003a00f0ff2f00c6
:109dbc00f1ff2f00f2ff2f00f3ff2700f0a79f0009
:109dcc0081af9f0092af9f00a3af9f0006003700aa
:109ddc006000b8006011b800f0a79f0081af9f0031
:109dec0092af9f00a3af9f007fa097008fa8970012
:109dfc001fa99700afa997000b00e00001003200eb
:109e0c0003f0a2004f06be004f05be004f04be007b
:109e1c000080fa0000000600889fbe008a1f7800b0
:109e2c008c9fbe00000478000206be00e6044000d1
:109e3c00190178000200d0004505de008a00780088
:109e4c00f07f2000800f55000c003a006f0061007d
:109e5c0065003a00280090000000e00062003a0023
:109e6c00180090000000e0005f003a001000200095
:109e7c001800e0005d0032005b0037000a00e000d3
:109e8c0007003a00080078000505070080007800fc
:109e9c000000e000020034000a0078005300370094
:109eac006108b9000c0140008d814800e07f200062
:109ebc00800f5100e08f59000d0034001900e000b4
:109ecc0004003d006000b8000200200003ff2f00da
:109edc00030037006000b8000200200003ff2700d9
:109eec00009cbe000294be00100020003f00370012
:109efc00e00f5100e08f590005003400f0002800fd
:109f0c0019006000c410dd00810c700034003700b3
:109f1c001900780001002800010360006f00600048
:109f2c000040a000800c780061015100e0815900d4
:109f3c00c0fc2f00f1ff2f00800f5100818f5900c2
:109f4c000d003d00860c78000000eb00200498000a
:109f5c0010049800000c7800240037008880e8007a
:109f6c00110c7800640044009008780019087800ff
:109f7c00800ceb0070014100f00f4100f7ff340042
:109f8c008202ea00150032008881e800708212001b
:109f9c00980078008508de00130078000400dd00ce
:109fac00008c700064014400930078008508de008a
:109fbc00120078000400dd008089700092007800a7
:109fcc008508de00190078000400dd0000897000af
:109fdc00190078000500de00800c7800990c7300e5
:109fec000080eb0001003700200020004f06be006f
:109ffc004f0578004f04be0000000600889fbe008d
:10a00c00800478006684400000ff27001800600080
:10a01c004401de00f07f2000800f51000e003a005a
:10a02c00800ceb00180478006f0064001c003a00f0
:10a03c00210090000000e00019003a00110090008f
:10a04c000000e00016003a00100020001100e000b3
:10a05c0014003200120037000200e00005003c0042
:10a06c00010078008e040700000178000000e00079
:10a07c0008003c00f00028001800600001fe2300de
:10a08c00010c700020c02f00800c41000080eb0000
:10a09c0004003700800ceb000000eb0001003700df
:10a0ac00200020004f04be00000006000400fa004f
:10a0bc00889fbe008a9fbe008c1f78000006780027
:10a0cc0092bf9f00a3bf9f000404be000401be000a
:10a0dc001fb89700afb89700540507000005be00e5
:10a0ec000001be000800be003a0507001fb997002a
:10a0fc00afb99700000051008180590020069800ec
:10a10c00310698000a8ebe000c0078004f067800cd
:10a11c004f05be004f04be000080fa000000060090
:10a12c000e00fa00889fbe008a9fbe008c9fbe0066
:10a13c00000478000145780002067800830478005a
:10a14c00840678000300e00002003c0019002000a7
:10a15c002c08220060c6b300804f55000e00320060
:10a16c0060c4b300804f55000b00320070c6b300c2
:10a17c00804f55000300320070c4b300804f55006f
:10a18c009c003a00e48f460080003500580890008f
:10a19c00808f56007d003d008d05e80060c6b30041
:10a1ac00804f55001000320060c4b300804f550042
:10a1bc000d003200081090000038a30004003a0093
:10a1cc0058089000808f540001003d00590c9800f5
:10a1dc00580890000b005000500c980002003b00f7
:10a1ec000000eb00500c98000b00e00027003c0036
:10a1fc00180990006800900001c3b3000170790049
:10a20c008201e800130c9800580890000000e00050
:10a21c0003003c00081090000038a3000500320039
:10a22c0068009000e1c2b30001f079000280e80000
:10a23c00100c9800d80890000b00ea00808f50009a
:10a24c0001003d008105ea000b00ea00200c98009b
:10a25c0001804500500c9800890f500001003d0012
:10a26c0080047800390c98006800900098089000e1
:10a27c0001004000090178008c0078005bee0700bb
:10a28c0058089000090050001a00370098089000f8
:10a29c00680090008b8f540018003d0001004000b6
:10a2ac00090178008c00780050ee07001808900027
:10a2bc0000814400120c980009805500200c980075
:10a2cc00580890000000e00003003c0008109000cb
:10a2dc000038a30006003200e8009000e0c2b30092
:10a2ec0080707900380890000000e800300c98006d
:10a2fc0058089000400c9800a60037000100400060
:10a30c000b0178008c00780038ee070018089000dc
:10a31c0000814500120c98008b8454005808900062
:10a32c000000e00003003c00081090000038a3007f
:10a33c000500320068009000e1c2b30001707900a2
:10a34c000200e800100c980058089000890f50008b
:10a35c0001003d008004780068009000980890008f
:10a36c00010040008b004600090178001fee070039
:10a37c001808900000804400100c980058089000b9
:10a38c0009005000200c98008200370070c6b30002
:10a39c00804f55000300320070c4b300804f55004d
:10a3ac0014003a0058089000808f540004003d00bf
:10a3bc00081090000038a30001003a00590c9800d6
:10a3cc00580890000000e900500c980002003b0077
:10a3dc000000eb00500c980070c6b300804f550085
:10a3ec0002003a005ac6b3000b0037005ac4b3003f
:10a3fc000900370010c6b300804f550002003a0028
:10a40c000ac7b3000400370010c4b300804f5500d6
:10a41c0001003a000ac5b3001809900068009000ca
:10a42c003c7079008201e800130c98000c02780053
:10a43c00580890000000e00003003c000810900059
:10a44c000038a30017003200e8009000e0c2b3000f
:10a45c0080f079008280e800110c98005808900078
:10a46c000000e0000f0034008904e900890f50005f
:10a47c0001003d00800478006800900000804000de
:10a48c000901780084007800d8ed070018089000c6
:10a49c0000804400100c98005808900009005000ef
:10a4ac00200c980068009000980890000100400073
:10a4bc000086e8000a587800800078000d00e00063
:10a4cc0004003500b0c2b300804878008c047800da
:10a4dc0004003700d0c2b300804878008c047800a8
:10a4ec008d06ea008005eb000a003700a200200070
:10a4fc008d00780070805700b50307000fb89700e7
:10a50c009fb897007a81550001f17f008b05e80018
:10a51c00800678000d00e000f4ff3c00e18f550050
:10a52c0009003c0050c6b300804f550003003200b8
:10a53c0050c4b300804f550003003a0000c3b30071
:10a54c00005e78008c0478000b00e0000400320000
:10a55c000b00e900fa80570000804000060037002d
:10a56c0000c3b300805c7800050037008b05e90060
:10a57c0002c3b300a05c41000b00e000fbff3c00f9
:10a58c006800900098089000010040000080540082
:10a59c00300c98000810900074006000f00f500010
:10a5ac000e003a00780090009808900001004000de
:10a5bc00a808900001004000b8089000010040007d
:10a5cc00c80890008100400078089000808f5000ef
:10a5dc0002003d0001005000000c98004f06be0028
:10a5ec004f05be004f04be000080fa0000000600bc
:10a5fc0000017800000020000000e000080032009c
:10a60c00000080000000e000050032000000e900be
:10a61c0000008800000040000100800002b07800bb
:10a62c0000000600500381000000e0000100320031
:10a63c0000000100c006220000000600889fbe003a
:10a64c008a9fbe008c1f7800000678008105780078
:10a65c00100578000a047800010037000804e800af
:10a66c00984478000900fb00d2ef070080007800c6
:10a67c000000e000f9ff3a00d0c2b30080cf5400d4
:10a68c0003003a000804e8008200200005003700af
:10a69c00b0c2b30080cf540001003a000804e800b7
:10a6ac000101780098407800e5c6b30085cf5000d2
:10a6bc0003003200e3c4b30083cf500022003a0001
:10a6cc009840900010c6b30080cf500003003200b9
:10a6dc0010c4b30080cf500050003a00a840900046
:10a6ec0085cf500003003200e0c4b30080cf50008f
:10a6fc004a003a006305440080c2b3009a4f100030
:10a70c00020032000a047800090037000a047800bd
:10a71c00d84478000900fb00f9fc07000000e000b9
:10a72c00fbff3a00f0c5b30080cf5400f8ff3200b5
:10a73c004200200090c2b300984f100038003a003d
:10a74c000805e8003600370094c6b30084cf5000eb
:10a75c000300320090c4b30080cf500034003a00a4
:10a76c0018409000854f500002003200834f50007b
:10a77c002a003a00a840900060c6b30080cf500079
:10a78c000300320060c4b30080cf500023003a00b5
:10a79c00630544003200b3009a40780084cf500027
:10a7ac000300320090c4b30080cf50001c003a006c
:10a7bc0048409000854f500002003200834f5000fb
:10a7cc0017003a00d840900084cf500003003200ac
:10a7dc0090c4b30080cf500011003a00e8409000c4
:10a7ec0040c7b30080cf50000300320040c5b30017
:10a7fc0080cf50000a003a00f840900090c7b30098
:10a80c0080cf50000300320090c5b30080cf5000c1
:10a81c0003003a0068054400010037000001eb001a
:10a82c000b00e000040032008a0d780002003700b3
:10a83c000200a000080578000a0e780002007800db
:10a84c004f0678004f05be004f04be000000060006
:10a85c00e4874700889fbe008a9fbe008c9fbe0085
:10a86c008e1f780080bf9f0081047800020778005b
:10a87c00030678006922b900040578008006eb0015
:10a88c00020037008904e8001d00200000c3b3005b
:10a89c00994f1000fbff3200000eeb003c167800c5
:10a8ac000c0478008005eb00280037008a8f5500d7
:10a8bc0016003d0092002000110009008205d8000e
:10a8cc00010078000000e00003003a00640444003a
:10a8dc00000ceb0038147800a200200003002000cc
:10a8ec001800be003b030700194178000201fb0071
:10a8fc00cf91de0000004100818049000003b100cf
:10a90c000180b100008cbe000d003700100020004b
:10a91c00010020001c0e40005c9648008a8f5500f8
:10a92c0008003a0040c3b300994f100005003400f2
:10a93c001000200001002000180c40005894480022
:10a94c008b05e8008904e8001d00200019417800ff
:10a95c000200fb000003b100e90f5000d3ff3600ea
:10a96c008b0f550001003d008a057800e0c2b30052
:10a97c00804f510001003a008904e8000b00e00010
:10a98c0007003200290037000080eb008080eb00cc
:10a99c001c0e40005c9648008904e8001d00200055
:10a9ac0000c3b300994f1000f7ff32008005eb0095
:10a9bc001e0037008a8f55001a003d0092002000bf
:10a9cc00110009008205d800010078000000e000a9
:10a9dc0003003a0064044400000ceb0038147800c7
:10a9ec00a2002000030020001800be00f90207009e
:10a9fc00194178000201fb00cf91de0000004100fc
:10aa0c00818049000003b1000180b100008cbe00c0
:10aa1c008b05e8000080eb008080eb001c0e4000f2
:10aa2c005c9648008904e8001d0020001900fb001a
:10aa3c000003b100e90f5000deff36009200200049
:10aa4c00110009008205d800010078000000e00028
:10aa5c0017003200690510001802be00e00f52000a
:10aa6c00e08f5a00070032004250dd0021ea21003d
:10aa7c00010040001001be000400be00d50207001a
:10aa8c00008cbe008a8545006150b9001c1e100068
:10aa9c001c96180006003700e98555009000200030
:10aaac00010020001c0e40005c9648006404540019
:10aabc00e88f5500040034001800be00e00f500071
:10aacc00e08f5800f4ff32000d00e000330032003c
:10aadc009940780050c6b30080cf5000030032007c
:10aaec0050c4b30080cf50002c003a008900e8001d
:10aafc0011447800b2c2b300824f540005003200fa
:10ab0c00d0c2b300804f54000200320002447800df
:10ab1c00010037008980e800810478008006eb0092
:10ab2c006022b80011003700f00f2e00515f20009a
:10ab3c00800f5200818f5a000a003c00a2002000b6
:10ab4c00030020000400be00a20207000a01fb0063
:10ab5c00cf91de0000024100818249000403b10064
:10ab6c000580b1008904e8001d002000194578001b
:10ab7c000a00fb000003b100e90f5000eaff3600a9
:10ab8c00d0c2b300804f540002003a0060021200a1
:10ab9c00e0821a001c0e42005c964a000e00e00097
:10abac00040032000d00e00001003a008fbc970059
:10abbc00090f780092002000110009008205d800ce
:10abcc004f0778004f06be004f05be004f04be0075
:10abdc004f00b10000000600e8874700889fbe00c8
:10abec008a9fbe008c9fbe008e1f780080bf9f0086
:10abfc008104780002077800030578006722b90009
:10ac0c00040678008006eb00020037008904e80097
:10ac1c001d00200000c3b300994f1000fbff320051
:10ac2c00000deb003a1578000a0478008005eb0063
:10ac3c002c0037008c8f550019003d00720020004d
:10ac4c00811f7800110009008205d80001007800ee
:10ac5c00cf0078000000e00003003a0064044400d8
:10ac6c00000ceb00381478001801be004418dd000d
:10ac7c00cc11de00830170004411dd0060e2210084
:10ac8c000080500001e12100614078000000fb00d1
:10ac9c00cf80de00001c4100019449000e003700fb
:10acac0012002000030020001a0d41005a954900a3
:10acbc008c8f550009003a0060e2210000805000a2
:10accc0001e1210061407800e74f5000030034009f
:10acdc00180c4100589449008b05e8008904e800e1
:10acec001d0020009900fb006201200060e22100a1
:10acfc006ff10700800078000000e000cdff3a0003
:10ad0c008b0f560001003d008c057800e0c2b300ab
:10ad1c00994f100001003a008904e8000b00e00094
:10ad2c00070032002c0037000080eb008080eb0025
:10ad3c001a0d40005a9548008904e8001d002000b7
:10ad4c0000c3b300994f1000f7ff32008005eb00f1
:10ad5c00210037008c8f55001d003d007200200033
:10ad6c00811f7800110009008205d80001007800cd
:10ad7c00cf0078000000e00003003a0064044400b7
:10ad8c00000ceb00381478001801be004418dd00ec
:10ad9c00cc11de00830170004411dd0060e2210063
:10adac000080500001e12100614078000000fb00b0
:10adbc00cf80de00001c4100019449008b05e800a7
:10adcc000081eb008081eb001a0d41005a9549007f
:10addc008904e8001d0020009900fb00620120009e
:10adec0060e2210032f10700800078000000e000f2
:10adfc00d8ff3a0072002000110009008205d8002b
:10ae0c00010078000000e000140032006700100020
:10ae1c004202dd001801be000402e9000300330009
:10ae2c000201410083814900fbff3700028cbe0008
:10ae3c0080854500cf80de001a1d10001a95180081
:10ae4c0006003700e7855500700020000100200047
:10ae5c001a0d40005a95480064045400e68f5500c2
:10ae6c00040034001800be00e00f5000e08f5800c2
:10ae7c00f4ff32001a00be004209dd00ce01de00f4
:10ae8c00830171004201dd00e2b79f00f3b79f0020
:10ae9c00028dbe000d00e0003500320099407800b4
:10aeac0000c7b30080cf50000300320000c5b300d0
:10aebc0080cf50002e003a008900e8001144780041
:10aecc00b2c2b300824f540005003200d0c2b300ae
:10aedc00804f540002003200024478000100370019
:10aeec008980e800810478008006eb006022b800bd
:10aefc0011003700f00f2e00515f2000800f520020
:10af0c00818f5a000a003c00a200200003002000a0
:10af1c000400be00af0107000c01fb00cf91de0066
:10af2c0000024100818249000403b1000580b10098
:10af3c008904e8001d002000194678000c00fb0075
:10af4c000003b100e90f5000eaff3600d0c2b30095
:10af5c00804f540002003a0060021200e0821a0096
:10af6c006fb09700ffb09700041d40000595480096
:10af7c000e00e000040032000d00e00001003a0079
:10af8c008fbc9700090f7800720020001100090097
:10af9c008205d8004f0778004f06be004f05be0053
:10afac004f04be008f00b100000006000200fa0042
:10afbc00889fbe008a9fbe008c1f78000006780018
:10afcc000404be000605be00800078006c805700ab
:10afdc000afc07003c02be002c03be000800be00a9
:10afec000a01be00cb040700009ebe000296be0004
:10affc002fb99700cf91de000c00780086fb07007c
:10b00c004f0678004f05be004f04be000080fa00ca
:10b01c00000006001400fa00889fbe008a9fbe0044
:10b02c008c1f780090b79f00a1b79f00b2b79f000c
:10b03c00c3b79f000405be00e00f5200e08f5a001a
:10b04c008e0032006022b8006033b800760407002e
:10b05c000000e00089003200e00f5500e08f5d0039
:10b06c0042003d0060051500e0851d00dab79f0029
:10b07c00ebb79f006044b8000a0020000bff2300d0
:10b08c006cd92100110037005fb097000008a300b5
:10b09c00070032003c02be002c03be000800be00bc
:10b0ac000a01be009b0407000004be000205be009e
:10b0bc005fb19700efb197008301d1000281d300fb
:10b0cc00d2b79f00e3b79f00680646005fb09700b9
:10b0dc00efb09700e00f5000e08f580003003200f3
:10b0ec0060dd2100800f5600e7ff3a000802be0029
:10b0fc000a03be006000b8000200200003ff23001a
:10b10c00f90407000002be000203be007e80570057
:10b11c00a6ff0700000678000000e00050003d008c
:10b12c005fb19700efb19700e00f5100e08f59002d
:10b13c00520032000204be0034f42600c54a260038
:10b14c008662200087ac20007e80570097ff0700a6
:10b15c00000678000000e00041003d00610454004e
:10b16c00e0845c0041003200f3ff3700e00f550033
:10b17c00e08f5d003a0034006000b800020020004f
:10b18c0003ff2300f0b79f0081bf9f0092bf9f0079
:10b19c00a3bf9f0068d921000a08a3000d0032004c
:10b1ac003802be002803be007fb097008fb897000e
:10b1bc001fb99700afb99700560407000002be00f4
:10b1cc000203be00f4b79f0085bf9f0096bf9f008f
:10b1dc00a7bf9f008b85d1000a85d300e00f5500d7
:10b1ec00e08f5d00040034006804440060dd210041
:10b1fc00800f5400e8ff3a007fb297008fba970097
:10b20c001fbb9700afbb97007e80570067ff0700fe
:10b21c00000678000000e00011003d00e00f550032
:10b22c00e08f5d00150034000a04be00c4f32b004f
:10b23c0035f72700d6fd2400575127007e80570094
:10b24c005aff0700000678000000e00004003d00f3
:10b25c0061045400e0845c0004003200f3ff37000a
:10b26c00000120000c00e00003003200e10f56004a
:10b27c0002003a0080002000600007001fb0970019
:10b28c00afb097003fb19700cfb197004f06780051
:10b29c004f05be004f04be000080fa0000000600ff
:10b2ac0000027800e602400015007800010028003a
:10b2bc00810360006f006000800a780012003a0081
:10b2cc00240090000000e0000f003a0014009000f1
:10b2dc000000e0000c003a00160020001400e00012
:10b2ec003800320008003700e4004200910a780070
:10b2fc000480e8009008780014087800000aeb003d
:10b30c007003530001003700160020001500e00008
:10b31c00f5ff32001300370064014200800040004a
:10b32c00120078004f00de00808a70008481e800f3
:10b33c009200780081804000130078004f00de00fe
:10b34c000089700093007800818040001400780020
:10b35c004f00de008089700014007800000a400065
:10b36c000603e90015007800ef0f5000eaff3600e5
:10b37c00100037000481e8009400d100120078001e
:10b38c004f00dd00008a7000e40042009201d10001
:10b39c00110078004f00dd00008971001101d1000f
:10b3ac00150078004f00dd0080087100950ad1006f
:10b3bc000603e80015007800ff0f5000edff3e007b
:10b3cc00ef0a6000958a7300060078000000060002
:10b3dc0002027800809fbe00110009008200d80094
:10b3ec00000178004f00be0002a2b900848050001a
:10b3fc001100980002087800000006008000780018
:10b40c006500600003003200100220006003890018
:10b41c00000006007880600002003200200220004c
:10b42c006003890000000600889fbe00800478003d
:10b43c000008e20004003a000000eb005600070090
:10b44c000000e0000a003500004080000900e00028
:10b45c0002003a000004780006003700000478006f
:10b46c00090040004c0007000000e00001003d0016
:10b47c000084eb00080078004f04be0000000600ba
:10b48c000a00fa0080017800e20f500025003e000f
:10b49c0070b48000e10f50000800320080232000bf
:10b4ac000000e000050032000423200025232000ca
:10b4bc00462320008001780004003700042220007d
:10b4cc0025222000462220008322200014409000d8
:10b4dc000004e000030035008009eb0000002800a8
:10b4ec00140a7000154090000028a30001003a00d7
:10b4fc0015a0a0008001eb0007003700154090005c
:10b50c000008a300fdff320063c078000000fb00c0
:10b51c00000b78008301e800828f5100f7ff3a009e
:10b52c000800370030002000b0bf9f00c3bf9f0051
:10b53c00d1bf9f00e2bf9f006a80570000c0da00b5
:10b54c006fb99700020078000080fa000000060036
:10b55c000a00fa0011002000b1bf9f00c0bf9f007d
:10b56c006a80570000c0da004fb897000080fa00dc
:10b57c00000006000a00fa0051002000b1bf9f0035
:10b58c00c0bf9f006a80570000c0da005fb8970008
:10b59c000080fa0000000600800078000000e00047
:10b5ac0004003a0060082200004088000101780085
:10b5bc00060037000081eb00e0c32200808f5000b2
:10b5cc0002003e00014088000001eb000200780000
:10b5dc0000000600020ab900001bb9000200b80006
:10b5ec008100420081004300000006006022b80088
:10b5fc00060220000000d0008180d2000482d2001c
:10b60c008582d2000000a0000202520083825a0000
:10b61c00030031000202420083824a000000a100b4
:10b62c000603e900f3ff3a0000000600839f680060
:10b63c000100e00002003d0060001000e0801800f6
:10b64c000300e00002003d0060011100e0811900e0
:10b65c00e6ff07004f00e00002003b006000100016
:10b66c00e080180000000600889fbe008a9fbe0084
:10b67c00010578000100e0000400350008003c00e2
:10b68c000000e000200032000500370060001000d0
:10b69c00e080180002003b0001f02c001a0037007b
:10b6ac000004be006011b8006b0920000982cf00b5
:10b6bc00020039000882cf000441b00069425200f8
:10b6cc000e00320008003b008281710061016400b1
:10b6dc008904d1000884d3008b05e8000442e800fb
:10b6ec00f9ff3a00050037000804440089844c0037
:10b6fc008b05e9000442e900fbff3a00f400070067
:10b70c000af0a70001f0a0004f05be004f04be00d8
:10b71c000000060003f0a200889fbe008a9fbe00b6
:10b72c008c1f780010010700170133006450e100f2
:10b73c004f0032006420e1005200320003826c00a2
:10b74c0007003b000905d0000306d000820f54000f
:10b75c000c065d00020039000200320089017800fd
:10b76c00030678008582550004003d000003fd00af
:10b77c008103fd008502ea008b854200840f720074
:10b78c0002003b0060001000e08018006011b8005f
:10b79c000005eb007a28e1000a0039000600780069
:10b7ac00c75ddd00f707b200878075002d003700fc
:10b7bc00828171000a017800610560008180d100ee
:10b7cc000080d3008502e900f9ff3b00060440002d
:10b7dc008784480002003b0060041400e0841c00d5
:10b7ec000988a300070032008a81710082817100f0
:10b7fc00610164008904d1000884d3008b05e80042
:10b80c00170037000978a30013003a000b00e00082
:10b81c00130034008b05e9000804440089844c00b3
:10b82c000a4474000978a3000d003a000b00e000f4
:10b83c00070034008b05e9000804440089844c009f
:10b84c0001003a000b0020000978a300f7ff32003a
:10b85c000001eb0002003700828171000a017800c0
:10b86c009b0007000cf0a70001f0a000cf003700f0
:10b87c006420e10002003a00838f6c00cf0033009b
:10b88c000801be000200be00c8003700889fbe0041
:10b89c008a9fbe008c1f7800b3000700ba003300eb
:10b8ac0003866c006450e1002e0032006420e1003d
:10b8bc00330032006150e1002f0032006120e100c2
:10b8cc003100320085855500eb07b00009002000df
:10b8dc0008042000050037000804440089844c004b
:10b8ec000a0031000603430087834b00000153001c
:10b8fc0081815b00f8ff33000203be000800a0004a
:10b90c000804440089844c00f6ff3900c639dd0078
:10b91c008301730001003200130020008904d10060
:10b92c000884d3000998a300050032000800a70082
:10b93c000300a0008904d1000884d3008b05e80023
:10b94c008904d1000884d3000001eb000281d200ed
:10b95c005f00070001f0a1000cf0a70001f0a000af
:10b96c00920037006420e100940032000801be0010
:10b97c000200be00f7ff37006120e1008f003200ab
:10b98c006000b800f3ff37000000200001f827002a
:10b99c00f0ff3700889fbe008a9fbe008c1f780086
:10b9ac00710007007800330003866c006450e100de
:10b9bc00240032006420e100270032006150e100d5
:10b9cc00220032006120e100210032008b85420010
:10b9dc00eb07b1000134b800003ab800080442008b
:10b9ec0089844a00013ab8000030b80088804000d1
:10b9fc0009014a0004003300000040008180480027
:10ba0c00020149008b05e900c909dd0083017000c2
:10ba1c000100320013002000c814de004814dd00c1
:10ba2c004709de001200b200c808de00088470006e
:10ba3c002700070001f0a1000cf0a70001f0a00006
:10ba4c005a0037006120e1005c0032000801be00a2
:10ba5c000200be00f7ff37006150e100fcff3a0026
:10ba6c00560037000001be00570007000470a70005
:10ba7c0003f0a10003f8a30013003a006509b1001c
:10ba8c0010003200090035006928e1000200350081
:10ba9c0001002800000005000000400081804800e3
:10baac008502e900fcff3a0000000600f88f420016
:10babc00050035008100d1000080d3008502e8002c
:10bacc00fcff3a00000006008000eb0000000500bf
:10badc0081002000618055000b003d000b00200010
:10baec0061fe2f000100e1001d0034008281710015
:10bafc00610164008904d1000884d3000000e800cf
:10bb0c00faff3a007100200061006400030070002d
:10bb1c00020060000900320061044400e0844c0023
:10bb2c000988a500050032008b05e8006808e100d3
:10bb3c0002003a008904d1000884d300f20f2000df
:10bb4c000258e10005003d00c75ddd00f907b200b9
:10bb5c008980750008007800000006000bf82700ab
:10bb6c008b007800000005000004be0016000700e2
:10bb7c000003be000405be000200be001200070058
:10bb8c00844f7500000006000200be006450e10006
:10bb9c00050036006420e100020036000968a300ad
:10bbac0001003a000800be000160a0004f067800ba
:10bbbc004f05be004f04be0000000600f0ff2f0032
:10bbcc00f1ff2700f9ff3700c70ade00f107b200ca
:10bbdc00f50fb20008003200e1cf42000200320043
:10bbec000170a00024000500810f700001003200dc
:10bbfc000408050044000500810f700002003a00a3
:10bc0c00140005008502e9000000400081c04800d6
:10bc1c00fcff3b000170a0002400050081037800ac
:10bc2c00e9ff07000001be006000b8000478a30023
:10bc3c0013003a006220e10015003e000d003900af
:10bc4c008301d1000281d3008180d3008301d10014
:10bc5c000281d3008180d3008301d1000281d30003
:10bc6c008180d3000538b000c42add00f300b20097
:10bc7c008381720007f0a70003f0a000000006000b
:10bc8c00f3ff2700f2ff2f006110b900fbff370014
:10bc9c0003ff2700f7ff3700881f780000047800a7
:10bcac005001be004000be000400400085804800ea
:10bcbc000601490087814900009cbe000294be0029
:10bccc000400e1000588e1000690e1000798e1001e
:10bcdc0002003100680044001008e8004f047800ae
:10bcec0000000600f4874700889fbe008a9fbe00b4
:10bcfc008c9fbe008e1f78000205be000004be00a3
:10bd0c00d4b79f00e5b79f00f6b79f0087bf9f0091
:10bd1c000000eb00c0b79f00b0b79f00a0b79f001a
:10bd2c0090b79f0080b79f000d042000bfb0970014
:10bd3c004fb09700000140000000e0000f003d00f4
:10bd4c004f08de0000007100c0b79f009e00070086
:10bd5c0001003d0012002000a100070001003d0081
:10bd6c0012002000a6000700b1000700b600070073
:10bd7c000f004000c8ff0700220037004f08de000c
:10bd8c0000067100ccb79f008f00070001003d003a
:10bd9c00120020009200070001003d00120020005c
:10bdac0097000700a20007000fb297009fb2970000
:10bdbc002fb39700bfb39700a900070000005200f3
:10bdcc0081805a0002015b0083815b0080b79f0079
:10bddc0091b79f00a2b79f00b3b79f000007eb007d
:10bdec009f0007000020e10001a8e10002b0e10083
:10bdfc0003b8e100010031001e0020000e005600c7
:10be0c00c0b79f004fb297000400e0000700350058
:10be1c0010002000010020006011b8000804700020
:10be2c00898470000a0571008b8571008d06e9000c
:10be3c00beff3a000400e00003003d008200070052
:10be4c000f00400094ff07004fa897000000e0008f
:10be5c0004003a000fb497009fb497002fb59700d9
:10be6c00bfb59700940007004f0778004f06be003f
:10be7c004f05be004f04be004f01b100000006008c
:10be8c00881f780018002000881f780095ff070095
:10be9c008f87e9004f04780000000600801feb003c
:10beac0090ff07008f87e90000000600889fbe0006
:10bebc008a9fbe008c1f78006e00070007003d00b3
:10becc0073000700e00f5b00e08f5b0007003d0094
:10bedc00320007000006eb000400370034000700b6
:10beec0002003d002a0007001c0020007200070021
:10befc00e3ff07000203be000002be000c00e000de
:10bf0c0001003200220007000400be000601be0042
:10bf1c004f0678004f05be004f04be00000006001f
:10bf2c00889fbe008a9fbe008c1f780051000700be
:10bf3c0005003d0056000700e00f5b00e08f5b0042
:10bf4c0006003d00040037001900070003003d0007
:10bf5c006000b8006011b800100007005600070020
:10bf6c00ceff07000203be000002be000c00e00082
:10bf7c0001003200060007000400be000601be00ee
:10bf8c004f0678004f05be004f04be0000000600af
:10bf9c006000b8006011b8000000370004025000c7
:10bfac00858258000603590087835900000006005b
:10bfbc000006eb00e00f5200e08f5a00e00f5b0030
:10bfcc00e08f5b00000006000180400090b79f00ee
:10bfdc000001eb008fb097000100e00000000600ac
:10bfec000200700090b79f000180400080b79f0056
:10bffc000001eb00ffa897000100e0000000060024
:10c00c000200700080b79f00018040006faa97006b
:10c01c00cf20de0001007000f0af9f000402420050
:10c02c00250007004f18de00000272000000060019
:10c03c00e4af9f000804440089844c000a054d00bd
:10c04c008b854d00000006003fb29700cfb29700e1
:10c05c005fb39700efb3970000fe2f0000000600bf
:10c06c003fb09700cfb097005fb19700efb197004a
:10c07c00000006000205be000004be00e00f5000e8
:10c08c00e08f5800e00f5900e08f590000000600c7
:10c09c006000b8006011b800080450008984580092
:10c0ac000a0559008b8559001c002000e00f520036
:10c0bc00e08f5a00000006000800be000a01be0016
:10c0cc0000000600889fbe008a9fbe008c1f78006f
:10c0dc000205be000004be000006eb00e00f50009d
:10c0ec00e08f5800e00f5900e08f590007003d0029
:10c0fc006000b8006011b800080450008984580032
:10c10c000a0559008b8559001c002000e00f5200d5
:10c11c00e08f5a00e00f5b00e08f5b0002003d00f7
:10c12c000f0007000c00a2000800be000a01be00b0
:10c13c00c40107000203be000002be000c00e000b8
:10c14c0001003200060007000400be000601be001c
:10c15c004f0678004f05be004f04be0000000600dd
:10c16c006000b8006011b8000402500085825800cd
:10c17c000603590087835900000006001400fa00da
:10c18c00889fbe008a9fbe008c9fbe000005be002b
:10c19c000206be00680047000c90be000a90be006c
:10c1ac00ca0107006400e1001a00320016003e00cc
:10c1bc006100e1001a0032006e049000fe04900051
:10c1cc000e0b90009e0b90006011b8009e05900025
:10c1dc000b38b100d501200082817100610164002f
:10c1ec008703d1000683d3008984d3000884d3004d
:10c1fc008502e900f8ff3a0035fe07000df0a700b4
:10c20c0001f0a000ec013700f1ff2700f0ff2f0038
:10c21c00e901370001f8270000002000f7ff370084
:10c22c006000b800f5ff37008f1fd100e701070051
:10c23c008f87e9000000e000000006001400fa00ff
:10c24c00889fbe008a9fbe008c9fbe000004be006b
:10c25c000205be00680047000a90be000890be00b0
:10c26c009a0107000070a7000bf0a10030432000da
:10c27c009e02900080825200b0fe2f000028e10048
:10c28c0011003d00b0fc2f000028e1001500340027
:10c29c001e0990008e0890007e0090000501b000f1
:10c2ac000201d1008180d3000080d3008502e80018
:10c2bc00fbff3a000b00e000bf013b0060001000e8
:10c2cc00e0801800bc013700f0ff2f00f1ff2700c1
:10c2dc000b00e000b8013b0001002800000020002a
:10c2ec00b50137006000b800b30137004f89de009c
:10c2fc0082017800de01370007f0a200d40037007d
:10c30c00809feb00b10107008f87e9000000e0007f
:10c31c00000006002800fa00889fbe008a9fbe001d
:10c32c008c9fbe0003866b008f0107000028a300c2
:10c33c0064003a000128a30067003a000008a3003b
:10c34c0062003a000108a30065003a001e0090004c
:10c35c00be08900081064000ed3fb100f48057000c
:10c36c00ee019000111ab8008e099000311bb80034
:10c37c009e099000311cb800511db800f48557007f
:10c38c0046000700fe0190003a0007008b85e8008c
:10c39c003e0007008e09900040000700ee0190005f
:10c3ac00340007008b85e800380007008e099000e8
:10c3bc00400007009e0990001b18b800890440003b
:10c3cc000a854800fe019000340007008b85e800c8
:10c3dc0038000700ee019000300007008e09900035
:10c3ec001b18b800890440000a8548000a98a3006d
:10c3fc0008003a000402420085824a0006034b0002
:10c40c0087834b0008044c0089844c000a054d00be
:10c41c008d06e90084827200850273004c3add00bf
:10c42c00850272000100320015002000443ade0043
:10c43c001400b2004538de00cb45dd000b00700067
:10c44c00c540de00cb4ddd008b8070004549de0021
:10c45c00cb55dd000b017100c551de000d037800da
:10c46c00ba01070003f0a1000cf0a70003f0a00034
:10c47c00510137001b18b8008502400006834800a4
:10c48c00e0834b0060044c00070037001b18b80019
:10c49c000603400087834800faff37001b18b800da
:10c4ac008703400008844800e0844c0060054d0080
:10c4bc00000006001b18b8000804400089844800de
:10c4cc00faff37000108a30038013a005800be00fb
:10c4dc005801be00e3ff37000008a30033013a0007
:10c4ec0009047800f9ff37002800fa00889fbe0085
:10c4fc008a9fbe008c9fbe0003866b001a0107004a
:10c50c006400e100440032006408e1004a0032009b
:10c51c006100e100460032006108e1004900320090
:10c52c00ec0647006000b8003d02be003d03be00b3
:10c53c00f48657006011b8003d04be003d05be00f6
:10c54c007d0320000b0037000000a0008d06e900e1
:10c55c00130032000402420085824a0006034b009d
:10c56c0087834b0000004000818048000201490095
:10c57c00838149000802520089825a000a035b0039
:10c58c008b835b00f0ff3b000802420089824a006b
:10c59c000a034b008b834b008d06e900edff3a003c
:10c5ac008482720086827200f707b2008782720062
:10c5bc0001003200150020001e0490003e0b90007c
:10c5cc0006035400e63fb0000368a30007003200e6
:10c5dc000000a7000500a0008301d1000281d30058
:10c5ec008180d3000080d3000603e8008301d100d2
:10c5fc000281d3008180d3000080d3000002eb00c5
:10c60c000482d2005101070003f0a1000cf0a70036
:10c61c0003f0a000e8003700640247006408e10062
:10c62c00e20032003400be003401be00f6ff3700d9
:10c63c006108e100dd0032006011b8006000b80054
:10c64c00f1ff370003ff270002002000fbff37003b
:10c65c002800fa00889fbe008a9fbe008c9fbe00f7
:10c66c0007067800878669000c003b0003047800fd
:10c67c008704780008f0a10009f0a100840f500095
:10c68c00858f5800860f5900890f5c00030033001a
:10c69c000cf0a20001003a000cf0a100b20007005f
:10c6ac006400e1005f003200780147006408e1009b
:10c6bc00610032006c014700748557003200be00e7
:10c6cc001201be003a04be001a05be001e03900003
:10c6dc00be0a90008503530006003d000004fd00d7
:10c6ec008104fd000205fd008305fd008703ea00bf
:10c6fc00050378000df8a300040032006004140058
:10c70c00e0841c0060051d00e0851d006022b8005f
:10c71c007d0320000d38e1008006eb000b00390092
:10c72c004433dd00f300b20083017300390037009d
:10c73c00848272000d027800e10664008b85d100c2
:10c74c000a85d3008984d3000884d3008703e900c9
:10c75c00f7ff3b0008004000898048000a014900af
:10c76c008b81490004003b0060001000e080180041
:10c77c0060011900e08119000358a3000900320080
:10c78c008d82720084827200610260008301d1008c
:10c79c000281d3008180d3000080d3000603e8001f
:10c7ac001b0037000348a30017003a000600e00006
:10c7bc00170034000603e9000d00a3000000480038
:10c7cc008180480002014900838149000348a3008d
:10c7dc000f003a000600e000090034000603e900ef
:10c7ec00000040008180480002014900838149001b
:10c7fc0001003a000003eb000348a300f5ff3200f0
:10c80c006022b800020037008482720061826600e8
:10c81c00ce00070003f0a1000cf0a70003f0a0006d
:10c82c0065003700640147006408e10002003a002b
:10c83c000df8a3005d003a003200be001201be00ec
:10c84c005d003700889fbe008a9fbe008c9fbe0093
:10c85c000404b8000506b8008904460060854e0043
:10c86c000606b8000a054600e0854e000706b8002b
:10c87c008b054600040eb800890446000a854e005c
:10c88c00e0854d00050eb8000a0546008b854e006c
:10c89c00060eb8008b0546000416b8000a054600c3
:10c8ac008b854e000516b8008b054600041eb8009b
:10c8bc008b0546000800be000a01be004f06be00f4
:10c8cc004f05be004f04be0000000600800078003b
:10c8dc005002be005003be004439de00f700b20027
:10c8ec00f37f200003016100090032000218e1000f
:10c8fc0016003a0085017200830173008381730076
:10c90c000008200015003a004000200013003700fa
:10c91c0085017200830173008381730005003a0066
:10c92c0004a8be0006a8be00100020000b003700b3
:10c93c000201e9000402420085824a0006034b0012
:10c94c0087834b000748a300f9ff32000740a00083
:10c95c0004a8be0006a8be0020002000800098009d
:10c96c009200980000000600680447000294be0084
:10c97c000094be00fc0447008694be008494be0064
:10c98c0009007800d1ff070008007800cfff0700ee
:10c99c0099007800814f70000b003b000800be002e
:10c9ac00960007004f00b10003003700f3ff27008b
:10c9bc00f2ff2f006110b9004f06be004f05be00fc
:10c9cc004f04be000080fa0000000600889fbe00e5
:10c9dc008a9fbe008c9fbe000404be000605be00ec
:10c9ec00809fbe00829fbe00920007000406780064
:10c9fc000800be000a01be008e0007008406780005
:10ca0c004f03be004f02be008d4f76007fb09700e3
:10ca1c0013003300f0ff2f008b8f6b0006003b00e0
:10ca2c000d0666000c00a7000a00370007f0a600f0
:10ca3c00100020000a003700880f5200898f5a001e
:10ca4c008a0f5b008b8f5b00030039001000200005
:10ca5c0001003e000000200007f0a7000000ea00e3
:10ca6c004f06be004f05be004f04be00000006007e
:10ca7c00889fbe00830478000300e0002c00350082
:10ca8c0003003c000082700004027100260032009a
:10ca9c0036432000c50020008383cf000a003900f4
:10caac000541b1008283cf00070039000541b10078
:10cabc008183cf00040039000541b1008083cf0091
:10cacc00010039000541b10085c353006022b80054
:10cadc00120032000a003b00848272006102600086
:10caec008301d1000281d3008180d3000080d30068
:10cafc000603e8008743e800f7ff3a000700370019
:10cb0c0000004000818048000201490083814900f7
:10cb1c000603e9008743e900f9ff3a000b00070020
:10cb2c0009f0a70003f0a0004f04be0000000600af
:10cb3c0060001000e080180060011900e08119000d
:10cb4c00d3ff3b00033e2c00f7ff370018002000fa
:10cb5c0057002000080453000d003d000600200083
:10cb6c0097fc2f000740e1001e0034008482720005
:10cb7c00610260008301d1000281d3008180d30067
:10cb8c000080d3000804e800f8ff3a0047002000ba
:10cb9c006104600005047400040464000d0032009c
:10cbac0061004000e080480060014900e0814900dc
:10cbbc0003b8a500070032000603e8006538e10061
:10cbcc0004003a008301d1000281d3008180d3009c
:10cbdc000080d300f87f20000830e100030035000e
:10cbec00080378006000b8006011b8004433dd0021
:10cbfc00f300b2008301730000000600e4824000e1
:10cc0c001078a30007003200640240001178a300e2
:10cc1c003400be001401be00040032000330a70033
:10cc2c00000006003500be001501be000330a00058
:10cc3c000000060005ff2700058261000700320096
:10cc4c000428e10001003200240005000600070062
:10cc5c0001003a004400050004080500020007002a
:10cc6c00f9ff3a00140005006f8261008102700028
:10cc7c00850271008502720000000600a110880078
:10cc8c00b01088000000060016a2a9001682a800a9
:10cc9c000000060017e2a9009a20a9009a40a900fa
:10ccac008a20a9008a40a9000000060016c2bf0015
:10ccbc000008a300fdff3a0016c2bf000028a30025
:10cccc00faff3a0016c2bf000038a300f7ff3a0083
:10ccdc0016c2bf000048a300f4ff3a0019c2bf00ff
:10ccec000068a300f1ff3a00000006001662a800dd
:10ccfc0016c2bf000038a300fdff3a0018c2a900fd
:10cd0c00801080000080fb00000006000080fb000b
:10cd1c009010880018c2bf0001c8b3000140600029
:10cd2c000080fb000000e9004f00de000000e9007d
:10cd3c00000006001602a800000006001642a8001b
:04cd4c0000000600dd
:020000040000fa
:020000040005f5
:0457f400ffff0000b3
:020000040000fa
:020000040005f5
:0457f800bd030000ed
:020000040000fa
:020000040005f5
:0457fc007f3e0000ec
:020000040000fa
:020000040001f9
:105000000000fe0000000000ecff040000000000b3
:10501000ecff040000000000ecff040000000000b2
:10502000ecff040000000000ecff040000000000a2
:10503000ecff040000000000ecff04000000000092
:10504000ecff040000000000ecff04000000000082
:10505000ecff040000000000ecff04000000000072
:10506000ecff040000000000ecff04000000000062
:10507000ecff040000000000ecff04000000000052
:10508000ecff040000000000ecff04000000000042
:105090009880040002000000ecff04000000000003
:1050a000ecff040000000000ecff04000000000022
:1050b000ecff0400000000008eac040001000000c2
:1050c000ecff040000000000ecff04000000000002
:1050d000ecff040000000000ecff040000000000f2
:1050e0007ee30400010000001280040002000000c2
:1050f000ecff0400000000003eb7040001000000c7
:10510000ecff040000000000ecff040000000000c1
:10511000ecff040000000000ecff040000000000b1
:10512000ecff040000000000ecff040000000000a1
:10513000ecff040000000000ecff04000000000091
:10514000ecff040000000000ecff04000000000081
:10515000ecff040000000000ecff04000000000071
:10516000ecff040000000000ecff04000000000061
:10517000ecff040000000000ecff04000000000051
:10518000ecff040000000000ecff04000000000041
:10519000ecff040000000000ecff04000000000031
:1051a000ecff040000000000ecff04000000000021
:1051b000ecff040000000000a6f504000100000060
:1051c000ecff040000000000ecff04000000000001
:1051d000ecff04000000000036f8040000000000ae
:1051e000ecff040000000000d6b60400010000003f
:1051f000ecff040000000000ecff040000000000d1
:10520000ecff040000000000ecff040000000000c0
:0c521000ecff040000000000000006009d
:020000040000fa
:020000040002f8
:10000000410000004f4b0000004900000034000098
:10001000382e0000312d000035360000496e0000fa
:100020002e20000000330000362e0000312d00008d
:1000300034380000496e00002e200000003200001d
:10004000332d000033360000496e00002e200000e2
:10005000202000000039000036300000300d000084
:100060000a00000039350000323000003030000056
:10007000004100006c6f0000676500006e6f0000bb
:10008000200a000000480000616c00006f6700005b
:10009000656e0000200a000000480000616c00004e
:1000a0006f670000656e0000652000000a00000018
:1000b000586500006e5c00006e2000000a00000021
:1000c000586500006e6f00006e2000000a000000fe
:1000d000426900002d580000656e00006f6e000040
:1000e000200a0000004c000045440000200a0000e7
:1000f00000420000692d00004c4500004420000033
:100100000a0000004d610000747200006978000070
:10011000200a0000004400004c410000200a0000ba
:100120000025000030320000753a00002530000044
:10013000327500003a2500003032000075000000e2
:1001400025300000327500002f25000030320000fd
:10015000752f0000253000003475000000250000d8
:10016000303400006600000000250000303200003e
:10017000753a0000253000003275000000250000af
:10018000303200007500000025300000347500009a
:1001900000250000303200007525000030320000dc
:1001a0007525000030340000752500003032000055
:1001b0007525000030320000752500003032000047
:1001c000750000003c380000300000003e380000a0
:1001d00030000000636d00002f310000306d000022
:1001e00020000000696e00002f320000356600001c
:1001f000742000000025000020000000646500005d
:100200006772000065650000732000000067000051
:100210007261000064690000200000004b63000070
:10022000616e000064200000004c00007578000042
:100230002f320000356d0000200000004b6c0000e4
:10024000757800002f3100006d2000000041000093
:1002500067670000696f0000726e0000616d00004a
:10026000656e0000746f000020460000570000001b
:10027000496e00007365000072690000726500003d
:10028000206c000061200000506500006e640000da
:100290007269000076650000206300006f6e000048
:1002a000206900006c200000465700003a00000062
:1002b00050720000656d000065720000652000004e
:1002c00041670000676900006f7200006e61000006
:1002d000206500002061000074740000656e00005d
:1002e00064650000726500002e2e000000410000d1
:1002f00067670000696f0000726e00006100000017
:100300004d6900007365000020610000206e000050
:100310006976000065610000752000004657000006
:10032000004900006e740000726f000064750000e8
:1003300069720000652000006c6500002063000009
:100340006c65000020550000534200002061000051
:1003500076650000632000006c6500002046000008
:10036000573a0000004100007070000075790000ed
:10037000657200002073000075720000204d0000bf
:10038000657400002e2000005c2000006e690000f3
:100390007665000061750000206500007420000093
:1003a00061740000746500006e64000072650000f6
:1003b0002e2e0000004d0000657400002e2000006d
:1003c0005c2000006e690000766500006175000029
:1003d00000460000572000005570000067720000c2
:1003e0006164000065000000496e00007365000054
:1003f0007274000020740000686500002050000046
:10040000656e0000647200006976000065200000df
:1004100077690000746800002074000068650000bf
:1004200020460000573a00000050000072650000ae
:1004300073730000205500007067000072610000b7
:1004400064650000206100006e64000020770000f9
:1004500061690000742e00002e000000557000003d
:1004600067720000616400006500000055500000e4
:10047000474e0000455400002e68000065780000db
:10048000001e00001f200000002000005365000037
:1004900072760000697a0000696f00002031000068
:1004a000005400006f7500006368000020630000c6
:1004b000616c00002e0000004d65000074720000a9
:1004c0006f000000436100006c6900006272000070
:1004d000617a0000696f00006e6500000054000042
:1004e0006f6c00006c650000726100006e7a0000a5
:1004f00065000000496e0000636c0000696e00003a
:100500006f6d000065740000726f00000055000000
:100510006e69000074610000270000005072000046
:100520006576000069650000770000002053000038
:1005300065720000766900006365000020310000ec
:1005400000430000616c0000696200002e20000082
:1005500054610000637400002e0000004d6500002f
:1005600074720000650000004527000074610000ff
:100570006c6c00006f6e0000616700006500000099
:10058000546f00006c650000726100006e63000033
:1005900065730000004900006e6300006c69000094
:1005a0006e6f00006d650000747200006500000051
:1005b000556e000069740000650000004170000085
:1005c000657200006375000000430000616c00006c
:1005d0006962000072610000746900006f6e0000c3
:1005e000005400006f6c000065720000616e000036
:1005f00063650000004900006e6300006c69000044
:100600006e6f00006d6500007465000072000000f0
:10061000556e00006974000079000000340000008d
:10062000496e0000666f000020430000656e000008
:1006300074720000616600006172000069000000d1
:100640004461000074610000206400006920000023
:100650006d6500007373000061200000696e00008a
:1006600020660000756e00007a6900006f6e000061
:10067000653a000000440000617400006120000041
:10068000756c0000746900006d6f00002069000047
:100690006e74000065720000766500006e740000e4
:1006a0006f3a0000004d00006172000063610000bd
:1006b0003a0000004d6f0000646500006c6c0000a3
:1006c0006f3a0000004d0000617400007269000084
:1006d000636f00006c6100003a0000004e7500007e
:1006e0006d2e0000204f00006d6f00006c6f000049
:1006f000672e00003a0000004461000074610000b1
:10070000207500006c740000696d00006f2000000f
:10071000636f00006e740000726f00006c6c00006c
:100720006f3a000000440000617400006120000086
:10073000706500006e7500006c740000696d00004b
:100740006f200000636f00006e740000726f000085
:100750006c6c00006f3a00000044000061740000ff
:1007600061200000756c0000746900006d6100007c
:10077000206d0000616e000075740000656e000061
:100780007a6900006f6e0000653a0000004e0000bc
:10079000756d00002e2000004f6d00006f6c000092
:1007a0006f6700002e2000004f540000434c0000f3
:1007b000414e00003a0000004461000074610000f6
:1007c0002073000063610000646500006e7a000021
:1007d000613a0000004900006e6600006f200000d2
:1007e000527e0000676c0000616700006520000019
:1007f0007068000061720000657300000044000032
:10080000617400006520000064650000206d000038
:100810006973000065200000656e00002073000011
:100820006572000076690000636500003a00000010
:100830004461000074650000206400006520000031
:100840006c61000020640000657200006e690000a9
:100850007e72000065200000696e00007465000073
:1008600072760000656e0000746900006f6e000013
:100870003a0000004d6100007271000075650000d3
:100880003a0000004d6f0000647e00006c650000bf
:100890003a0000004e7500006d7e0000726f00008f
:1008a0002064000065200000737e00007269000073
:1008b000653a0000004e0000756d00007e72000079
:1008c0006f2000006427000061670000727e000056
:1008d0006d6500006e7400003a0000004465000081
:1008e000726e0000697e00007265000020640000e6
:1008f000617400006520000064650000207600003f
:100900007e72000069660000696300006174000087
:10091000696f00006e3a000000410000766100003f
:100920006e74000020640000657200006e690000b3
:100930007e720000652000006461000074650000a4
:1009400020640000652000006d610000696e0000f9
:10095000746500006e6100006e630000653a00007f
:1009600000440000657200006e6900007e720000a5
:1009700065200000646100007465000020640000d0
:10098000652000006d610000696e00007465000064
:100990006e6100006e630000653a0000004f0000c9
:1009a000544300004c4100004e2000004e750000f2
:1009b0006d2e0000206400002761000067720000b7
:1009c0007e6d0000656e0000743a00000044000077
:1009d0006174000065200000642700006578000055
:1009e0007069000072610000746900006f6e0000a1
:1009f0003a000000416200006f75000074200000a2
:100a000048650000616400006c69000067680000d0
:100a100074200000736500007474000065720000ab
:100a2000004300006f6d00006d69000073730000eb
:100a3000696f00006e6900006e67000020640000ae
:100a400061740000650000004c61000073740000d8
:100a5000206900006e740000657200007665000079
:100a60006e740000696f00006e2000006461000079
:100a70007465000000420000726100006e640000b6
:100a80003a0000004d6f0000646500006c3a000001
:100a90000053000065720000696100006c200000d6
:100aa0006e7500006d620000657200003a00000083
:100ab00041700000707200006f760000616c0000f1
:100ac000206e0000756d00002e3a0000004c000002
:100ad0006173000074200000636f00006e740000fa
:100ae000726f00006c2000006461000074650000fb
:100af0003a000000506500006e7500006c74000044
:100b0000696d00006174000065200000636f0000e3
:100b10006e740000726f00006c20000064610000c1
:100b2000746500003a0000004c610000737400001e
:100b300020730000657200007669000063650000a4
:100b40002064000061740000653a0000004f00005e
:100b5000544300004c4100004e2000004170000052
:100b6000707200002e2000006e7500006d2e0000d7
:100b70003a000000457800007069000072610000d2
:100b8000746900006f6e0000206400006174000052
:100b9000653a00000046000057200000646900002c
:100ba000737000006c610000793a000000310000b1
:100bb0002e300000312e0000323000000000000016
:100bc0004657000020430000616d00003a0000001d
:100bd0004f540000436c0000616e00003a000000ba
:100be00047690000656700006e650000743a000008
:100bf0000047000069650000676400006174000040
:100c000061200000564c00003a00000047690000d7
:100c100065670000646100007461000020500000fe
:100c20004c3a0000004f0000544300004c410000cb
:100c30004e20000073740000657000003a00000050
:100c4000426100007564000072610000746500007c
:100c50003a0000005369000072650000743a000019
:100c6000001e000020000000204f0000505a00002d
:100c7000494f00004e490000002000004170000074
:100c8000706c000069630000617a0000696f000009
:100c90006e69000000500000726f00007661000075
:100ca000207500006666000069630000696100004d
:100cb0006c65000000500000726f0000766100005b
:100cc000206c000069620000657200006100000095
:100cd0004f500000544900004f4e000073000000c8
:100ce00020410000707000006c690000636100002a
:100cf000746900006f6e000073000000546500000e
:100d000073740000206f00006666000069630000d5
:100d1000696500006c0000005465000073740000f9
:100d2000206c00006962000072650000004f000046
:100d30006666000069630000696100006c200000c5
:100d400074650000737400000046000072650000c6
:100d500065200000746500007374000000530000fb
:100d600045520000564900005a4900004f0000005b
:100d70005345000052560000494300004500000062
:100d8000210000004c4900004e4700005541000082
:100d90000044000049530000504c0000415900003d
:100da0000044000061740000612000006520000024
:100db0004f720000610000004c4100004e470000ef
:100dc0005545000000410000464600004943000030
:100dd00048450000555200000044000061740000c6
:100de0006520000065740000206800006575000043
:100df00072650000004c0000414e000047550000a5
:100e00004147000045000000446100007465000097
:100e1000202d0000204800006f75000072000000c7
:100e2000494e0000464f00000046000057000000f9
:100e3000504900004e00000052650000616c000047
:100e4000650000005365000072760000697a0000ba
:100e5000696f000020320000005200006561000050
:100e60006c000000536500007276000069630000aa
:100e7000652000003200000047690000656700003f
:100e80004f540000436e00006574000000470000ee
:100e900069650000676e000065740000002d0000a9
:100ea0002d000000446500006d6f0000004c000044
:100eb00041420000004c0000415300004552000038
:100ec000004f00006e0000004f660000660000004a
:100ed0004e7500006f7600006f2000005049000042
:100ee0004e000000537500007200000044650000d1
:100ef000004e00006f75000076650000617500000f
:100f000020500000494e0000004e000065770000b0
:100f100020500000494e000000000000417a00000f
:100f20007a65000072610000004100006363000008
:100f3000657300006f00000053700000656e0000d4
:100f4000746f0000004500006666000061630000e9
:100f50006500000052650000736500007400000029
:100f60004f4e0000004f00004646000000410000c8
:100f70006666000069630000682e00003a200000e9
:100f80004f660000660000004166000066690000d0
:100f9000636800002e3a0000203100006d00000060
:100fa0004166000066690000636800002e3a000098
:100fb000203500006d0000004166000066690000f9
:100fc000636800006575000072000000446900005d
:100fd000737000006c610000793a0000204100004d
:100fe000757300000044000069730000706c00001d
:100ff000617900003a200000316d000000440000db
:1010000069730000706c0000617900003a200000f4
:10101000356d00000044000069730000706c000032
:10102000617900000044000069730000706c0000ea
:10103000617900003a2000004f6600006600000061
:1010400050540000492000004d6f0000646500000e
:1010500000410000646a00002e2000004d6f000077
:1010600064650000004500006e6700006c690000c8
:101070007368000000490000746100006c690000a2
:10108000616e00006f00000046720000616e00009b
:101090005e6100006973000000530000656c000091
:1010a000657a0000696f00006e6100002069000031
:1010b0006c20000076650000696300006f6c000022
:1010c0006f000000436100006e630000656c00006b
:1010d0006c6100000053000069000000537e0000b6
:1010e0006c65000063740000696f00006e2e0000e4
:1010f000206c000065200000767e0000686900001a
:10110000637500006c650000005500006e00000073
:10111000436800006f6f00007365000020740000da
:1011200068650000207600006568000069630000c3
:101130006c650000004500007261000073650000ee
:101140000059000065730000004e00006f000000b1
:10115000302f00000023000022000000556e000028
:10116000697400006520000064650000206d0000c7
:10117000657300007572000065000000486f000094
:10118000726900007a6f00006e740000616c0000ec
:101190000056000065720000746900006361000081
:1011a0006c000000496e0000746500006e73000062
:1011b0006974000065000000426900007269000067
:1011c0006d690000203c00006c5e00007b6e00003a
:1011d00000590000617400006179000000440000c3
:1011e000696b000065790000005900006f23000062
:1011f000756e00006c7500006b0000004d6500000e
:10120000617300007572000065200000756e0000bb
:101210006974000079000000496e000074650000e8
:101220006e7300006974000079000000556e0000c4
:10123000697400006127000020640000692000003c
:101240006d6900007375000072610000004f0000be
:10125000726900007a7a00006f6e0000746100000d
:101260006c650000005600006572000074690000a3
:10127000636100006c650000004900006e740000ae
:10128000656e0000736900007461000027000000b3
:101290002a2d0000002a00002c0000002a2e000049
:1012a00000320000330000001d0000001c000000a0
:1012b0004400000041790000617200006c61000090
:1012c0006d610000004b0000616c0000696200006d
:1012d00072610000766900006d6f0000004400003c
:1012e0002e4100006c6f0000004400002e580000ea
:1012f000656e00002e000000442e00004c650000ca
:1013000064000000496e0000747200006f64000009
:101310007569000072650000206c00006520000007
:10132000504900004e3a0000005600006965000078
:1013300075780000002600006966000072650000f4
:10134000796900002047000069720000696e0000a2
:101350003a000000457300006b6900002026000081
:101360006966000072650000004500006e740000b0
:101370006572000020500000494e0000206300000c
:101380006f640000653a0000004f00006c640000cc
:10139000004900006e730000657200006973000070
:1013a00063690000206900006c20000050490000c3
:1013b0004e3a0000005600006563000063680000bc
:1013c000696f0000003000000031000000320000b2
:1013d0000033000000350000003600000037000038
:1013e000003800000039000000440000454c0000b7
:1013f000004900006d7000006f7300007461000010
:101400007a6900006f6e000069320000004600003b
:10141000656e0000646900006e6500006262000095
:1014200069610000004100006c6f0000676500000a
:101430006e6f0000004100006c740000657a0000cf
:101440007a61000000500000726f000067720000b7
:10145000616d00006d610000746900006f6e000036
:1014600073320000004600006f670000204c00004f
:10147000696700006874000000480000616c0000ab
:101480006f670000656e00006500000048610000a5
:101490007574000065750000720000004f75000053
:1014a000690000005365000074740000696e00005c
:1014b0006773000032000000486100006c6f00009c
:1014c000676500006e000000486500006967000065
:1014d00068740000003c000038300000636d0000bc
:1014e000004c00004544000000440000617400000e
:1014f00061200000652000006f72000061000000a4
:10150000476900006f7200006e6f0000004d000020
:101510006573000065000000416e00006e6f000002
:10152000004f000072610000004d0000696e000075
:1015300075740000690000004461000074650000db
:1015400020650000742000006865000075720000ce
:1015500065200000004a00006f7500007200000066
:101560004d6f000069730000004100006e6e0000c6
:1015700065650000004800006575000072650000a8
:10158000004d0000696e0000757400006573000076
:1015900000540000696d00006520000073650000c4
:1015a00074740000696e0000670000004461000070
:1015b000790000004d6f00006e74000068000000ac
:1015c0005965000061720000004800006f7500005e
:1015d000720000004d6900006e7500007465000027
:1015e000005300006574000000500000726f00009e
:1015f000672e0000004d0000657400006572000059
:1016000000440000656600002e000000204d000030
:10161000616e0000756100006c0000002053000046
:10162000656e0000736f00007200000063610000cf
:101630006d2000006164000064720000006300001f
:10164000616d000020640000617400006f00000004
:101650005072000065730000732000004f4b0000c3
:1016600000410000646400007265000073730000b4
:101670002000000044610000746f000020000000a2
:10168000202000002020000020200000202000005a
:101690002000000045550000204100007379000043
:1016a0006d2e0000200a000000530000796d00003c
:1016b0002e2000000a00000053000000554b0000df
:1016c00020200000200a0000004700000043000026
:1016d00061720000200a0000004d00006f740000dd
:1016e0006f2000000a0000004d6f0000746f0000c2
:1016f00072630000796300002e2000000a000000e1
:1017000054720000756300006b2000000a000000a6
:101710004e330000470a00000041000075740000cd
:101720006f0a0000004d00006f7400006f0a000097
:10173000004d00006f7400006f63000069630000db
:101740006c6f00000a000000436100006d6900003a
:101750006f6e0000200a0000004100007574000058
:101760006f2000000a000000496d0000706f00004b
:1017700073740000617a0000696f00006e690000f8
:10178000310000004c750000636500000056000049
:1017900065690000636f00006c6f00000046000088
:1017a000617200006f000000546100007267000069
:1017b00061000000507200006f670000726100005d
:1017c0006d6d000061740000696f00006e730000b1
:1017d000310000004c7500006d690000657200006a
:1017e0006500000056650000686900006375000030
:1017f0006c65000000500000686100007265000028
:10180000005000006c6100007175000065740000fc
:1018100074650000005300006574000074690000e6
:101820006e67000073310000004c00006967000023
:1018300068740000005600006568000069630000dd
:101840006c6500000048000065610000646c0000e9
:101850006967000068740000005000006c610000bf
:1018600074650000003c00003830000000000000fb
:101870003e380000302000003c31000030300000d5
:10188000000000003e31000030300000203c00002d
:101890003132000030000000003e00003132000014
:1018a0003000000000350000360000003e38000027
:1018b000302000003c31000030300000003e0000cd
:1018c00031300000302000003c3100003230000098
:1018d000003e000031320000300000004c6f00007c
:1018e00077200000426100007474000065720000ff
:1018f000793a0000200a0000506c00006561000089
:101900007365000020720000652d00006368000010
:101910006172000067650000004400007b24000045
:101920007b6b000020500000696c00003a20000032
:101930000a240000617200006a2000006564000053
:10194000696e0000004200006174000074650000d0
:101950007269000061200000736300006172000082
:1019600069630000613a0000200a0000436f000034
:101970006c6c00006567000061720000652000006b
:101980006c270000616c0000696d0000656e00004e
:1019900074610000746f0000726500002070000028
:1019a000657200000a6c000061200000726900008e
:1019b000636100007269000063610000004900007b
:1019c0004e4600004f20000030310000004400006f
:1019d00061740000612000007265000076690000fb
:1019e000736900006f6e00006520000073630000e3
:1019f0006164000075740000613a0000004100005d
:101a000070700000726f0000766100006c200000b2
:101a100064610000746500002065000078700000bb
:101a200069720000656400003a0a00000a54000070
:101a30006f75000063680000207400006865000096
:101a40002073000063720000656500006e200000d6
:101a5000746f0000206300006f6e00007469000066
:101a60006e75000065000000494e0000464f000002
:101a70002030000033000000507200006f7600003c
:101a8000616600006172000069200000646100006e
:101a9000207200006576000069730000696f000025
:101aa0006e610000726500002c2000006368000079
:101ab000696100006d61000072650000006c00004b
:101ac00027610000737300006973000074650000f3
:101ad0006e7a00006120000074650000636e0000f3
:101ae000696300006120000061750000746f0000f0
:101af000726900007a7a000061740000612e0000b3
:101b000000500000726500006d6500007265000005
:101b1000206c00006f200000736300006865000007
:101b2000726d00006f2000007065000072200000e0
:101b3000636f00006e740000696e00007561000044
:101b400072650000005400006f75000063680000bb
:101b500020630000616c0000696200007261000097
:101b6000746900006f6e0000005000006c6500009a
:101b70006173000065200000746f00007563000051
:101b80006820000074680000652000007363000096
:101b900072650000656e0000206900006e20000084
:101ba00074680000650a0000657800006163000049
:101bb00074200000706f00007369000074690000f9
:101bc0006f6e0000206900006e6400006963000011
:101bd000617400006564000020620000792000004c
:101be000746800006520000061720000726f0000e0
:101bf0007773000000430000616c00006962000020
:101c0000726100007a6900006f6e000065200000bc
:101c1000546f00007563000068000000546f0000fe
:101c200063630000612000006c6f000020730000ff
:101c300063680000657200006d6f0000206e000098
:101c4000656c00006c610000207000006f73000084
:101c5000697a0000696f00006e6500000a450000a7
:101c6000534100005454000041200000696e000000
:101c7000646900006361000074610000206400007a
:101c8000616c00006c650000206600007265000059
:101c90006363000069650000005300007461000088
:101ca000727400000054000061720000676100005f
:101cb0003a000000506c0000617100007565000082
:101cc00074740000653a0000005000006c61000070
:101cd000746500003a00000053540000300000001a
:101ce0004142000031000000434400003200000087
:101cf0004546000033000000474800003400000063
:101d0000494a0000350000004b4c0000360000003e
:101d10004d4e0000370000004f500000380000001a
:101d200051520000390000005556000057000000d5
:101d3000585900005a0000004142000043000000d2
:101d40005461000062000000616200006300000056
:101d500073740000306100006231000063640000b1
:101d600032650000663300006768000034690000d7
:101d70006a3500006b6c0000366d00006e370000a5
:101d80006f70000038710000723900007576000035
:101d900077780000797a000000530000543000008a
:101da000414200003143000044320000454600003b
:101db0003347000048340000494a0000354b00001a
:101dc0004c3600004d4e0000374f000050380000e8
:101dd0005152000039550000565700005859000074
:101de0005a000000504900004e20000065720000bb
:101df000726100006e650000004300006f6e00001d
:101e0000662e000020500000494e00000026000011
:101e100069660000726500002048000061740000df
:101e2000616c000021000000596500006e6900002f
:101e3000202600006966000072650000004f000067
:101e40006e610000792e0000202600006966000007
:101e50007265000000500000494e0000206900003b
:101e60006e6300006f720000726500006374000012
:101e700000500000494e0000206500007272000012
:101e8000617400006f0000002d000000520000008f
:101e90004c00000028290000002000002000000065
:101ea0004e4f00004b000000546f00006c650000b6
:101eb000726100006e730000005400002e4f00009d
:101ec0002e4400002e000000542e00004f2e000073
:101ed000532e0000005400002e5600002e55000026
:101ee0002e000000542e0000562e0000442e00004c
:101ef000004c00002e4d000041580000004c000036
:101f00002e6d0000696e0000004400002e4c0000a1
:101f10002e000000542e000059000000542e000036
:101f2000522e0000002600000027000000240000c0
:101f30000022000000500000430000000d0a0000d5
:101f40002a2a00002a2a00002a20000055530000f7
:101f50004220000045720000726f000072200000f5
:101f60002d200000646500007669000063650000b4
:101f70002072000065710000756900007265000044
:101f800073200000746f00006f2000006d7500006a
:101f90006368000020630000757200007265000035
:101fa0006e740000202a00002a2a00002a2a00005d
:101fb0000d0a0000000d00000a2a00002a2a000075
:101fc0002a2a00002055000053420000204500004e
:101fd000727200006f720000202d00002068000067
:101fe000756200007320000061720000652000002f
:101ff0006e6f0000742000007375000070700000a8
:102000006f72000074650000642000002a2a00003e
:102010002a2a00002a0d00000a0000000d0a000014
:102020002a2a00002a2a00002a2000005553000016
:102030004220000045720000726f00007220000014
:102040002d200000646500007669000063650000d3
:1020500020690000732000006e6f000074200000f3
:1020600073750000707000006f72000074650000ee
:10207000642000002a2a00002a2a00002a0d0000fd
:102080000a0000000d0a00002a2a00002a2a000087
:102090002a20000055530000422000004572000035
:1020a000726f0000722000002d20000063610000ac
:1020b0006e6e00006f740000206500006e750000f9
:1020c0006d6500007261000074650000206400000e
:1020d0006576000069630000652000002a2a000080
:1020e0002a2a00002a0d00000a0000000d0a000044
:1020f0002a2a00002a2a00002a2000005553000046
:102100004220000045720000726f00007220000043
:102110002d200000636c0000696500006e740000f3
:1021200020640000726900007665000072200000e3
:10213000696e000069740000696100006c6900004c
:102140007a610000746900006f6e00002065000075
:10215000727200006f720000202a00002a2a00001c
:102160002a2a00000d0a0000000d00000a2a0000c3
:102170002a2a00002a2a00002055000053420000ad
:1021800020450000727200006f720000202d0000d8
:10219000206f000075740000206f000066200000b2
:1021a0006865000061700000206d0000656d000032
:1021b0006f720000792000002a2a00002a2a0000fd
:1021c0002a0d00000a0000000d0a00002a2a000063
:1021d0002a2a00002a200000555300004220000057
:1021e00045720000726f0000722000002d20000078
:1021f000756e000073700000656300006966000082
:1022000069650000642000002a2a00002a2a0000d4
:102210002a0d00000a00000041500000503a000062
:10222000204300006f7500006c640000206e000009
:102230006f740000206d00006f7500006e74000068
:10224000206d000065640000696100000d0a000057
:10225000002a00002e2a0000002100002045000076
:10226000727200006f720000207700007269000037
:10227000746900006e670000206c00006f6700004a
:1022800020660000696c0000650d00000a00000077
:1022900025300000327500003a2500003032000081
:1022a000755f000025300000327500002f2500000a
:1022b00030320000752f000025300000347500001a
:1022c0005f4600007720000064690000733a000058
:1022d000257300005f460000772000006361000066
:1022e0006d3a0000257300005f700000773a00002f
:1022f00025730000202000000d0a000000000000ef
:1023000061000000474c00004f4700002e740000a1
:1023100078740000003100003233000034350000d2
:1023200036000000006d0000696e00002d340000d2
:102330002c300000252000006d610000782d000089
:10234000312c000030250000006d0000696e000097
:102350002d3200002c350000252000006d610000aa
:10236000782d0000302c000035250000006d0000a5
:10237000696e00002d3300002c3000002520000085
:102380006d610000782d0000302c00003525000024
:10239000006d0000696e00002d3300002c3000003d
:1023a000252000006d610000782d0000312c000018
:1023b00030250000006d0000696e00002d33000024
:1023c0002c350000252000006d610000782d0000f4
:1023d000312c000035250000003e000038300000a0
:1023e000636d0000003e000038300000636d0000a7
:1023f0003c31000030300000636d0000003e000002
:1024000031300000306300006d3c000031320000cc
:10241000306300006d0000003e31000032300000eb
:10242000636d000000720000004700004e45000090
:102430005444000041540000412e00007478000014
:1024400074000000474e0000455400004346000061
:10245000472e000074780000740000004d47000013
:102460004152000041470000452e000074780000f2
:102470007400000075700000636100006d2e0000a4
:1024800062690000740000006f6b0000636100006f
:102490006d2e0000626900007400000048450000d5
:1024a000414400004c49000047480000543a0000f5
:1024b0000a00000048450000414400004c4900006b
:1024c0004748000054200000523a00000a00000073
:1024d000204c00006f770000204200006561000082
:1024e0006d3a00000a000000204600006f670000ff
:1024f000204c000069670000687400003a0a000080
:102500000052000065730000756c0000743a000012
:10251000204700004f4f00004400000052650000bb
:10252000737500006c7400003a2000004241000006
:1025300044000000205400006f6f0000204800009d
:1025400069670000680a000000200000546f000066
:102550006f2000004c6f0000770a0000004e000062
:102560006f740000206d000065610000737500004d
:1025700072650000640a000000460000415200003d
:102580004f3a00000a00000046410000524f000090
:1025900020440000583a00000a00000020410000da
:1025a0006e61000062620000616700006c690000fb
:1025b000616e0000746500003a0a0000002000000f
:1025c000466500006e640000696e000065620000f0
:1025d00062690000613a00000a00000045730000d3
:1025e000697400006f3a0000205200004547000067
:1025f0004f4c0000415200004500000045730000b0
:10260000697400006f3a0000204900005252000037
:10261000454700004f4c00004152000045000000bb
:1026200020540000726f0000707000006f200000e6
:10263000416c0000746f00000a000000205400008c
:10264000726f0000707000006f2000004261000097
:10265000737300006f0a0000004e00006f6e0000f0
:10266000206d000069730000757200006174000045
:102670006f0a000000500000484100005245000071
:102680003a0a000000500000484100005245000096
:10269000204700006175000063680000653a000093
:1026a0000a00000050480000415200004520000090
:1026b000447200006f690000743a00000a000000d4
:1026c0002046000065750000782000006465000069
:1026d00020630000726f000069730000656d0000e8
:1026e000656e0000743a00000a00000020410000fe
:1026f0006e740000692d0000627200006f750000aa
:10270000696c00006c610000726400003a0a00000d
:10271000005200007e730000756c000074610000c0
:10272000743a0000204200004f4e000000520000aa
:102730007e730000756c000074610000743a000044
:102740002050000041530000204200004f4e000086
:1027500000200000547200006f700000204800004c
:1027600061750000740a000000200000547200002f
:102770006f70000020420000617300000a0000003a
:102780004e6f00006e2000006d6500007375000044
:1027900072820000650a0000004e00006f6e0000ab
:1027a000206d000065730000757200007e650000fa
:1027b0000a00000052820000737500006c74000073
:1027c000617400003a200000424f00004e000000fb
:1027d00052820000737500006c7400006174000088
:1027e0003a2000005041000053200000424f0000fa
:1027f0004e00000046410000524f000020530000f0
:10280000583a00000a00000048450000414400001a
:102810004c49000047480000542000004c3a00009a
:102820000a000000312e00003031000000000000de
:102830000a0a00002a2a00002a2a00002a2a000088
:102840002a2a00002a2a00002a2a00002a2a000038
:102850002a2a00002a2a00002a2a00002a2a000028
:102860002a2a0000002500003032000073250000f5
:102870003032000073250000303400007325000062
:102880003032000073250000303200007325000054
:1028900030320000730000002e2e00002e2e0000ab
:1028a0002e0000000a2a00002a2a00002a2a00001e
:1028b0002a2a00002a2a00002a2a00002a2a0000c8
:1028c0002a2a00002a2a00002a2a00002a2a0000b8
:1028d0002a2a00002a000000436f000073740000e1
:1028e00072750000747400006f720000653a000099
:1028f00020250000730a0000004d00006f640000f6
:10290000656c00006c6f00003a2000002573000029
:102910000a000000532f00004e3a0000202500005e
:10292000730a0000004600005720000056650000b2
:10293000722e00003a200000257300000a000000fb
:102940004f6d00006f6c00006f6700002e3a0000b2
:1029500020250000730a0000005500006c74000080
:10296000696d00006f200000436f00006e7400006e
:10297000726f00006c6c00006f3a00000a250000c6
:10298000730a0000000a00002a2a00002a2a000018
:102990002a2a00002a2a00002a2a00002a2a0000e7
:1029a0002a2a00002a2a00002a2a00002a2a0000d7
:1029b0002a2a00002a00000044610000746100001f
:1029c000206900006e6900007a6900006f20000035
:1029d000707200006f760000613a00000025000070
:1029e00030320000732f00002530000032730000e9
:1029f0002f25000030340000732000002530000037
:102a0000327300003a25000030320000733a0000b3
:102a100025300000327300000a0a00000054000054
:102a200061720000676100003a2000002573000019
:102a30000a0000004d6100006e7500006661000034
:102a40006374000075720000657200003a20000097
:102a5000257300000a0000004d6f0000646500004f
:102a60006c3a000020250000730a000000410000bd
:102a700070700000726f0000766100006c3a000018
:102a800020250000730a0000004c00006173000064
:102a90007420000043680000656300006b3a00008a
:102aa0000a250000730a0000005300007461000052
:102ab0007274000020740000657300007420000030
:102ac00064610000746500003a000000506c000072
:102ad00061740000653a000020250000730a0000c0
:102ae000004600006162000072690000636100003e
:102af0006e7400003a200000257300000a000000f8
:102b00004d6f0000648200006c6500003a200000f8
:102b1000257300000a0000004657000020720000e4
:102b2000827600002e3a000020250000730a000083
:102b30000041000070700000726f000062610000d0
:102b4000742e00003a200000257300000a000000e7
:102b500044650000726e0000696500007265000047
:102b6000205600006572000069660000696300007d
:102b700061740000696f00006e3a000020250000bb
:102b8000730a00000044000061740000652000002a
:102b90006482000062750000742000006427000059
:102ba0006573000073610000693a00000050000086
:102bb0006c61000071750000653a0000202500007e
:102bc000730a0000006800003c3800003063000019
:102bd0006d0a00006d6900006e2d0000322c0000af
:102be00035250000206d0000617800002d300000c8
:102bf0002c350000250a0000006800003e3d000062
:102c000038300000636d0000203c00003d310000c2
:102c100030300000636d00000a6d0000696e000036
:102c20002d3300002c300000252000006d610000d5
:102c3000782d0000302c0000352500000a0000002f
:102c4000683e000031300000306300006d3c000041
:102c50003d31000032300000636d00000a6d00005d
:102c6000696e00002d3300002c300000252000008c
:102c70006d610000782d0000312c0000302500002f
:102c80000a000000683e000031320000306300009e
:102c90006d0a00006d6900006e2d0000332c0000ed
:102ca00035250000206d0000617800002d31000006
:102cb0002c350000250a00000025000073200000cc
:102cc000005500005000000044570000006800005c
:102cd0003c380000306300006d0a00006d690000a0
:102ce0006e2d0000342c000030250000206d000007
:102cf000617800002d3100002c300000250a000012
:102d0000006800003e3d000038300000636d0000a8
:102d10000a6d0000696e00002d3400002c300000a8
:102d2000252000006d610000782d0000312c00008e
:102d3000302500000a0000004461000074610000ba
:102d400020660000696e00006520000070720000bf
:102d50006f760000613a0000004500006e640000dc
:102d6000207400006573000074200000646100009e
:102d7000746500003a0000004461000074650000c2
:102d80002064000065200000666900006e200000dd
:102d90006573000073610000693a0000000a0000da
:102da0000a2a00002a2a00002a2a00002a2a0000f3
:102db0002a2a00002a2a00002a2a00002a2a0000c3
:102dc0002a2a00002a2a00002a2a00002a2a0000b3
:102dd0002a0a00000a0a0000006800003c380000cf
:102de000306300006d2000006d6900006e2d000052
:102df000322c000035250000206d000061780000b5
:102e00002d3000002c35000025000000683e000039
:102e10003d380000306300006d2000003c3d0000a4
:102e200031300000306300006d2000006d6900004b
:102e30006e2d0000332c000030250000206d0000b6
:102e4000617800002d3000002c35000025000000c6
:102e5000683e000031300000306300006d2000004b
:102e60003c3d000031320000306300006d20000066
:102e70006d6900006e2d0000332c0000302500002d
:102e8000206d0000617800002d3100002c30000022
:102e900025000000683e0000313200003063000071
:102ea0006d2000006d6900006e2d0000332c0000c5
:102eb00035250000206d0000617800002d310000f4
:102ec0002c35000025000000683c00003d38000063
:102ed000306300006d2000006d6900006e2d000061
:102ee000342c000030250000206d000061780000c7
:102ef0002d3100002c30000025000000683e00004d
:102f000038300000636d0000206d0000696e000025
:102f10002d3400002c300000252000006d610000e1
:102f2000782d0000312c000030250000002b00001f
:102f3000302e0000300000000041000063630000fc
:102f4000656e000064690000206900006c200000cc
:102f500066610000726f0000206900006e6400006e
:102f600069630000617400006f0a000000650000e2
:102f7000207000006f690000207000007265000082
:102f80006d690000206900006c2000007075000071
:102f90006c730000616e0000746500000a000000a0
:102fa000416c00006c7500006d650000722000002f
:102fb0006c65000020700000686100007265000010
:102fc000206900006e6400006971000075650000f2
:102fd00020650000740a0000006500006e730000a8
:102fe0007569000074650000206500006e660000d1
:102ff0006f6e000063650000722000006c650000c9
:10300000206200006f750000746f00006e0a0000ff
:10301000005300007769000074630000682000001e
:103020006f6e0000207400006865000020680000da
:1030300065610000646c000069670000687400004e
:103040000a000000616e0000642000007468000047
:10305000656e000020700000726500007373000050
:103060002074000068650000206200007574000094
:10307000746f00006e0a0000004300006f6e0000d5
:1030800066650000726d0000612000006361000051
:103090006e630000656c00006c6100007a690000de
:1030a0006f6e0000653a0000004300006f6e000084
:1030b00066690000726d0000652000006c2700004a
:1030c000616e00006e7500006c61000074690000a4
:1030d0006f6e00003a000000506c00006561000057
:1030e00073650000206300006f6e000066690000d9
:1030f000726d0000206500007261000073650000c1
:103100003a0000002000000037320000303000009c
:10311000255b00005e0a00005d73000000300000c7
:1031200032300000302500005b5e00000a5d0000c8
:1031300073000000253400006425000031310000d8
:103140007300000025300000346400002564000096
:1031500000250000303400006425000073000000ea
:1031600025340000642500007300000025300000b5
:1031700034640000252d0000323000007300000090
:103180002530000034640000252d00003873000055
:103190000025000030340000642500002d350000bb
:1031a000730000002530000034640000252d00006d
:1031b00038730000252d000031320000730000003c
:1031c0002530000034640000252d0000313000005f
:1031d0007300000025300000386c000078250000e6
:1031e000303800006c78000000430000616c000083
:1031f0006962000072610000746900006f6e000077
:10320000206300006f6d0000706c000065740000aa
:10321000656400002f3000003000000043610000b2
:103220006c69000062720000617a0000696f000042
:103230006e650000206300006f6d0000706c000080
:103240006574000061740000612f000030300000e0
:1032500000450000727200006f7200003a2000000a
:10326000706c000065610000736500002072000052
:103270006570000065610000742000007468000043
:1032800065200000636100006c690000627200004c
:1032900061740000696f00006e2f00003030000084
:1032a00000450000727200006f720000653a000075
:1032b00020720000697000006574000065720000f3
:1032c000652000006c61000020630000616c00005c
:1032d00069620000726100007a6900006f6e000090
:1032e000652f000030300000004d00006f760000b8
:1032f00065200000746f00002025000030330000be
:10330000756300006d200000616e00006420000005
:103310007072000065730000732000007365000088
:1033200074000000506f0000736900007a690000ab
:103330006f6e000061200000612000002530000059
:1033400033750000636d00002065000020700000f0
:103350006f69000020700000726500006d69000058
:10336000207300006574000000460000696c0000d6
:10337000652000006e6f00006e2000007472000077
:103380006f760000617400006f000000457200005d
:10339000726f000072650000206200006f6f000015
:1033a000746c00006f610000646900006e670000cb
:1033b0000041000067670000696f0000726e000046
:1033c000616d0000656e0000746f000020690000f0
:1033d0006e200000636f0000727300006f2e00000b
:1033e0002e2e0000004e00006f6e000020740000c2
:1033f0006f6700006c6900006572000065200000c6
:103400006c270000616c0000696d0000656e0000b3
:10341000746100007a6900006f6e000065000000b2
:1034200046690000636800006965000072200000c2
:103430006e6f00006e200000747200006f75000057
:1034400076650000200000004572000072650000f3
:1034500075720000206200006f6f0000746c000045
:103460006f610000646900006e670000004d00009d
:103470006973000065200000612000006e69000093
:103480007665000061750000206500006e20000078
:10349000636f000075720000732e00002e2e000076
:1034a000004e0000652000007061000073200000e5
:1034b000696e000074650000727200006f6d00009c
:1034c00070720000652000006c270000616c000035
:1034d000696d0000656e0000746100007469000091
:1034e0006f6e000000460000696c0000652000005f
:1034f0006e6f000074200000666f0000756e0000a3
:103500006400000045720000726f000072650000e8
:103510002070000065720000666f0000726d000090
:10352000696e000067200000626f00006f74000089
:1035300000550000706700007261000064690000bf
:103540006e6700002e2e00002e2e000020200000ae
:10355000202000002020000020200000200000008b
:10356000446f0000206e00006f74000020720000a5
:10357000656d00006f76000065200000506f000050
:103580007765000072200000537500007070000025
:103590006c7900000050000049500000504f0000be
:1035a0005f300000302e00006865000078000000e9
:1035b000506500006e4400007269000076650000ee
:1035c0002043000068650000636b0000696e000026
:1035d000672e00002e200000200000005065000033
:1035e0006e44000072690000766500002043000010
:1035f00068650000636b0000696e0000672e0000c4
:103600002e4f00004b00000056650000726900005c
:10361000666900006361000020500000656e0000d4
:103620006472000069760000652e00002e20000004
:103630002000000056650000726900006669000005
:103640006361000020500000656e0000647200009d
:1036500069760000652e00002e4f00004b00000030
:10366000567e000072690000666900006361000018
:10367000746900006f6e0000206300006c7e000023
:1036800020550000534200002e2e0000005600007e
:103690007e720000696600006963000061740000ca
:1036a000696f00006e200000636c00007e20000047
:1036b00055530000422e00002e4f00004b0000002a
:1036c00052450000544f000055430000482e0000b2
:1036d00074780000740000007a2e0000482e00006c
:1036e000007a00002e5400002e0000002b32000053
:1036f000250000002d3400002500000020200000df
:103700002041000074740000656e000064690000d0
:103710002e2e00000a000000496e00002046000026
:10372000756e00007a6900006f6e0000650a000087
:10373000002000002020000041740000746500009b
:103740006e640000726500002e2e00000a0000006a
:10375000456e0000206600006f6e0000637400007c
:10376000696f00006e2e00002e0a0000002000008d
:103770002020000057610000697400002e2e000018
:103780000a000000576f0000726b0000696e0000b5
:10379000672e00002e0a00000031000032300000c9
:1037a000300d00000a00000032340000303000000c
:1037b0000d0a00000034000038300000300d000019
:1037c0000a0000003139000032300000300d0000e6
:1037d0000a0000003338000034300000300d0000d3
:1037e0000a00000038330000353200003331000099
:1037f0000025000030320000642500003032000057
:103800006425000030340000640000002530000012
:10381000326400002f25000030320000642f0000c9
:103820002530000034640000004100006c6c000092
:10383000756d000065720000206c000065200000be
:10384000706800006172000065200000696e000071
:103850006469000071750000650a000000650000e1
:1038600074200000656e000073750000697400002c
:1038700065200000656e0000666f00006e6300004a
:1038800065720000206c000065200000626f00007f
:10389000757400006f6e00000a000000706900007f
:1038a00074630000683d0000252e000033660000b0
:1038b0002020000020200000726f00006c6c0000cf
:1038c0003d2500002e33000066200000004100006e
:1038d00074740000656e0000646900003a25000001
:1038e00030330000640000004d000000253000006f
:1038f00034640000004500006e200000466f0000a8
:103900006e630000746900006f6e00000a00000022
:103910004c7b000074660000656e000020450000ce
:103920006b6c000065790000696e00000a00000001
:103930003e6100006c21000024210000796f00002e
:10394000722e00002e0a0000004600006172000086
:103950006c61000072210000204100005e21000027
:103960006e0a0000005300006f6e000072610000dc
:1039700020420000757400006f6e0000612000009e
:1039800042610000732100006e0a0000002a00005e
:103990003a0000002a2b000000320000333c0000f7
:1039a00000370000380000002a260000002a00002e
:1039b0002700000000000000200000007f00000041
:1039c0003d0c00000003000088010000000a000018
:1039d0009401000000040000ac010000000600009b
:1039e000b801000000060000c4010000000a000049
:1039f000d001000000070000e80100000002000004
:103a0000f4010000000400000002000000040000b7
:103a10000c02000000040000180200000006000074
:103a20002402000000030000300200000004000037
:103a30003c020000000300004802000000030000f8
:103a400054020000000600006002000000060000b2
:103a50006c02000000060000780200000006000072
:103a60008402000000060000900200000006000032
:103a70009c02000000060000a802000000060000f2
:103a8000b402000000060000c002000000060000b2
:103a9000cc02000000030000d80200000003000078
:103aa000e402000000060000f00200000006000032
:103ab000fc020000000600000803000000060000f1
:103ac00014030000000b00002003000000080000a9
:103ad0003803000000070000440300000007000056
:103ae00050030000000700005c0300000006000017
:103af00068030000000600007403000000080000d6
:103b000080030000000700008c030000000200009a
:103b10009803000000050000a40300000007000057
:103b2000b003000000060000bc0300000008000015
:103b3000c803000000070000d403000000080000d4
:103b4000e003000000060000ec0300000008000095
:103b5000f803000000070000040400000007000054
:103b600010040000000600001c0400000007000014
:103b7000280400000008000034040000000a0000cf
:103b80004004000000070000580400000008000086
:103b9000640400000007000070040000000300003f
:103ba0007c040000000600008804000000060000fd
:103bb0009404000000060000a004000000060000bd
:103bc000ac04000000060000b8040000000600007d
:103bd000c404000000060000d0040000000600003d
:103be000dc04000000060000e804000000060000fd
:103bf000f4040000000400000005000000060000be
:103c00000c0500000006000018050000000200007e
:103c1000240500000002000030050000000500003f
:103c20003c050000000200004805000000080000fc
:103c300054050000000600006005000000060000ba
:103c40006c0500000006000078050000000600007a
:103c5000840500000004000090050000000600003c
:103c60009c05000000030000a805000000060000fd
:103c7000b405000000060000c0050000000a0000b6
:103c8000cc05000000060000e4050000000600006e
:103c9000f005000000060000fc0500000006000022
:103ca00008060000000600001406000000070000df
:103cb00020060000000600002c060000000800009e
:103cc00038060000000000000000000000000000b6
:103cd00000000000000000000000000000000000e4
:103ce000000000000000000000000000770000005d
:103cf000888000007f80000088000000888000002d
:103d0000770000000000000000000000000000003c
:103d1000e060000020000000000000000000000043
:103d200000000000000000003030000038480000b3
:103d30000878000088780000000000000000000003
:103d40000000000068980000a8a80000c8b00000ab
:103d500000000000000000000000000072000000f1
:103d60005200000054000000740000000b0000002e
:103d70000a80000012800000138000000000000094
:103d8000000000001028000010280000282c00006f
:103d9000447c00004282000000000000000000009f
:103da000c0c0000000000000000000000000000093
:103db0000000000000000000204000004040000023
:103dc0004040000040400000402000000000000093
:103dd00040400000202000002020000020200000a3
:103de000404000000000000040f0000060000000c3
:103df00000000000000000000000000000000000c3
:103e000000000000101000007c10000010000000f6
:103e100000000000000000000000000000000000a2
:103e200000000000004000004040000000000000d2
:103e3000000000000000000000e0000000000000a2
:103e40000000000000000000000000000000000072
:103e50000000000000400000000000000000000022
:103e60002020000040400000404000008080000012
:103e7000000000000000000070880000888800003a
:103e8000888800008870000000000000000000002a
:103e900020600000a0200000202000002020000062
:103ea000000000000000000070880000080800000a
:103eb0001020000040f8000000000000000000009a
:103ec00070880000083000000808000088700000ba
:103ed0000000000000000000103000005050000002
:103ee00090f800001010000000000000000000002a
:103ef0007840000080f00000080800008870000092
:103f000000000000000000007088000080f0000049
:103f10008888000088700000000000000000000099
:103f2000f810000010200000204000004040000079
:103f30000000000000000000708800008870000091
:103f40008888000088700000000000000000000069
:103f500070880000888800007808000088700000e1
:103f600000000000000000000000000080000000d1
:103f700000000000008000000000000000000000c1
:103f80000000000080000000000000000080000031
:103f90008080000000000000000000001c600000a5
:103fa0006018000004000000000000000000000095
:103fb0000000000000f8000000f800000000000011
:103fc00000000000000000000080000070080000f9
:103fd00070800000f80000000000000000000000f9
:103fe0001020000030480000848400004c7800005d
:103ff0000000000000000000000000001f000000a2
:10400000608000004d40000093400000a24000008e
:10401000a2400000a68000009b000000404000007d
:104020003f80000000000000102800002828000049
:10403000447c0000828200000000000000000000bc
:10404000f884000084fc00008484000084f80000f0
:1040500000000000000000003844000080800000e4
:1040600080800000443800000000000000000000d4
:10407000f0880000848400008484000088f0000040
:104080000000000000000000f880000080f8000040
:104090008080000080f800000000000000000000a8
:1040a000f880000080f00000808000008080000028
:1040b0000000000000000000384400008280000082
:1040c0008e82000044380000000000000000000064
:1040d0008484000084fc0000848400008484000048
:1040e00000000000000000008080000080800000d0
:1040f00080800000808000000000000000000000c0
:1041000010100000101000001090000090600000df
:1041100000000000000000008488000090b0000053
:10412000d08800008884000000000000000000002b
:1041300080800000808000008080000080f8000007
:10414000000000000000000082c60000c6aa0000b7
:10415000aaaa0000929200000000000000000000e7
:1041600084c40000a4a40000949400008c84000087
:1041700000000000000000003844000082820000bf
:1041800082820000443800000000000000000000af
:10419000f088000088880000f08000008080000027
:1041a000000000000000000038440000828200008f
:1041b000829a0000443a0000000000000000000065
:1041c000f884000084f800009088000088840000d3
:1041d0000000000000000000788400008060000003
:1041e00018040000847800000000000000000000b7
:1041f000f8200000202000002020000020200000e7
:10420000000000000000000084840000848400009e
:10421000848400008478000000000000000000009a
:104220008282000044440000282800001010000092
:104230000000000000000000000000000840000036
:10424000144000009480000094800000a2800000d0
:10425000a2800000410000004100000000000000ba
:10426000000000000000000084480000483000000a
:1042700030480000488400000000000000000000fa
:1042800082440000442800001010000010100000bc
:1042900000000000000000007c080000101000007a
:1042a0002020000040fc0000000000000000000092
:1042b000204000004040000040400000404000001e
:1042c000000000000000000010200000384800003e
:1042d000087800008878000000000000000000005e
:1042e0002810000038480000087800008878000096
:1042f0000000000000000000000000003048000046
:10430000808000004878000030300000000000008d
:104310002810000030480000848400004c78000021
:104320000000000000000000304800003848000095
:1043300008780000887800000000000000000000fd
:104340000000000070880000788800009868000075
:10435000000000000000000080800000b0c80000e5
:1043600088880000c8b000000000000000000000c5
:10437000000000007088000080800000887000004d
:10438000000000000000000008080000689800001d
:10439000888800009868000000000000000000000d
:1043a0000000000070880000f880000088700000a5
:1043b000000000000000000020400000e04000007d
:1043c00040400000404000000000000000000000ed
:1043d00000000000689800008888000098680000cd
:1043e00008f000000000000080800000b0c800005d
:1043f000888800008888000000000000000000009d
:10440000800000008080000080800000808000002c
:10441000000000000000000080000000808000001c
:10442000808000008080000080000000000000000c
:104430008080000090a00000c0a00000a0900000bc
:10444000000000000000000080800000808000006c
:10445000808000008080000000000000000000005c
:1044600000000000bcd20000929200009292000076
:10447000000000000000000000000000f0880000c4
:10448000888800008888000000000000000000000c
:10449000000000007088000088880000887000001c
:1044a000000000000000000000000000b0c8000094
:1044b00088880000c8b00000808000000000000074
:1044c00000000000689800008888000098680000dc
:1044d000080800000000000000000000a0c000006c
:1044e00080800000808000000000000000000000cc
:1044f000000000007088000060100000887000005c
:10450000000000000000000080800000c08000006b
:104510008080000080c0000000000000000000005b
:10452000000000008888000088880000986800006b
:10453000000000000000000000000000888800006b
:10454000505000002020000000000000000000008b
:104550000000000000000000000000008880000053
:10456000948000005500000055000000220000006b
:104570002200000000000000000000000000000019
:10458000000000008850000020200000508800003b
:10459000000000000000000000000000888800000b
:1045a00050500000202000002040000000000000cb
:1045b00000000000f81000002020000040f800007b
:1045c0000000000000000000280000004848000033
:1045d000484800004878000000000000000000008b
:1045e00028000000384800000878000088780000a3
:1045f00000000000000000003848000048500000a3
:1046000048440000447c000000000000000000005e
:10461000102000003048000084f800004c780000b2
:104620000000000000000000007e00004242000088
:1046300042420000427e0000000000000000000036
:10464000da9c000000000000200000007f00000055
:104650003d1400000005000088010000001000006b
:104660009c01000000060000c4010000000a0000d8
:10467000d8010000000a0000000200000010000045
:1046800028020000000c000050020000000300009f
:1046900078020000000600008c0200000006000006
:1046a000a002000000070000b4020000000b0000a0
:1046b000c802000000050000f00200000006000033
:1046c00004030000000500001803000000050000be
:1046d0002c030000000a000040030000000a000054
:1046e00068030000000a000090030000000a0000b8
:1046f000b8030000000a0000e0030000000a000008
:1047000008040000000a000030040000000a000055
:1047100058040000000a000080040000000a0000a5
:10472000a804000000050000d004000000050000ff
:10473000e4040000000b0000f8040000000b00007f
:1047400020050000000a000048050000000a0000e3
:10475000700500000012000098050000000b00002a
:10476000d4050000000c0000fc050000000d000056
:1047700024060000000d00004c060000000c0000a4
:1047800074060000000b00009c060000000e0000f4
:10479000c4060000000d0000ec060000000400004c
:1047a000140700000009000028070000000c0000aa
:1047b00050070000000a000078070000000f00000a
:1047c000a0070000000d0000c8070000000e000058
:1047d000f0070000000c000018080000000e0000a8
:1047e00040080000000d000068080000000c0000f8
:1047f00090080000000c0000b8080000000d000048
:10480000e0080000000b0000080900000011000093
:1048100030090000000b00006c090000000c0000d3
:1048200094090000000b0000bc0900000005000016
:10483000e4090000000a0000f8090000000a000076
:10484000200a000000090000480a0000000a0000d9
:10485000700a0000000a0000980a0000000a000028
:10486000c00a0000000a0000e80a00000009000079
:10487000100b0000000a0000380b0000000a0000c6
:10488000600b000000050000880b0000000a00001b
:104890009c0b0000000a0000c40b00000004000094
:1048a000ec0b000000040000000c000000090000f8
:1048b000140c0000000400003c0c0000000e00007e
:1048c000500c0000000a0000780c0000000a0000f4
:1048d000a00c0000000a0000c80c0000000a000044
:1048e000f00c000000060000180d00000009000098
:1048f0002c0d000000050000540d0000000a00000f
:10490000680d000000090000900d0000000d00007f
:10491000b80d000000080000e00d000000090000d4
:10492000f40d0000000800001c0e0000000a00004a
:10493000300e0000000a0000580e0000000b0000be
:10494000800e0000000a0000a80e0000000e00000b
:10495000d00e000000000000000000000000000079
:104960000000000000000000000000000000000047
:104970000000000000000000000000000000000037
:104980000000000000000000000000000000000027
:10499000000000001f3c00003ffe000061c6000058
:1049a000078300003fff000079ff000061800000e6
:1049b00063c700007ffe00003e3c000000000000d6
:1049c00000000000000000000000000000000000e7
:1049d000006c00006c680000484800000000000007
:1049e00000000000000000000000000000000000c7
:1049f00000000000000000000000000000000000b7
:104a000000000000120000000c0000000c0000007c
:104a10003f0000006180000001800000078000006e
:104a20003f80000061800000418000006380000042
:104a30003d800000000000000000000000000000b9
:104a40000000000000000000000000000000000066
:104a50000000000000000000000000001d800000b9
:104a60003f00000073000000678000006d800000c0
:104a70006980000079800000338000007f00000022
:104a80006e000000000000000000000000000000b8
:104a90000000000000000000000000000000000016
:104aa0003c1000006420000046200000464000004a
:104ab00064c000002c80000019800000013c000050
:104ac00003260000026600000662000004260000c3
:104ad0000c3c00000000000000000000000000008e
:104ae00000000000040000000800000008000000b2
:104af000060000000e0000000f0000000b00000088
:104b000019800000198000003080000030c00000d3
:104b10003fc00000606000006060000040200000b6
:104b2000c030000000000000000000000000000095
:104b30000000000000000000006000006060000055
:104b400040400000000000000000000000000000e5
:104b50000000000000000000000000000000000055
:104b6000000800001010000030200000606000000d
:104b70006060000060600000202000003010000035
:104b80001808000000000000006000002030000055
:104b900010180000180800000808000008080000ad
:104ba0001818000010300000204000000000000035
:104bb00000100000547c0000386c00000000000071
:104bc00000000000000000000000000000000000e5
:104bd00000000000000000000000000000000000d5
:104be00000000000000000000400000004000000bd
:104bf00004000000040000007fc00000040000006a
:104c00000400000004000000040000000000000098
:104c10000000000000000000000000000000000094
:104c20000000000000000000000000000000000084
:104c30000000000000000000000000000000000074
:104c400030300000102000000000000000000000d4
:104c50000000000000000000000000000000000054
:104c6000f8f8000000000000000000000000000054
:104c70000000000000000000000000000000000034
:104c80000000000000000000000000000000000024
:104c900030300000000000000000000000000000b4
:104ca0000008000018100000103000002020000054
:104cb0002060000040400000c080000000000000b4
:104cc00000000000000000000000000000000000e4
:104cd0001e0000003f0000007380000061800000a3
:104ce0006180000061800000618000006180000040
:104cf0006180000061800000738000003f000000c0
:104d00001e00000000000000000000000000000085
:104d10000000000000000000000000000000000093
:104d2000060000000e0000001e000000360000001b
:104d3000260000000600000006000000060000003b
:104d4000060000000600000006000000060000004b
:104d5000060000000000000000000000000000004d
:104d60000000000000000000000000000000000043
:104d70001e0000003f000000738000006180000002
:104d80000180000001800000030000000600000018
:104d90000c00000018000000300000007f800000c0
:104da0007f80000000000000000000000000000004
:104db00000000000000000000000000000000000f3
:104dc0001c0000003f000000630000000300000022
:104dd000030000000e0000000f0000000180000032
:104de0000180000061800000618000003f00000041
:104df0001e00000000000000000000000000000095
:104e000000000000000000000000000000000000a2
:104e1000060000000e0000000e0000001e00000052
:104e2000360000003600000066000000c6000000ea
:104e3000ff800000ff800000060000000600000068
:104e4000060000000000000000000000000000005c
:104e50000000000000000000000000000000000052
:104e60003f0000003f000000300000006000000034
:104e70006e0000007f0000006180000001800000e3
:104e80000180000061800000618000003f000000a0
:104e90001e000000000000000000000000000000f4
:104ea0000000000000000000000000000000000002
:104eb0001e0000003f000000318000006000000084
:104ec000600000006e0000007f00000071800000a4
:104ed0006180000061800000318000003f00000020
:104ee0001e000000000000000000000000000000a4
:104ef00000000000000000000000000000000000b2
:104f00007f8000007f80000001000000030000009f
:104f100006000000060000000c0000000c0000006d
:104f20000c0000000c000000180000001800000039
:104f30001800000000000000000000000000000059
:104f40000000000000000000000000000000000061
:104f50001e0000003f000000618000006180000032
:104f6000618000003f0000003f0000006180000001
:104f70006180000061800000618000003f0000004f
:104f80001e00000000000000000000000000000003
:104f90000000000000000000000000000000000011
:104fa0001e0000003f0000006180000061800000e2
:104fb00061800000638000003f8000001d800000d1
:104fc0000180000001800000630000003f0000003d
:104fd0001e000000000000000000000000000000b3
:104fe00000000000000000000000000000000000c1
:104ff0003030000000000000000000000000000051
:105000003030000000000000000000000000000040
:105010000000000000000000303000000000000030
:1050200000000000000000003030000010200000f0
:105030000000000000000000000000000000000070
:1050400000000000000000000040000001c000005f
:105050000f0000003c00000060000000780000002d
:105060000e00000003c0000000c0000000000000af
:105070000000000000000000000000000000000030
:105080000000000000000000000000000000000020
:105090000000000000000000000000007fc00000d1
:1050a0007fc0000000000000000000007fc0000082
:1050b0007fc00000000000000000000000000000b1
:1050c00000000000000000000000000000000000e0
:1050d00000000000000000000000000000000000d0
:1050e0000000000040000000700000003c000000d4
:1050f0000700000001800000070000003c000000e5
:105100007000000040000000000000007f800000f0
:105110007f80000000000000000000000000000090
:10512000000000000000000000000000000000007f
:105130000600000004000000080000000c00000051
:105140003f0000006180000061800000408000009e
:1051500040800000408000006180000073800000fb
:105160003e00000000000000000000000000000001
:10517000000000000000000000000000000000002f
:105180000000000000010000f800000007fe000021
:10519000000e00000700000018ef00008031000042
:1051a000fdc0000033380000c067000018c00000d8
:1051b00066180000c066000010c0000066310000e4
:1051c000806700003380000073ff000000330000a0
:1051d000bc00000038010000c01e00000380000079
:1051e0000fff000000030000fc00000000000000b2
:1051f00000000000000000000e0000000e00000093
:105200001b0000001b0000001b000000318000009c
:10521000318000003f8000007fc0000060c00000bf
:1052200060c00000c0600000c0600000000000001e
:10523000000000000000000000000000000000006e
:1052400000000000000000007f8000007fc0000020
:105250006060000060600000606000007fc00000cf
:105260007fc00000606000006060000060600000bf
:1052700060e000007fc000007f80000000000000b0
:10528000000000000000000000000000000000001e
:1052900000000000000000000f8000001fe0000080
:1052a0003870000030300000600000006000000036
:1052b000600000006000000060000000303000006e
:1052c000386000001fe000000780000000000000c0
:1052d00000000000000000000000000000000000ce
:1052e00000000000000000007f8000007fc0000080
:1052f00060e000006070000060300000603000007e
:10530000603000006030000060300000607000001d
:1053100060e000007fc000007f800000000000000f
:10532000000000000000000000000000000000007d
:1053300000000000000000007fe000007fe00000af
:105340006000000060000000600000007fc00000fe
:105350007fc00000600000006000000060000000ee
:10536000600000007fe000007fe00000000000001f
:10537000000000000000000000000000000000002d
:1053800000000000000000007fc000007fc000009f
:105390006000000060000000600000007f800000ee
:1053a0007f800000600000006000000060000000de
:1053b00060000000600000006000000000000000cd
:1053c00000000000000000000000000000000000dd
:1053d000000000000000000007c000001ff00000f7
:1053e000383000003018000060000000600000004d
:1053f00061f8000061f8000060180000301800003b
:10540000383800001ff0000007c000000000000056
:10541000000000000000000000000000000000008c
:10542000000000000000000060300000603000005c
:105430006030000060300000603000007ff000004d
:105440007ff000006030000060300000603000003d
:10545000603000006030000060300000000000009c
:10546000000000000000000000000000000000003c
:10547000006000006060000060600000606000008c
:1054800060600000606000006060000000000000dc
:10549000000000000000000000000000000000000c
:1054a00003000000030000000300000003000000f0
:1054b00003000000030000000300000003000000e0
:1054c0000300000063000000630000007e00000095
:1054d0003c00000000000000000000000000000090
:1054e00000000000000000000000000000000000bc
:1054f00060e0000061c00000638000006700000001
:105500006e0000007c0000007e00000077000000bc
:10551000638000006180000061c0000060e0000066
:1055200060700000000000000000000000000000ab
:10553000000000000000000000000000000000006b
:1055400060000000600000006000000060000000db
:1055500060000000600000006000000060000000cb
:105560006000000060000000600000007f8000001c
:105570007f8000000000000000000000000000002c
:10558000000000000000000000000000000000001b
:10559000701c0000783c0000783c0000783c000063
:1055a0006c6c00006c6c00006c6c0000644c0000c3
:1055b00066cc000066cc000066cc0000638c000066
:1055c000638c0000000000000000000000000000ec
:1055d00000000000000000000000000000000000cb
:1055e000603000007030000078300000783000003b
:1055f0006c3000006630000067300000633000004f
:1056000061b0000060f0000060f000006070000019
:1056100060300000000000000000000000000000fa
:10562000000000000000000000000000000000007a
:1056300007c000001fe0000038700000303000009c
:10564000601800006018000060180000601800007a
:105650006018000030300000387000001fe00000cb
:1056600007800000000000000000000000000000b3
:10567000000000000000000000000000000000002a
:105680007f8000007fc0000060e0000060600000dc
:105690006060000060e000007fc000007f800000cc
:1056a000600000006000000060000000600000007a
:1056b000600000000000000000000000000000008a
:1056c00000000000000000000000000000000000da
:1056d0000fc000001fe000003870000030380000ec
:1056e00060180000601800006018000060180000da
:1056f0006018000031b0000038e000001fe000003a
:105700000fb80000000000000000000000000000d2
:105710000000000000000000000000000000000089
:105720007fc000007fe0000060700000603000007b
:10573000607000007fe000007fc00000618000001a
:1057400061c0000060e00000606000006070000068
:1057500060380000000000000000000000000000b1
:105760000000000000000000000000000000000039
:105770000f8000003fc0000070e00000606000008b
:10578000600000003c0000001f80000003c000001b
:10579000006000006060000070e000003fc000009a
:1057a0001f8000000000000000000000000000005a
:1057b00000000000000000000000000000000000e9
:1057c0007fe000007fe0000006000000060000000f
:1057d00006000000060000000600000006000000b1
:1057e00006000000060000000600000006000000a1
:1057f00006000000000000000000000000000000a3
:105800000000000000000000000000000000000098
:105810006030000060300000603000006030000048
:105820006030000060300000603000006030000038
:105830006030000060300000707000003fe0000049
:105840000f800000000000000000000000000000c9
:105850000000000000000000000000000000000048
:10586000c0600000c060000060c0000060c00000b8
:1058700060c00000318000003180000031800000f5
:105880001b0000001b0000001b0000000e000000b9
:105890000e000000000000000000000000000000fa
:1058a00000000000000000000000000000000000f8
:1058b0000000000000c10000c1800000c1c1000064
:1058c0008063000063000000636300000063000069
:1058d0006300000063630000006600002300000016
:1058e0003636000000360000360000003636000074
:1058f00000360000360000001c1c0000001c0000e8
:105900001c0000000000000000000000000000007b
:105910000000000000000000000000000000000087
:10592000000000000000000071c000003180000095
:105930001b0000001b0000000e0000000e00000015
:105940000e0000001b0000001b0000003b80000058
:105950003180000060c00000e0e0000000000000b6
:105960000000000000000000000000000000000037
:105970000000000000000000e07000006060000017
:1059800030c0000039c00000198000000f00000086
:105990000f000000060000000600000006000000e6
:1059a00006000000060000000600000000000000e5
:1059b00000000000000000000000000000000000e7
:1059c00000000000000000007fc000007fc0000059
:1059d0000180000003000000070000000600000036
:1059e0000c0000001800000038000000300000002b
:1059f00060000000ffc00000ffc0000000000000c9
:105a00000000000000000000000000000000000096
:105a100000180000302000000020000020200000be
:105a200020200000202000002020000000000000b6
:105a30000000000000000000000000000000000066
:105a40000600000004000000080000000c00000038
:105a50003f0000006180000001800000078000001e
:105a60003f800000618000004180000063800000f2
:105a70003d80000000000000000000000000000069
:105a80000000000000000000000000000000000016
:105a9000190000003f000000000000000c000000a2
:105aa0003f000000618000000180000007800000ce
:105ab0003f800000618000004180000063800000a2
:105ac0003d80000000000000000000000000000019
:105ad00000000000000000000000000000000000c6
:105ae0000000000000000000000000000c000000aa
:105af0003f00000061000000610000004000000065
:105b00004000000040000000618000003300000001
:105b10001e00000008000000040000001c0000003f
:105b2000180000000000000000000000000000005d
:105b3000190000003f000000000000000c00000001
:105b40003f00000061800000618000004080000094
:105b500040800000408000006180000073800000f1
:105b60003e000000000000000000000000000000f7
:105b70000000000000000000000000000000000025
:105b80000c0000001e000000330000000c000000ac
:105b90003f000000618000000180000007800000dd
:105ba0003f800000618000004180000063800000b1
:105bb0003d80000000000000000000000000000028
:105bc00000000000000000000000000000000000d5
:105bd0000000000000000000000000001f000000a6
:105be0003f80000061800000078000003f800000cf
:105bf0007980000061800000638000007f800000e9
:105c00003d800000000000000000000000000000d7
:105c10000000000000000000000000000000000084
:105c20006000000060000000600000006e000000e6
:105c30007f00000073800000618000006180000030
:105c40006180000061800000738000007f00000020
:105c50006e000000000000000000000000000000d6
:105c60000000000000000000000000000000000034
:105c70000000000000000000000000001e00000006
:105c80003f000000730000006000000060000000a2
:105c90006000000060000000730000003f00000092
:105ca0001e000000000000000000000000000000d6
:105cb00000000000000000000000000000000000e4
:105cc0000180000001800000018000001d800000b4
:105cd0003f80000073800000618000006180000050
:105ce0006180000061800000738000003f80000040
:105cf0001d80000000000000000000000000000007
:105d00000000000000000000000000000000000093
:105d10000000000000000000000000001e00000065
:105d20003f00000073000000618000007f800000e1
:105d30007f80000060000000718000003f000000d4
:105d40001e00000000000000000000000000000035
:105d50000000000000000000003800007860000033
:105d6000f8f8000060600000606000006060000003
:105d70006060000000000000000000000000000063
:105d80000000000000000000000000000000000013
:105d9000000000001d8000003f80000073800000b4
:105da000618000006180000061800000618000006f
:105db000738000003f8000001d8000000180000013
:105dc000638000007f0000003e0000000000000033
:105dd0000000000000000000600000006000000003
:105de000600000006f0000007f80000071800000f4
:105df000618000006180000061800000618000001f
:105e000061800000618000006180000000000000ef
:105e10000000000000000000000000000000000082
:105e20000060000060000000606000006060000032
:105e30006060000060600000606000000000000022
:105e40000000000000000000006000006000000092
:105e50006060000060600000606000006060000042
:105e60006060000060600000e0c000000000000012
:105e70000000000000000000600000006000000062
:105e80006000000063800000670000006e000000fa
:105e9000780000007c0000006c000000660000003c
:105ea0006600000063000000638000000000000046
:105eb00000000000000000000000000000000000e2
:105ec0000060000060600000606000006060000032
:105ed0006060000060600000606000000000000082
:105ee00000000000000000000000000000000000b2
:105ef0000000000000000000000000006e700000c4
:105f00007ef800007398000063180000631800001a
:105f10006318000063180000631800006318000095
:105f200063180000000000000000000000000000f6
:105f30000000000000000000000000000000000061
:105f40000000000000000000000000006f000000e2
:105f50007f8000007180000061800000618000008f
:105f600061800000618000006180000061800000ad
:105f70006180000000000000000000000000000040
:105f80000000000000000000000000000000000011
:105f90000000000000000000000000001e000000e3
:105fa0003f000000738000006180000061800000fd
:105fb0006180000061800000738000003f000000ed
:105fc0001e000000000000000000000000000000b3
:105fd00000000000000000000000000000000000c1
:105fe0000000000000000000000000006e00000043
:105ff0007f0000007380000061800000618000006d
:106000006180000061800000738000007f0000005c
:106010006e000000600000006000000060000000f2
:106020006000000000000000000000000000000010
:106030000000000000000000000000001d800000c3
:106040003f800000738000006180000061800000dc
:106050006180000061800000738000003f800000cc
:106060001d80000001800000018000000180000010
:10607000018000000000000000000000000000009f
:106080006c7c0000706000006060000060600000d8
:106090006060000000000000000000000000000040
:1060a00000000000000000000000000000000000f0
:1060b000000000003e0000007f00000063000000c0
:1060c000700000003c0000000e000000070000000f
:1060d000630000007f0000003e00000000000000a0
:1060e00000000000000000000000000000000000b0
:1060f0000060000060600000f0f0000060600000e0
:10610000606000006060000070700000000000002f
:10611000000000000000000000000000000000007f
:10612000000000000000000000000000618000008e
:1061300061800000618000006180000061800000db
:106140006180000061800000638000007f800000ab
:106150003d80000000000000000000000000000082
:10616000000000000000000000000000000000002f
:10617000000000000000000000000000c1800000de
:10618000c1800000630000006300000063000000a5
:1061900036000000360000001c0000001c0000005b
:1061a00008000000000000000000000000000000e7
:1061b00000000000000000000000000000000000df
:1061c000000000000000000000000000c2180000f5
:1061d000c7180000c7180000653000006db000004f
:1061e0006db0000028a0000038e0000038e000009a
:1061f00018c00000000000000000000000000000c7
:10620000000000000000000000000000000000008e
:10621000c3660000663c0000181800003c660000e1
:1062200066c3000000000000000000000000000045
:10623000000000000000000000000000000000005e
:1062400000000000c1800000c18000006300000069
:106250006300000033000000360000001e00000054
:106260001e0000000c0000000c0000000c000000ec
:10627000180000007800000070000000000000001e
:106280000000000000000000ffff0000070e0000fb
:106290001c38000070e00000ffff0000000000005c
:1062a00000000000000000000000000000000000ee
:1062b000320000003200000000000000000000007a
:1062c000618000006180000061800000618000004a
:1062d0006180000061800000618000006380000038
:1062e0003d800000000000000000000000000000f1
:1062f000000000000000000000000000000000009e
:106300003200000032000000000000000c0000001d
:106310003f00000061800000018000000780000055
:106320003f80000061800000418000006380000029
:106330003d800000000000000000000000000000a0
:10634000000000000000000000000000000000004d
:106350001e0000003300000061000000610000002a
:10636000630000006200000066000000630000009f
:1063700061c0000060c00000604000006cc0000010
:106380006780000000000000000000000000000026
:1063900000000000000000000000000000000000fd
:1063a0000600000004000000080000000c000000cf
:1063b0003f00000061800000618000007f800000dd
:1063c0007f800000400000006180000071800000bc
:1063d0001f0000000000000000000000000000009e
:1063e00000000000000000000000000000000000ad
:1063f000000000000000000020000000200000005d
:10640000200000002000000020000000200000000c
:1064100020000000200000002000000020000000fc
:10642000200000000000000000000000000000004c
:10643000000000000000000022a300000000000097
:106440001c0000007f000000001c00000010000085
:106450009801000000100000d001000000100000b2
:1064600008020000001000004002000000100000c0
:106470007802000000100000b002000000100000d0
:10648000e8020000001000002003000000100000df
:1064900058030000001000009003000000100000ee
:1064a000c8030000001000000004000000100000fd
:1064b000380400000010000070040000001000000c
:1064c000a804000000100000e0040000001000001c
:1064d000180500000010000050050000001000002a
:1064e0008805000000100000c0050000001000003a
:1064f000f805000000100000300600000010000049
:106500006806000000100000a00600000010000057
:10651000d806000000100000100700000010000066
:106520004807000000100000800700000010000075
:10653000b807000000100000f00700000010000085
:106540002808000000100000600800000010000093
:1065500098080000001000000c0800000010000067
:1065600044080000001400007c080000000e000039
:10657000d0080000000d000008090000000d000018
:1065800040090000000e000078090000000c000027
:10659000b0090000000b0000e8090000000e000038
:1065a000200a000000100000580a00000007000048
:1065b000900a000000070000ac0a0000000e000076
:1065c000c80a0000000b0000000b000000130000d0
:1065d000380b0000001000008c0b0000000e0000c3
:1065e000c40b0000000d0000fc0b0000000e0000ba
:1065f000340c0000000d00006c0c0000000b0000cb
:10660000a40c0000000d0000dc0c000000100000d5
:10661000140d0000001000004c0d000000140000dc
:10662000840d0000000f0000d80d0000000e0000d7
:10663000100e0000000d0000480e000000070000d2
:10664000800e0000000b00009c0e000000080000ff
:10665000d40e0000000c0000f00e0000000b000043
:10666000280f000000080000600f0000000b000071
:106670007c0f0000000c0000b40f0000000a0000b6
:10668000ec0f0000000c000024100000000b0000c4
:106690005c1000000007000094100000000c0000d7
:1066a000b0100000000d0000e8100000000700001e
:1066b00020110000000600003c110000000c00004a
:1066c00058110000000700009011000000140000a5
:1066d000ac110000000d000000120000000c0000d2
:1066e00038120000000d000070120000000c0000c5
:1066f000a8120000000a0000e012000000090000db
:10670000181300000008000050130000000d0000e6
:106710006c130000000c0000a41300000011000026
:10672000dc130000000c000030140000000c00001e
:1067300068140000000b0000a01400000008000016
:10674000d814000000060000f41400000008000047
:1067500010150000000c00002c15000000050000c2
:106760006415000000050000801500000000000016
:106770000000000000000000000000000000000019
:106780000000000000000000000000000000000009
:10679000000000000000000000000000ffff0000fb
:1067a000ffff0000ffff0000ffff000000000000ef
:1067b00000000000000000000000000000000000d9
:1067c00000000000000000000000000000000000c9
:1067d00000000000000000000000000000000000b9
:1067e00000000000000000000000000000000000a9
:1067f0000000000003c0000003c0000003c0000050
:1068000003c0000003c0000003c00000ffff000041
:10681000ffff0000ffff0000ffff000003c00000bb
:1068200003c0000003c0000003c0000003c000005c
:1068300003c0000000000000000000000000000095
:106840000000000000000000000000000000000048
:106850000000000000000000000000000000000038
:106860000040000000c0000001c0000003c00000a4
:1068700007c000000fc000001fc000003fff000065
:106880007fff00003fff00001fc000000fc000009e
:1068900007c0000003c0000001c0000000c00000ed
:1068a00000400000000000000000000000000000a8
:1068b00000000000000000000000000000000000d8
:1068c00000000000000000000000000000000000c8
:1068d00000000000000000000000000000000000b8
:1068e000000000000000000000000000ffff0000aa
:1068f000ffff0000ffff000000000000000000009c
:106900000000000000000000000000000000000087
:106910000000000000000000000000000000000077
:106920000000000000000000000000000000000067
:106930000000000000000000000000000000000057
:106940000000000000000000001e0000001e00000b
:10695000003e0000007c000000f80000fff0000096
:10696000ffe00000ffc00000000000000000000089
:106970000000000000000000000000000000000017
:106980000000000000000000000000000000000007
:1069900000000000000000000000000000000000f7
:1069a00000000000010000000100000001000000e4
:1069b00003800000038000000380000007c0000087
:1069c00007c0000007c000000fe000000fe000005b
:1069d0000fe000001ff000001ff000001ff000009b
:1069e0003ff800003ff800003ff800007ffc000087
:1069f0007ffc00007ffc0000fffe0000fffe0000a7
:106a0000fffe000000000000000000000000000089
:106a10000000000000000000000000000000000076
:106a20000000000000000000000000000000000066
:106a300000000000e0000000fc000000ff800000fb
:106a4000fff00000ff800000fc000000e0000000fc
:106a50000000000000000000000000000000000036
:106a60000000000000000000000000000000000026
:106a70000000000000000000000000000000000016
:106a80000000000000000000000000000000000006
:106a9000000000000e0000000fc000000ff8000012
:106aa0000fff00000fff00000fff00000fff0000ae
:106ab0000fff00000fff00000fff00000fff00009e
:106ac0000fff00000ff800000fc000000e000000d4
:106ad00000000000000000000000000000000000b6
:106ae00000000000000000000000000000000000a6
:106af0000000000000000000000000000000000096
:106b00000000000000000000000000000000000085
:106b10000000000000070000003f000001ff00002f
:106b20000fff000001ff0000003f00000007000011
:106b30000000000000000000000000000000000055
:106b40000000000000000000000000000000000045
:106b50000000000000000000000000000000000035
:106b60000000000000000000000000000000000025
:106b7000000000000070000003f000001ff00000a3
:106b8000fff00000fff00000fff00000fff0000049
:106b9000fff00000fff00000fff00000fff0000039
:106ba000fff000001ff0000003f000000070000084
:106bb00000000000000000000000000000000000d5
:106bc00000000000000000000000000000000000c5
:106bd00000000000000000000000000000000000b5
:106be00000000000000000000000000001000000a4
:106bf000010000000100000003800000038000008d
:106c00000380000007c0000007c0000007c00000ac
:106c10000fe000000fe000000fe0000000000000a7
:106c20000000000000000000000000000000000064
:106c30000000000000000000000000000000000054
:106c40000000000000000000000000000000000044
:106c50000000000000000000000000000fe0000045
:106c60000fe000000fe0000007c0000007c00000b8
:106c700007c00000038000000380000003800000c4
:106c80000100000001000000010000000000000001
:106c900000000000000000000000000000000000f4
:106ca00000000000000000000000000000000000e4
:106cb00000000000000000000000000000000000d4
:106cc000000f000000180000003000001fff00004f
:106cd00018070000180f000018180000181900000d
:106ce0001833000018330000183300001833000078
:106cf00018190000181800001fff000018070000f6
:106d00001fff00001fff00001fff00000000000029
:106d10000000000000000000000000000000000073
:106d20000000000000000000000000000000000063
:106d3000f0000000180000000c000000fff8000048
:106d4000e0180000f0180000181800009818000063
:106d5000cc180000cc180000cc180000cc180000a3
:106d60009818000018180000fff80000e018000054
:106d7000fff80000fff80000fff80000000000002e
:106d80000000000000000000000000000000000003
:106d90000000000000000000000f0000003f0000a5
:106da00000ff000001f3000003c300000703000020
:106db0000e0300001c0300001c0300003803000049
:106dc0003803000038030000380300001c030000f3
:106dd0001c0300000e0300000703000003c30000b3
:106de00001f3000000ff0000003f0000000f000062
:106df0000000000000000000000000000000000093
:106e00000000000000000000000000000000000082
:106e100000000000000000000c0000000f00000057
:106e200003c0000000f00000003c0000000f000064
:106e3000000000003906000025090000250f0000b1
:106e400039e9000000000000000000000f00000011
:106e500003c0000000f00000003c0000000f000034
:106e6000000300000000000000000000000000001f
:106e70000000000000000000000000000000000012
:106e800000000000000000000fff00000fff0000e6
:106e900000000000000000000000000000000000f2
:106ea0000fff00000fff00000000000000000000c6
:106eb00000000000000000000fff00000fff0000b6
:106ec00000000000000000000000000000000000c2
:106ed00000000000000000000000000000000000b2
:106ee00000000000000000000000000000000000a2
:106ef00000000000000000000c0000000f00000077
:106f000003c0000000f00000003c0000000f000083
:106f10000c0300000f00000003c0000000f00000a0
:106f2000003c0000000f00000c0300000f000000f8
:106f300003c0000000f00000003c0000000f000053
:106f4000000300000000000000000000000000003e
:106f50000000000000000000000000000000000031
:106f600000000000010000000d0000000f00000004
:106f700003c0000001f20000013e0000010f00000c
:106f80000d0300000f02000003c2000001f2000028
:106f9000013e0000010f00000d0300000f02000081
:106fa00003c2000001f20000013e0000000f0000db
:106fb00000030000000200000000000000000000cc
:106fc0000000000000000000fff80000fff80000d3
:106fd000001800000018000000180000ff980000d2
:106fe000ff980000019800000398000004180000ba
:106ff0000818000008180000081800000418000015
:10700000021800000118000001180000011800001b
:1070100002180000041800000ff800001ff800001c
:10702000e000000000000000000000000000000080
:1070300000000000000000001fff00001fff000014
:1070400018000000180000001800000019ff0000e0
:1070500019ff000019800000190000001a0000004c
:107060001c0000001c0000001c0000001a000000b2
:10707000190000001880000018800000188000002f
:10708000190000001a0000001c0000001800000099
:107090001fff0000000000000000000000000000d2
:1070a00000000000000000000000000000000000e0
:1070b00000000000000000000000000000030000cd
:1070c000000f0000003c000000f0000003c00000c2
:1070d0000fff00000fff0000000000000000000094
:1070e000820800008208000092490000ffff0000b3
:1070f0000000000000000000000000000000000090
:10710000000000000000000000000000000000007f
:1071100000000000000000001fff00001e00000033
:107120001e0000001e0000001e0000001e000000e7
:107130001e0000001e0000001e0000001e000000d7
:107140001e0000001e0000001e0000001fff0000c7
:107150001fff00001fff00001fff00001fff0000b7
:107160001fff00001fff00000fff000007ff0000cf
:10717000000000000000000000000000000000000f
:107180000000000000000000fff800000078000090
:10719000004800000048000000780000007800006f
:1071a00000780000007800000078000000780000ff
:1071b000007800000078000000780000fff8000070
:1071c000fff80000fff80000fff80000f078000072
:1071d000f0780000f0780000f0780000fff8000080
:1071e000000000000000000000000000000000009f
:1071f00000000000fffe0000fffe0000fffe000098
:107200007ffc00007ffc00007ffc00003ff80000d6
:107210003ff800003ff800001ff000001ff00000e2
:107220001ff000000fe000000fe000000fe0000082
:1072300007c0000007c0000007c000000380000076
:107240000380000003800000010000000100000036
:10725000010000000000000000000000000000002d
:10726000000000000000000000000000000000001e
:10727000000800000008000000080000012a0000cb
:1072800000aa0000005d000001ff0000007f000078
:107290000fff0000007f000001ff0000005d000004
:1072a00000aa0000012a00000008000000080000f9
:1072b00000080000000000000000000000000000c6
:1072c00000000000000000000000000000000000be
:1072d00000000000000000000000000000000000ae
:1072e000000000000000000000000000400000005e
:1072f0008000000000000000a0000000000000006e
:10730000fff0000000000000a000000000000000ee
:1073100080000000400000000000000000000000ad
:10732000000000000000000000000000000000005d
:10733000000000000000000000000000000000004d
:10734000000000000000000000000000000000003d
:10735000000000000000000000000000000000002d
:10736000000000000000000000000000000000001d
:107370000fff0000000000000000000000000000ff
:10738000820800008208000092490000ffff000010
:1073900000000000000000000000000000000000ed
:1073a00000000000000000000000000000000000dd
:1073b00000000000000000000000000000000000cd
:1073c00000000000000000000000000000000000bd
:1073d00000c00000030000000c00000030000000ae
:1073e000c0000000000000000000000000000000dd
:1073f000208200002082000024920000fffe000096
:10740000000000000000000000000000000000007c
:10741000000000000000000000000000000000006c
:10742000000000000000000000c0000003c00000d9
:107430000f0000003c000000f4000000c20000004b
:107440000200000002000000020000000400000032
:10745000fff00000fff0000000000000000000004e
:10746000208200002082000024920000fffe000025
:10747000000000000000000000000000000000000c
:1074800000000000000000000000000000000000fc
:1074900000000000000000000000000000000000ec
:1074a00000000000000000000fff00000fff0000c0
:1074b00000000000080400000c0c00000e1c00007e
:1074c0000f3c00000dec00000ccc00000c0c000088
:1074d0000c0c0000000000000fff00000fff000078
:1074e000000000000000000000000000000000009c
:1074f000000000000000000000000000000000008c
:10750000000000000000000000000000000000007b
:107510000000000007f000000ff80000180c000049
:107520003006000060030000c00100008000000081
:10753000000000000000000000000000000000004b
:10754000000000000000000000000000000000003b
:10755000000000000000000000000000000000002b
:10756000000000000000000000000000000000001b
:10757000000000000000000000000000000000000b
:1075800002000000030000000380000003c00000b0
:1075900003e0000003f0000003f80000fffc00001f
:1075a000fffe0000fffc000003f8000003f00000f5
:1075b00003e0000003c0000003800000030000009f
:1075c00002000000000000000000000000000000b9
:1075d00000000000000000000000000000000000ab
:1075e0001eb20000253000003464000000300000ae
:1075f000393000003500000037350000303200001f
:10760000300000003735000030320000310000004b
:1076100025310000307300000025000030320000ea
:107620006425000030320000642500003034000082
:107630006425000030320000642500003032000074
:107640006425000030320000640000002530000096
:1076500033640000003000003134000031250000a8
:1076600030330000640000002573000000000000bb
:107670002530000032580000003a0000253000009c
:10768000325800002530000032580000253000003c
:107690003458000025300000345800000025000058
:1076a00030320000580d00000a0000002563000081
:1076b00000000000253000003258000000170000d4
:1076c0000025000073250000630000002530000045
:1076d00034640000000000002e2e00000020000096
:1076e000202000002020000020200000202000009a
:1076f0002020000000000000303100003233000084
:1077000034350000363700003839000041420000af
:107710004344000045460000303100003233000091
:10772000343500003637000038390000414200008f
:107730004344000045460000302f000033000000a5
:020000040000fa
:020000040002f8
:10774000881f7800004478002102200000002800f3
:1077500044e6020000000000a0e602000000000075
:107760005ce6020000000000e0cdb3008ce6020001
:10777000000000005ce602000000000000000000c5
:1077800000000000000000009121200091407800de
:1077900000c8b30000c06000fbff3a008ce60200a6
:1077a000000000005ce60200000000001942e20058
:1077b000feff3500084078008ce602000000000063
:1077c0005ce60200000000001942e200feff350006
:1077d000a0e60200000000005ce6020000000000dd
:1077e000f0cdb3008ce60200000000005ce6020071
:1077f000000000001942e200feff35007ce60200b6
:107800000000000000447800a4e602000000000030
:107810005ce602000000000050e6020000000000ec
:1078200008007800000fb2004400de006a00b900d2
:107830006f416400004041000080fb004f0478006d
:1078400000000600889fbe00804478000180fb0095
:10785000a2002000811f7800110009000280d800da
:10786000cf0078000080fb006a01b90082c05000a0
:10787000efc060004400dd0000c470002102200061
:107880000000280044e6020000000000a0e602001c
:10789000000000005ce6020000000000e0cdb30044
:1078a0008ce60200000000005ce602000000000020
:1078b000912120009140780000c8b30000c0600012
:1078c000fbff3a008ce60200000000005ce60200cc
:1078d000000000001942e200feff3500f0c3b300d3
:1078e0008ce60200000000005ce6020000000000e0
:1078f00020c0b3008ce60200000000005ce602003d
:10790000000000001942e200feff3500a4e602007c
:10791000000000005ce6020000000000a0e602009b
:10792000000000005ce6020000000000e0cdb300b3
:107930008ce60200000000005ce60200000000008f
:10794000912120009140780000c8b30000c0600081
:10795000fbff3a008ce60200000000005ce602003b
:10796000000000001942e200feff3500f0c3b30042
:107970008ce60200000000005ce60200000000004f
:1079800060c0b3008ce60200000000005ce602006c
:10799000000000001942e200feff3500a4e60200ec
:1079a000000000005ce6020000000000a0e602000b
:1079b000000000005ce6020000000000e0cdb30023
:1079c0008ce60200000000005ce6020000000000ff
:1079d000912120009140780000c8b30000c06000f1
:1079e000fbff3a008ce60200000000005ce60200ab
:1079f000000000001942e200feff35000940780057
:107a00008ce60200000000005ce6020000000000be
:107a10001942e200feff3500084078008ce60200c3
:107a2000000000005ce60200000000001942e200d5
:107a3000feff3500a4e60200000000005ce6020044
:107a40000000000050e60200000000004f04be00ed
:107a50000000060012538000e30f510002003200c4
:107a6000e60f510002003a0081ce200005003700e9
:107a7000e10f510002003200e40f510003003a0010
:107a800091ce2000a0ce200011487800a0ce20008a
:107a900010407800e34f50004e00320005003c00db
:107aa000e14f50001b003200e24f500006003a0048
:107ab00034003700e54f500082003200600035008e
:107ac000e64f50008800320010a9200011c4b30016
:107ad000014878008040eb001140980080538000fe
:107ae0000000e00003003200e30f500003003a0002
:107af00006003700900328000100370030042800fa
:107b0000109088000090880000000600d004280033
:107b1000fbff37008353800080052800ea8f510067
:107b200001003200000628001090880010a92000f3
:107b300081c5b300014878008040eb0011409800f7
:107b4000e60f510075003e00100020008200dd00ad
:107b500001007800c006b20005003a0072806000a3
:107b60006e003200ea8f51003100320032003700df
:107b70000300e0004d003200e38f51004d003a0059
:107b80004e00370011a9200020c4b30080487800bf
:107b900076404000904098000040eb00a0409800e4
:107ba0008006280010908800e60f51005b003e0020
:107bb000100020008200dd00010078008004b20087
:107bc00034003a00010078006003b2005300320034
:107bd0001400370010a92000c1c4b3000148780088
:107be0008040eb0011409800330728001390880074
:107bf000e60f510049003e00100020008200dd0029
:107c000001007800a005b20004003a0001007800ed
:107c10004002b20003003a00000006000390880012
:107c20000000060080538000ea0f500002003a0076
:107c300080052800b3ff370000062800b1ff370099
:107c4000900728001090880011a9200020c4b300dc
:107c5000804878006a404000904098000040eb0067
:107c6000a0409800e60f51002c003e0010002000bc
:107c70008200dd00010078008004b20005003a00b7
:107c8000010078006003b2002400320030072800b1
:107c90009cff3700805380000000e00003003200aa
:107ca000e30f500003003a0004003700900328005f
:107cb00094ff37003004280092ff3700d0042800da
:107cc00090ff3700210828001190880010a920009b
:107cd0000048eb000200e900e50f50000f003e00f5
:107ce0000190880000000600b30828001390880067
:107cf00011a9200020c4b3008048780076404000dd
:107d0000904098000040eb00a04098000200e9007d
:107d1000e50f500001003e000390880000000600bf
:107d2000889fbe008a9fbe008c1f780000057800e7
:107d30008104780002467800502421001a48780017
:107d40000a047800060037008900780002407800b5
:107d5000c69e020002000000d84d78008904e800a9
:107d60005b2421001b417800ed4f510005003200db
:107d70000204e000030032000a4054008c4f50001f
:107d8000f1ff3500502421000048eb008900780005
:107d90000040eb00c69e0200020000004f06780083
:107da0004f05be004f04be00000006001421ef0086
:107db00000e82300d0088800b1c0a800b1a0a90045
:107dc000b180a9008760a9009760a8001fe1a80002
:107dd00000000600889fbe0080c320008080eb006a
:107de000908f100011003a000000eb000b003700ec
:107df0008000400000c120006100780082c32000a4
:107e0000803079002210220082804000229f0200f0
:107e100002000000309280000000e80030928800ec
:107e200030928000f30f5000f1ff34000000eb00af
:107e30000800370000044000201022000000440029
:107e4000369f02000200000000b47c0030928000e7
:107e50000000e800309288003092800089c3200042
:107e6000f30f5000f3ff34000000eb003092880065
:107e700089007800a3be2000220120000300370003
:107e800071b89700911950000201e9008180e80063
:107e90000200e000faff3d00505f80004200de007b
:107ea000205e8800605f8000520020001100090001
:107eb0000280d800305e8800705f800011000900e9
:107ec0000280d800405e8800300020003092880098
:107ed00005bf2000a4bc200043002000350078002e
:107ee000a2002000110009000280d800001a7800ca
:107ef0008301e900f9ff3b008300200033928800f2
:107f0000d05f800052002000110009000280d800dc
:107f1000a05e8800e05f8000110009000280d800a8
:107f2000b05e8800f05f8000110009000280d80078
:107f3000c05e880000608000110009000280d80047
:107f4000d05e880010608000110009000280d80017
:107f5000e05e880020608000110009000280d800e7
:107f6000f05e880030608000110009000280d800b7
:107f7000005f880040608000110009000280d80086
:107f8000105f880050608000110009000280d80056
:107f9000205f880060608000110009000280d80026
:107fa000305f880070608000110009000280d800f6
:107fb000405f880020bc20000048eb004f04be005a
:107fc0000000060030002000a053880000000600da
:107fd000889fbe008a1f78000004be005024210044
:107fe00000c8eb000d00370009007800fc9e02007d
:107ff00002000000004d7800ed4f500002003200fa
:10800000004c780003003700004ceb00000000003b
:10801000000000000804e8008904e8005a24210058
:108020001a407800ed4f5000020032000004e000da
:10803000edff3a004f0578004f04be000000060037
:10804000881f780040242200fc9e020002000000ed
:1080500048242200e14f40000c003a0088007800dc
:1080600000c3b300c69e02000200000000c3b300bc
:1080700041bf2e0080707c000804e800a02422008c
:10808000800f54000a003200f4ff37000800780027
:10809000fc9e02000200000041bf2e0080707c00a8
:1080a0000804e800a0242200800f5400f7ff3a00e3
:1080b0004f0478000000060020002000a053880034
:1080c0000000060050f68000cf80de00c08f8800e0
:1080d000d18f880042ce200003002000f0da020099
:1080e000000000004609dd004a00de0000007100cb
:1080f000ca08de00928f80004412de0004015100a5
:1081000000014100928f88004411de00030020002e
:10811000a28f8800b38f8800808f8000c400de00ab
:108120000100500002004000808f88004400de0003
:10813000608f8800708f88000000060060002000bb
:10814000a053880000000600889fbe008a9fbe00e2
:108150008c1f780000c3b30079fd07006c15210067
:10816000004e780010c3b30075fd07005a152100ba
:10817000004d780020c3b30071fd070048152100b1
:10818000004c780030c3b3006dfd07003b152100a3
:10819000804d780040c3b30069fd07002915210018
:1081a000804c780050c3b30065fd07000080fb00e1
:1081b000017d200001004000808a8800c0c0b3001b
:1081c000984f100001003a00004ceb0000c2b300d1
:1081d000984f100002003a00c0c0b300004c780075
:1081e0009840780075c05000ea4f500001003e00f2
:1081f00068cc50001c80fb00801f78001a80fb00b8
:10820000801f78001880fb00801f7800100928006c
:10821000801f7800d0162100b4ab020000000000df
:108220005011f8001980fb00801f78001b80fb00b4
:10823000801f7800000a2800801f78002016210087
:10824000b4ab020000000000f0875700e05380004c
:10825000e10f500017003200e0312a002a780200b6
:1082600002000000f0772d00d000890003022000fa
:108270004210200051002000d00c2000585702006e
:10828000020000000000eb00d0008900d21621009f
:1082900091002000200d2000e27802000200000082
:1082a0002216210051012000d00c2000e2780200ab
:1082b000020000004f0678004f05be004f04be00cc
:1082c0000000060000037800814378000202780075
:1082d0008000eb0000c2b30000f278008100e800eb
:1082e000e58f5000fbff3a000704e00005003a006c
:1082f00070404000004a780000c0e9001042980039
:108300000482e800823e2000110009000203d80028
:10831000800178000300fb000280b90000035300d5
:108320000304e0000300320000c3b30000da4100a0
:1083300004003700e1cf530002003c0000c3b3004b
:10834000005a7800e1cf530002003a00e0c2b300c7
:10835000005a780042062000110009000203d800ec
:10836000800178000300fb000280b9000003530085
:108370000304e0000300320000c3b30000da410050
:1083800004003700e2cf530002003c0000c3b300fa
:10839000005a7800e2cf530002003a00e0c2b30076
:1083a000005a7800a2002000110009000203d80042
:1083b000000178000200fb006a00b9008000530051
:1083c0000204e0000300320000c3b300005a410081
:1083d00004003700e3cf530002003c0000c3b300a9
:1083e000005a7800e3cf530002003a00e0c2b30025
:1083f000005a78000100e0000300320000c3b3001f
:1084000000ca400000000600e4cf530002003c0018
:1084100000c3b300004a78000000060030ff2000cf
:108420009040780020ff20001040780080cf50005e
:10843000030036008181fb000080fb000400370050
:1084400080cf5000080031008081fb000180fb00dc
:1084500000805100420620000280b900110009008e
:108460000300d800010037000000eb00807f880087
:10847000817f800030062000808f500006003e0083
:1084800044062000048ab900c2d8200021c0b300ed
:10849000040078008bff3700c1d8200010c3b30060
:1084a000804878000040e90090409800a040980083
:1084b00000c0e900b0409800000006000024210040
:1084c00090407800f02321001040780080cf5000c9
:1084d000030036008181fb000080fb0004003700b0
:1084e00080cf5000080031008081fb000180fb003c
:1084f00000805100420620000280b90011000900ee
:108500000300d800010037000000eb00c0b4880071
:10851000c1b4800030062000808f500006003e006d
:1085200044062000048ab90052d9200021c0b300bb
:108530000400780063ff370051d9200010c3b30056
:10854000804878000040e90090409800a0409800e2
:1085500000c0e900b040980000000600e0232100c0
:108560009040780070da20001040780080cf5000f2
:10857000030036008181fb000080fb00040037000f
:1085800080cf5000080031008081fb000180fb009b
:1085900000805100420620000280b900110009004d
:1085a0000300d800010037000000eb00d0b48800c1
:1085b000d1b4800030062000808f500006003e00bd
:1085c00044062000048ab900e2d9200021c0b3008b
:1085d000040078003bff3700e1d9200010c3b3004e
:1085e000804878000040e90090409800a040980042
:1085f00000c0e900b040980000000600881f780025
:1086000048ff200018407800f540500010c8b30023
:1086100080cf500017003e0020a120001004e00091
:1086200014003a0000062000fafb020000000000df
:10863000800178001881fb00a0e520009080fb00fd
:108640000100e900800f5100040035000100e8003e
:10865000017e2000800f51000100340001802f00b6
:10866000c08d8000510098003300900000e0a00011
:10867000b00198004f0478000000060010002000b0
:10868000a05388000000060070002000a05388005e
:1086900000000600d153800040022000808f50006f
:1086a0002e00320013003e00a0002000ec8f50008e
:1086b0003700320006003e000000eb00e38f500060
:1086c00033003200e98f50001e003a001f003700cf
:1086d00030012000f58f50002d003200c001200035
:1086e000fe8f50002a003200f28f500015003a0031
:1086f0001800370090032000808f50001f003200c8
:1087000007003e0066005000808f500019003200c4
:1087100063004000808f50000a003a0011003700cb
:1087200030042000808f50001600320066004000a8
:10873000808f5000150032006d005000808f500077
:108740000a003200400020001100370070002000b5
:108750000f003700000120000d003700200220002c
:108760000b0037004003200009003700a003200061
:1087700007003700100320000500370070032000b9
:1087800003003700000420000100370070042000bf
:10879000e05388000000060011017800ec0f510042
:1087a00011003200ed0f510003003200eb0f5100b9
:1087b0002b003a0005003700e60f500028003a0071
:1087c00070002000e053880025003700e60f5000bd
:1087d00023003a00d0002000e053880020a12000b0
:1087e0000048eb001e003700e60f50001c003a0066
:1087f000a0032000e053880000a220000048eb0006
:1088000011c0b30020a120000148780050032100ce
:108810000048eb00f0022100014878000000eb0066
:1088200030928800a1ba2000020078008058eb0046
:108830000000e900fdff3b00d000200030928800de
:1088400060a820000048eb00801d21000048eb00dc
:1088500070a820000048eb000080240030598800f8
:108860001000050091007800ee8f50001b003200d0
:1088700006003e00ec8f50001000320013003e0056
:10888000eb8f50002c003a0008003700f08f5000aa
:108890001d00320015003900f18f50001e0032001b
:1088a000f28f500024003a001f003700e60f5000fe
:1088b00021003a00a00020001e003700e60f500003
:1088c0001d003a00000120001a003700e60f50009a
:1088d00019003a003001200016003700e60f500062
:1088e00015003a00c001200012003700e60f5000ca
:1088f00011003a00b0052000e053880010a22000cb
:108900000048eb000c003700e60f50000a003a0068
:108910007c00400007003700e60f500006003a00d8
:108920004000200003003700e60f500002003a002c
:10893000f0012000e053880010000500910078004d
:1089400092022000828f50000d00320006003e008f
:10895000eb8f50001200320080022000808f500008
:1089600013003a0004003700a0022000808f50005e
:108970000f003a0008003700100020000100370007
:108980000000eb008053880011042200c69e020004
:10899000020000000600370030002000f9ff370019
:1089a000e60f500002003a0070002000e0538800fb
:1089b000100005000001780091007800e00220001e
:1089c000808f50001100320009003e006600500008
:1089d000808f50001f0032000000e800808f5000a0
:1089e00021003200eb8f500028003a0023003700ae
:1089f000f0022000808f5000070032000000e800e5
:108a0000808f500021003a000d0037002000200028
:108a100040538800060037000000eb0040538800f8
:108a200002a62e0003002000627288007372880084
:108a300001042200c69e020002000000130037005d
:108a40001000200040538800023e2900430020000f
:108a5000f5ff370010c0b300d180200080487800b7
:108a600081032200f3ff3700d08020000048eb0094
:108a7000810322000040eb00eeff3700e60f5100bb
:108a800002003a0070002000e0538800100005004a
:108a9000b2002000910f110006003a00e60f5000ce
:108aa00004003a0070002000e05388000000eb0052
:108ab0002053880010000500889fbe0091007800b8
:108ac000ee8f50000201320006003e00ec8f500095
:108ad0005100320075003e00eb8f50000b013a0050
:108ae0001600370082022000828f50000b003200f7
:108af00003003e00f08f500004013a00ff003700f1
:108b000090022000808f5000060032000000e80034
:108b1000808f5000fd003a000600370011c0b300fe
:108b20000100370021c0b30050ce2000014878007a
:108b3000f600370031c0b300fbff3700e60f5000ee
:108b4000f2003a0011538000e68f5000ef003e0023
:108b5000100020008100dd00010078004002b2001a
:108b600011003a00010078008004b2001e003a00b3
:108b700072806000e500320011092200d0d620008a
:108b800010407800c69e0200020000007109220019
:108b900090d5200010407800c69e02000200000020
:108ba000a10922000b00370021092200d0d62000a5
:108bb00010407800c69e02000200000081092200d9
:108bc00090d5200010407800c69e020002000000f0
:108bd000b109220010d4200010407800c69e020087
:108be00002000000c900370031092200d0d6200061
:108bf00010407800c69e0200020000009109220089
:108c000090d5200010407800c69e020002000000af
:108c1000c1092200efff3700e60f5000bb003a0009
:108c200050ce200010407800e24f50000d0032007e
:108c3000e34f500014003200e14f5000b3003a00ff
:108c4000d2d620009240780020c3b30080cf5000dd
:108c5000020036000149e9002700370060c9b3006f
:108c60002400370092d520009240780020c3b30042
:108c700080cf5000020036000149e900450037006e
:108c800060c9b3004200370012d42000924078003f
:108c900020c3b30080cf5000020036000149e90034
:108ca0006300370060c9b30060003700e60f500072
:108cb00096003a0050ce200010407800e24f50005d
:108cc0002b003200e34f500050003200e14f5000c3
:108cd0008e003a00d2d620009240780050c9b300ee
:108ce00080cf500002003e000149e800020037003a
:108cf00020c3b30000497800d0d62000104478008b
:108d00000800fb00cf80de003adb0200000000001c
:108d10000804e00004003d000200200003382400a5
:108d200092db0200000000000001be0000002000f5
:108d3000812c24004cdc020000000000d06b880075
:108d4000e16b8800809fbe00f00a2800801f780039
:108d500040232100b4ab02000000000049232100a1
:108d60000040eb00d0449800000520004d00370083
:108d700092d520009240780050c9b30080cf5000b7
:108d800002003e000149e8000200370020c3b300a2
:108d90000049780090d52000104478000800fb00be
:108da000cf80de003adb0200000000000804e00093
:108db00004003d00020020000338240092db020082
:108dc000000000000001be0000002000812c2400f3
:108dd0004cdc020000000000306b8800416b880012
:108de000809fbe00f00a2800801f7800a02221008a
:108df000b4ab020000000000a92221000040eb00fb
:108e0000d0449800b00520002600370012d420007e
:108e10009240780050c9b30080cf500002003e005d
:108e20000149e8000200370020c3b3000049780080
:108e300010d42000104478000800fb00cf80de0032
:108e40003adb0200000000000804e00004003d00de
:108e5000020020000338240092db02000000000022
:108e60000001be0000002000812c24004cdc020028
:108e700000000000706a8800816a8800809fbe0040
:108e8000f00a2800801f780000222100b4ab020005
:108e900000000000092221000040eb00d0449800af
:108ea000c0052000fafb020000000000000478006a
:108eb000890078004c910200020000003800900008
:108ec00000e0a00030049800e68757000f0037004c
:108ed000e60f50000d003a00105380000000e8003b
:108ee00010538800e40f500002003a0010002000e8
:108ef000105388006001200003003700e60f500087
:108f000002003a007f004000e0538800100020007b
:108f10004f04be000000060091007800ee8f500064
:108f20002500320003003e00eb8f50002a003a007b
:108f300007003700b0022000808f50000e00320082
:108f40000000e800808f500023003a001300370033
:108f5000e60f500020003a000000eb00b06e8800e1
:108f6000a06e880011c0b300a0dc2000014878008a
:108f7000c012200017003700e0a720000048eb00d7
:108f8000711020000040eb00c69e020002000000ad
:108f900090012000e05388000f00370010c0b3009c
:108fa000e1a720008048780071102000c69e0200d2
:108fb0000200000008003700e60f500006003a00eb
:108fc0007f004000e0538800a0dc20000048eb0058
:108fd00000192000406e8800100005009100780004
:108fe000e2022000828f50000a00320005003e009d
:108ff000eb8f50000f003200ec8f50001c003a0045
:1090000017003700f0022000808f500018003a004f
:10901000020037000000eb000100370010002000c4
:109020005053880031042200c69e02000200000056
:109030000f003700e60f50000d003a00200020001e
:109040006053880011c0b30000e22000014878009e
:109050000000eb00e0538800307288000400370005
:10906000e60f500002003a0070002000e053880034
:1090700010000500889fbe008a9fbe008c1f7800ec
:109080009100780082022000828f50001700320089
:109090000b003e00ee8f50008600320003003e00c1
:1090a000eb8f50002f013a001c003700ef8f50006b
:1090b000b7003200fe8f50002a013a0076003700d8
:1090c000a0022000808f50000e00320009003900fd
:1090d0000000e800808f50000c0032000000e80023
:1090e000808f50001f013a000a00370011c0b30002
:1090f0000100370021c0b30050ce200001487800a5
:109100001901370031c0b300fbff370041c0b30085
:10911000f9ff370051c0b300f7ff3700e60f5000ea
:1091200011013a0099852000c0c0b300994f10008a
:1091300002003a0074404000804c78001904e000be
:1091400002003a00c0c0b300804c7800994078001b
:109150006dc05000ea4f500001003e00e8cc4000d6
:10916000808520009040780010c3b300b5f9070057
:109170009940780020c3b300b2f90700f1428000a3
:1091800030c3b300aff90700e142800040c3b30031
:10919000acf90700d14280000143b00050c3b300d6
:1091a000a8f9070001c1b30060c3b300a5f9070027
:1091b00010c3b30062f907005b152100804d7800f1
:1091c00020c3b3005ef9070048152100004c780069
:1091d00030c3b3005af907003c152100004e780057
:1091e00040c3b30056f907002a152100004d78004e
:1091f00050c3b30052f907000080fb00017d20003e
:1092000001004000808a8800c0c0b300984f100061
:1092100001003a00004ceb0000c2b300984f100070
:1092200002003a00c0c0b300004c780098407800bb
:1092300075c05000ea4f500001003e0068cc50005d
:109240001880fb00804c78009b80fb00811f780019
:10925000801f7800500b2800801f7800d016210056
:10926000b4ab0200000000005011f8001a80fb00af
:10927000801f78001c80fb00801f7800000a2800f7
:10928000801f780020162100b4ab0200000000000f
:10929000ee875700b4003700e60f5000b2003a00e6
:1092a00070022000d053880070002000e053880036
:1092b000ad003700e60f5000ab003a0050ce200062
:1092c00010407800e34f50001a00320005003c00c7
:1092d000e14f500008003200e24f5000a2003a0077
:1092e0000d003700e44f500018003200e54f5000e9
:1092f0009d003a001d003700f04280000000e800a9
:10930000f042880001022000810f500037003a002f
:109310001000200034003700e04280000000e80028
:10932000e0428800ed0f500042003a00100020009b
:109330003f003700d04280000000e800d0428800a3
:10934000801f7800400c28004b00370091852000da
:1093500011407800f64f500002003e008048e800bf
:10936000570037008048eb00550037008285200009
:109370009240e80001497800c0c3b30080cf50009c
:1093800001003a000049eb001280fb006200370048
:10939000e60f500074003a0050ce200010407800d4
:1093a000e34f50002f00320005003c00e14f500019
:1093b00008003200e24f50006b003a0017003700ff
:1093c000e44f500036003200e54f500066003a008e
:1093d00049003700f04280000000e900f0428800b8
:1093e00002003a00f0012000f04288005e08f80018
:1093f000f00b2800801f780040182100b4ab020059
:109400000000000000052000fafb02000000000040
:1094100000047800411821004a003700e042800033
:109420000000e900e042880002003a00c00020008d
:10943000e04288005c08f800f00b2800801f7800ec
:1094400010182100b4ab020000000000b00520009d
:10945000fafb02000000000000047800111821004f
:1094600038003700d04280000000e900d042880078
:10947000801f7800f00b2800801f7800c0172100a3
:10948000b4ab020000000000c0052000fafb02009f
:109490000000000000047800c117210029003700f7
:1094a00091852000114078000004e00002003200a5
:1094b0008048e9000200370070c1b300804878009e
:1094c000908520001080fb00801f7800f00b2800a2
:1094d000801f780090172100b4ab0200000000004c
:1094e000d0052000fafb0200000000000004780014
:1094f0009117210013003700818520001140e900f9
:1095000080487800e14f400002003a00b0c3b30049
:10951000804878001180fb00801f7800f00b280045
:10952000801f780060172100b4ab0200000000002b
:10953000e0052000fafb02000000000000047800b3
:1095400061172100080078004c9102000200000021
:109550003800900000e0a00030049800e487570035
:109560000100370001003700100020004f0678008e
:109570004f05be004f04be000000060091007800b9
:10958000ed8f500003003200f28f500009003a00c6
:1095900004003700e60f500006003a007f0040004c
:1095a00003003700e60f500002003a007000200070
:1095b000e0538800100005000001be00f05180005b
:1095c0000152800044062000840f5000e08f5800b4
:1095d0005200360013007800ef0f500029003200cf
:1095e0000b003e00ec0f50001700320003003e005d
:1095f000eb0f50004a003a000d003700ed0f50000d
:1096000018003200ee0f500045003a0019003700f4
:10961000f10f5000340032001e003900f20f5000ec
:1096200035003200fe0f50003d003a003600370092
:10963000e60f51003a003a00100020001053880055
:10964000d004200033003700e60f510034003a0008
:1096500050052000e05388001000200010538800bf
:109660002f00370090012000e60f51002900320042
:109670002b00370060012000e60f5100250032006a
:109680002700370070032000e60f51002100320050
:1096900023003700e60f510021003a0000000000cf
:1096a000000000000000000052c2bf000018a3002c
:1096b0000300320000000000000000005222a90058
:1096c00000062200fc9e0200020000000080fb0059
:1096d000c072880000052000e05388007000200060
:1096e000205388000e003700b0022000e60f510022
:1096f000080032000a00370080022000e60f510007
:109700000400320006003700e60f510004003a0062
:10971000f0012000e053880001003700000006003f
:109720001000050091007800f2022000828f5000a6
:10973000250032000d003e00f28f50004f00320035
:1097400003003e00eb8f500050003a004700370006
:10975000a0022000808f50000f0032006400400003
:10976000808f500049003a000d00370010032000a0
:10977000808f50002b003200200039000000e800ec
:10978000808f5000340032000000e800808f5000cd
:109790003e003a0033003700500020002f00370011
:1097a00050cb20000048eb00d10722000040eb0026
:1097b000c69e02000200000040cb20000048eb00e3
:1097c000b09720000700370010c0b30051cb200035
:1097d00080487800d1072200c69e020002000000e7
:1097e00040cb20000048eb00010822000040eb00c5
:1097f000c69e0200020000002400370050cb20006b
:109800000048eb00d10722000040eb00c69e02009a
:109810000200000011c0b300b0972000014878009a
:10982000efff370050cb20000048eb00b09720003e
:109830000048eb00d10722000040eb00c69e02006a
:109840000200000010c0b30041cb20008048780027
:1098500001082200e6ff3700d0002000f052880007
:109860000a003700e0002000fcff3700e60f500040
:1098700006003a00f001200003003700e60f500018
:1098800002003a007f004000e0538800100005000d
:109890001000fa00889fbe008a9fbe008c1f7800cf
:1098a0009100780082022000828f50002300320055
:1098b0000b003e00ee8f50009100320003003e008e
:1098c000eb8f5000e4003a002d003700ef8f50007e
:1098d000a8003200fe8f5000df003a00d0003700b1
:1098e000c0022000808f50001800320007003e00a8
:1098f00063005000808f50000e0032000000e8002e
:10990000808f5000d4003a0007003700d0022000ba
:10991000808f50000f0032000000e800808f500060
:10992000cd003a001000370011c0b300d0a12000d4
:1099300004003700d0a120000900370011c0b30097
:1099400050ce200001487800c300370021c0b3008a
:10995000fbff3700300321000048eb0080ce2000e1
:109960000048eb00bc00370011c0b30030032100f9
:109970000148780031c0b30080ce2000f1ff3700ed
:10998000e60f5000a8003200e70f5000b2003a0086
:1099900031a1200010c0b300914f1000ae003a007a
:1099a000d0a1200022c0b300904f1100aa003200c5
:1099b0008048eb0000042000e0538800a18e800066
:1099c000007e2000d000980000402000e0009800b9
:1099d000007f2800900098000000000000000000b8
:1099e0000000000052c2bf000018a30003003200b4
:1099f00000000000000000005222a90000c3b300d4
:109a00004ff707006c152100004e780010c3b3001b
:109a10004bf707005b152100804d780020c3b30091
:109a200047f7070048152100004c780030c3b30009
:109a300043f707003a152100004d780040c3b300fa
:109a40003ff7070029152100804c780050c3b30070
:109a50003bf707000080fb00017d20000101400072
:109a6000828a8800c0c0b300984f100001003a00fd
:109a7000004ceb0000c2b300984f100002003a0007
:109a8000c0c0b300004c78009840780075c050000a
:109a9000ea4f500001003e0068cc50001c80fb00e3
:109aa000801f78001b80fb00801f78001880fb005f
:109ab000801f7800821f78001980fb00801f7800cb
:109ac0001a80fb00801f7800910c2800811f78000d
:109ad00080fd2f000f004000b4ab0200000000002a
:109ae000315980002104b000e2c0b30080fd2f0096
:109af0000f0040008af80700ee8757005600370035
:109b0000e60f500054003a00f051800001528000ee
:109b1000ea0f5000e08f58004f0036006000b80098
:109b2000f05188000152880050ce200022c0b300be
:109b3000904f110048003a0011f72000f0c4b30024
:109b4000914f100002003e006940500001003700b4
:109b5000a0c5b3008048780019f7200019407800ac
:109b6000fac4b3008a4f50001e003e00f44c40007f
:109b70001c003700e60f500037003a00f05180001b
:109b800001528000ea0f5000e08f5800320036008a
:109b90006000b800f05188000152880050ce2000cb
:109ba00021c0b30090cf10002b003a0011f7200025
:109bb000f0c4b300914f100002003e006940500015
:109bc00001003700a0c5b3008048780019f72000d5
:109bd000194078000ac5b3008a4f500001003600d2
:109be000f44c5000e0052000fafb020000000000e9
:109bf00000047800610e2800994f150001003e0016
:109c0000210e2800080078004c910200020000009c
:109c10003800900000e0a000300498000e003700eb
:109c2000e60f500003003a0011c0b30030a120003d
:109c300044ff3700e70f500007003a0030a1200032
:109c400012c0b300904f110003003a000048eb002f
:109c5000a0032000e0538800100020004f06780089
:109c60004f05be004f04be000080fa000000060051
:109c7000889fbe0091007800ef8f500022003200d4
:109c80000b003e00ec8f50009400320003003e00b9
:109c9000eb8f500021013a003e003700ed8f50005d
:109ca000b0003200ee8f50001c013a000c0137006a
:109cb00082022000828f50000b00320003003e0021
:109cc000f08f500015013a0010013700900220007b
:109cd000808f5000060032000000e800808f5000a6
:109ce0000e013a000600370011c0b3000100370032
:109cf00021c0b30050ce2000014878000701370092
:109d000031c0b300fbff3700e60f500003013a00fb
:109d100011538000e68f50001b003e001000200011
:109d20000100dd00800078004102b2000b003a0023
:109d3000000178008204b2000e003a007200600058
:109d40001100320021c0b30020c720000148780074
:109d500010c72000024878000900370021c0b30076
:109d600020c720000148780010c720000148780073
:109d70000300370010c720000148780021c0b3005d
:109d800000c720000148780050052000e0538800fb
:109d900002003700e60f5000e0003a00e052800079
:109da000e40f50000e00320003003e00e30f5000ad
:109db00005003a0006003700e50f500006003200ab
:109dc000e60f50000200320000302200050037008c
:109dd0000032220003003700003422000100370067
:109de00000362200e090880011538000e68f50007a
:109df000ca003e00100020008100dd000100780054
:109e00004002b20013003a00010078008004b20062
:109e100023003a0072806000c0003200e1908000b0
:109e200020c7200010407800c69e020002000000fb
:109e3000e19080008100e80010c720001040780009
